:100000009EC10000CDC10000CBC10000C9C10000ED
:10001000C7C10000C5C10000C3C10000C1C10000CC
:10002000BFC10000BDC10000BBC10000B9C10000DC
:10003000B7C10000B5C10000B3C10000B1C10000EC
:10004000AFC100000C941B4AABC10000A9C1000065
:100050000C94494AA5C10000A3C100000C94474973
:100060009FC100000C9411490C94E74899C100000D
:1000700097C1000095C1000093C1000091C100002C
:100080000C94ED498DC100008BC1000089C10000B6
:1000900087C1000085C1000083C1000081C100004C
:1000A0007FC100007DC100000C94BF4979C10000F0
:1000B00077C1000075C1000073C100000C94914924
:1000C0006FC100006DC100006BC1000069C100007C
:1000D00067C1000065C1000063C1000061C100008C
:1000E0005FC100004E414E494E495459494E46CDDC
:1000F000CCCC3D0AD7233C17B7D13877CC2B3295DF
:1001000095E6241FB14F0A000020410000C84200BC
:10011000401C4620BCBE4CCA1B0E5AAEC59D740086
:10012000407A10F35A00A0724E18090010A5D4E8C6
:100130000000E87648170000E40B54020000CA9A59
:100140003B000000E1F505000080969800000040AB
:10015000420F000000A086010000001027000000F0
:1001600000E803000000006400000000000A000036
:100170000000000100000000002C76D888DC674FEA
:100180000823DFC1DFAE59E1B1B796E5E3E453C61A
:100190003AE651997696E8E6C28426EB898C9B6212
:1001A000ED407C6FFCEFBC9C9F40F2BAA56FA5F4BC
:1001B00090055A2AF75C936B6CF9676DC11BFCE0E4
:1001C000E40D47FEF520E6B500D0ED902E03009437
:1001D0003577050080841E080000204E0A000000CC
:1001E000C80C333333330F986E12831141EF8D21D6
:1001F00014893BE65516CFFEE6DB18D1844B381B3D
:10020000F77C1D901DA4BBE424203284725E228101
:1002100000C9F124ECA1E53D2700002200250028BB
:10022000002B002E003100340002010000050108FF
:10023000010B01000020002300260029002C002FC4
:100240000032000001000003010601090100000A5C
:100250000B02090C0D0E080703040100000000004A
:10026000000000000000000000000000000000008E
:10027000000000000000000000121110000000004B
:10028000000000000000000000000000000000006E
:1002900000000000002100240027002A002D00306B
:1002A00000330001010000040107010A01010210EE
:1002B0002020080810204010204080020102010880
:1002C0000402010102040810204080804020100830
:1002D0000402018004020180402010080402010889
:1002E00004020101020408102040800102040810E9
:1002F00020408005050505070508080808020202D8
:10030000020A0A08080404040401010101010101B0
:10031000010303030303030303040707070C0C0C87
:100320000C0C0C0C0C02020202060606060606065F
:10033000060B0B0B0B0B0B0B0B00934A07581124EE
:100340001FBECFEFD1E2DEBFCDBF00E00CBF18E093
:10035000A0E0B2E0ECE0F6EC00E00BBF02C00790DA
:100360000D92AE3AB107D9F724E1AEEAB8E001C088
:100370001D92AB39B207E1F711E0CEE9D1E000E020
:1003800006C021970109802FFE010E94E061CD394E
:10039000D10780E00807A9F70E94844C0C94F5620D
:1003A0002FCE9C01803E910508F021C5FC018827D5
:1003B000E352FE4F8F4F0C94E061BD02CA02D3029C
:1003C000DC02E902F202F706F706F706F706F7067F
:1003D000FF020C031903F70626032F033803450316
:1003E0004E035703600369037203F7067B0384031C
:1003F0008D03F706F706F70696039F03A803F70693
:10040000F706B103BE03F706F706F706CB03D803DA
:10041000E503F706F203FB030404F706F706F70605
:100420000D0416041F04F7062C0439044604F706CD
:10043000F706F706530460046D04F7067A04870490
:100440009404F706F706F706A104AE04BB04F7060A
:10045000C804D104DA04F706F706F706FE040B0514
:100460001805F706250532053F05F706F706F706D6
:100470004C0555055E05F706F706F706F706F7067D
:10048000F706F706670570057905F70682058B05FF
:100490009405F706F706F7069D05AA05B705F706C2
:1004A000C405D105DE05F706F706F706EB05F805E6
:1004B0000506F70612061B062406F706F706F706DA
:1004C0002D0636063F06F706F706F706F706F70687
:1004D000F706F706F706F706F706F706E304EC0457
:1004E000F504F706F706F706F706F706F706F70628
:1004F000F706F706F706F706F706F706F706F70614
:10050000F706F706F706F706F706F706F706F70603
:10051000F706F706F706F706F706F706F706F706F3
:10052000F706F706F706F706F706F706F706F706E3
:10053000F706F706F706F706F706F706F706F706D3
:10054000F706F706F706F706F706F7064806510618
:100550005E06F7066B0674068106F706F706F706D1
:100560008E069706A406F706B106BA06C706F70672
:10057000F706F706D406DD06EA0681E090E0A0E083
:10058000B0E08093D2099093D309A093D409B0939B
:10059000D50908951092D6091092D7091092D8095A
:1005A0001092D90908951092DA091092DB0910927D
:1005B000DC091092DD09089581E090E0A0E0B0E050
:1005C0008093DE099093DF09A093E009B093E109DD
:1005D00008951092E2091092E3091092E409109232
:1005E000E509089583E090E0A0E0B0E08093E6099B
:1005F0009093E709A093E809B093E909089588E783
:1006000090E0A0E0B0E08093FE099093FF09A093F2
:10061000000AB093010A089588E790E0A0E0B0E0F6
:100620008093020A9093030AA093040AB093050AE8
:10063000089588E790E0A0E0B0E08093060A9093E8
:10064000070AA093080AB093090A089510920E0AA7
:1006500010920F0A1092100A1092110A0895109227
:10066000120A1092130A1092140A1092150A089591
:1006700081E090E0A0E0B0E08093160A9093170A22
:10068000A093180AB093190A089510921A0A1092AA
:100690001B0A10921C0A10921D0A089510921E0A3D
:1006A00010921F0A1092200A1092210A08951092A7
:1006B000220A1092230A1092240A1092250A089501
:1006C0001092260A1092270A1092280A1092290ADC
:1006D000089510922A0A10922B0A10922C0A109256
:1006E0002D0A089510922E0A10922F0A1092300AA5
:1006F0001092310A08951092360A1092370A109219
:10070000380A1092390A089510923A0A10923B0A58
:1007100010923C0A10923D0A089510923E0A1092DF
:100720003F0A1092400A1092410A089510924E0A10
:1007300010924F0A1092500A1092510A0895109286
:10074000520A1092530A1092540A1092550A0895B0
:100750001092560A1092570A1092580A1092590A8B
:10076000089581E090E0A0E0B0E08093620A909369
:10077000630AA093640AB093650A089581E090E04B
:10078000A0E0B0E08093660A9093670AA093680A9D
:10079000B093690A08958CE291E0A0E0B0E0809304
:1007A000760A9093770AA093780AB093790A08950D
:1007B0008CE291E0A0E0B0E080937A0A90937B0A0B
:1007C000A0937C0AB0937D0A08958CE291E0A0E0AA
:1007D000B0E080937E0A90937F0AA093800AB09342
:1007E000810A08951092860A1092870A1092880A48
:1007F0001092890A089510928A0A10928B0A109218
:100800008C0A10928D0A089510928E0A10928F0A07
:100810001092900A1092910A089510929E0A1092D6
:100820009F0A1092A00A1092A10A08951092A20A9B
:100830001092A30A1092A40A1092A50A089581E0CA
:1008400090E0A0E0B0E08093A60A9093A70AA0935E
:10085000A80AB093A90A089585E090E0A0E0B0E06E
:100860008093AE0A9093AF0AA093B00AB093B10AF6
:10087000089585E090E0A0E0B0E08093B20A909304
:10088000B30AA093B40AB093B50A089589E190E041
:10089000A0E0B0E08093B60A9093B70AA093B80A9C
:1008A000B093B90A089582E390E0A0E0B0E08093AD
:1008B000C60A9093C70AA093C80AB093C90A0895BC
:1008C00082E390E0A0E0B0E08093CA0A9093CB0A64
:1008D000A093CC0AB093CD0A089582E390E0A0E003
:1008E000B0E08093CE0A9093CF0AA093D00AB09341
:1008F000D10A089582E390E0A0E0B0E08093D60AA8
:100900009093D70AA093D80AB093D90A089582E3A6
:1009100090E0A0E0B0E08093DA0A9093DB0AA09325
:10092000DC0AB093DD0A089582E390E0A0E0B0E035
:100930008093DE0A9093DF0AA093E00AB093E10A65
:10094000089580E991E0A0E0B0E08093EE0A9093F2
:10095000EF0AA093F00AB093F10A089580E991E0BC
:10096000A0E0B0E08093F20A9093F30AA093F40A17
:10097000B093F50A089580E991E0A0E0B0E080939B
:10098000F60A9093F70AA093F80AB093F90A08952B
:100990001092FE0A1092FF0A1092000B1092010BA7
:1009A00008951092020B1092030B1092040B1092F8
:1009B000050B08951092060B1092070B1092080B6E
:1009C0001092090B08951092160C1092170C1092A9
:1009D000180C1092190C089510921A0C10921B0CFE
:1009E00010921C0C10921D0C089510921E0C109267
:1009F0001F0C1092200C1092210C089588E592E0B3
:100A0000A0E0B0E08093160B9093170BA093180B07
:100A1000B093190B089588E592E0A0E0B0E08093D0
:100A20001A0B90931B0BA0931C0BB0931D0B0895F6
:100A300088E592E0A0E0B0E080931E0B90931F0B3E
:100A4000A093200BB093210B08958EE190E0A0E0DD
:100A5000B0E08093260B9093270BA093280BB093C4
:100A6000290B08958EE190E0A0E0B0E080932A0B7E
:100A700090932B0BA0932C0BB0932D0B08958EE12C
:100A800090E0A0E0B0E080932E0B90932F0BA0930A
:100A9000300BB093310B089510923E0B10923F0B28
:100AA0001092400B1092410B08951092420B10923D
:100AB000430B1092440B1092450B08951092460B75
:100AC0001092470B1092480B1092490B0895109208
:100AD000660B1092670B1092680B1092690B0895C9
:100AE00010926A0B10926B0B10926C0B10926D0BA4
:100AF000089510926E0B10926F0B1092700B109263
:100B0000710B08951092760B1092770B1092780B60
:100B10001092790B089510927A0B10927B0B109221
:100B20007C0B10927D0B089510927E0B10927F0B20
:100B30001092800B1092810B089585E090E0A0E068
:100B4000B0E080938E0B90938F0BA093900BB0939B
:100B5000910B089585E090E0A0E0B0E08093920BC7
:100B60009093930BA093940BB093950B089585E00D
:100B700090E0A0E0B0E08093960B9093970BA09349
:100B8000980BB093990B089584EB95E1A0E0B0E049
:100B900080939E0B90939F0BA093A00BB093A10BFF
:100BA000089584EB95E1A0E0B0E08093A20B9093D0
:100BB000A30BA093A40BB093A50B089584EB95E130
:100BC000A0E0B0E08093A60B9093A70BA093A80B96
:100BD000B093A90B089585E090E0A0E0B0E0809389
:100BE000B60B9093B70BA093B80BB093B90B0895C5
:100BF00085E090E0A0E0B0E08093BA0B9093BB0B4F
:100C0000A093BC0BB093BD0B089585E090E0A0E0ED
:100C1000B0E08093BE0B9093BF0BA093C00BB0933A
:100C2000C10B08951092C60B1092C70B1092C80BFF
:100C30001092C90B08951092CA0B1092CB0B109210
:100C4000CC0B1092CD0B08951092CE0B1092CF0BBF
:100C50001092D00B1092D10B08951092DE0B1092CF
:100C6000DF0B1092E00B1092E10B08951092E20B53
:100C70001092E30B1092E40B1092E50B0895109282
:100C8000E60B1092E70B1092E80B1092E90B089517
:100C90001092F60C1092F70C1092F80C1092F90CBE
:100CA00008958CE390E0A0E0B0E08093FA0C90937C
:100CB000FB0CA093FC0CB093FD0C089581E090E038
:100CC000A0E0B0E08093FE0C9093FF0CA093000D89
:100CD000B093010D08951092060D1092070D109219
:100CE000080D1092090D08958CE390E0A0E0B0E0AB
:100CF00080930A0D90930B0DA0930C0DB0930D0DE6
:100D0000089581E090E0A0E0B0E080930E0D909314
:100D10000F0DA093100DB093110D089510921E0D9C
:100D200010921F0D1092200D1092210D08958CE34A
:100D300090E0A0E0B0E08093220D9093230DA0936B
:100D4000240DB093250D089581E090E0A0E0B0E07F
:100D50008093260D9093270DA093280DB093290D15
:100D6000089510922E0D10922F0D1092300D1092AA
:100D7000310D08958CE390E0A0E0B0E08093320D57
:100D80009093330DA093340DB093350D089581E009
:100D900090E0A0E0B0E08093360D9093370DA093E3
:100DA000380DB093390D08951092460D1092470DED
:100DB0001092480D1092490D08958CE390E0A0E048
:100DC000B0E080934A0D90934B0DA0934C0DB093DF
:100DD0004D0D089581E090E0A0E0B0E080934E0DCD
:100DE00090934F0DA093500DB093510D0895220F85
:100DF000331F220F331FF901EE52F64F108211827A
:100E0000128213820895883591050CF04BC0853508
:100E10009105CCF4803391054CF58D3291059CF40D
:100E20008C319105BCF4893191056CF48E309105BB
:100E300064F48B3091053CF4009729F097FD08C0CD
:100E40000297049728F481E008950F970997D8F343
:100E500080E00895863291053CF4843291059CF738
:100E60004F970397A8F7EFCF8997FBCF843491056D
:100E70006CF4813491053CF78A3391052CF4873367
:100E800091050CF7C397EDCFCD97EBCF8E3491053D
:100E900034F48B349105BCF687549109E2CF815527
:100EA0009109DFCF863891051CF5833891055CF6F2
:100EB0008237910584F48F3691052CF6883691059A
:100EC0003CF4853691050CF0BECF8B559109C9CF06
:100ED00089569109C6CF8C3791053CF48937910525
:100EE0000CF0B1CF83579109BCCF8D579109B9CF81
:100EF000803D91058CF48D3C91050CF0A4CF843994
:100F000091053CF4813991050CF09DCF8D589109E4
:100F1000A8CF895C9109A5CF8A3D91053CF4873D16
:100F200091050CF090CF835D91099BCF8D5D910968
:100F300098CFAF92BF92CF92DF92EF92FF920F9332
:100F40001F93CF93DF936C017B018B01040F151F5F
:100F5000EB015E01AE18BF08C017D10759F06991C7
:100F6000D601ED91FC910190F081E02DC60119951B
:100F7000892B79F7C501DF91CF911F910F91FF90D8
:100F8000EF90DF90CF90BF90AF900895FC01538D0C
:100F9000448D252F30E0842F90E0821B930B541753
:100FA00010F0CF96089501970895FC01918D828DE0
:100FB000981761F0A28DAE0FBF2FB11D5D968C9179
:100FC000928D9F5F9F73928F90E008958FEF9FEFB8
:100FD0000895FC01918D828D981731F0828DE80F74
:100FE000F11D858D90E008958FEF9FEF0895FC012E
:100FF000918D228D892F90E0805C9F4F821B9109FB
:101000008F739927089587E59DE0F1DF21E0892B13
:1010100009F420E0822F0895FC01A48DA80FB92FB8
:10102000B11DA35ABF4F2C91848D90E001968F7310
:101030009927848FA689B7892C93A089B1898C912F
:10104000837080648C93938D848D981306C002887E
:10105000F389E02D80818F7D80830895EF92FF9248
:101060000F931F93CF93DF93EC0181E0888F9B8DCB
:101070008C8D98131AC0E889F989808185FF15C085
:101080009FB7F894EE89FF896083E889F9898081A8
:101090008370806480839FBF81E090E0DF91CF9177
:1010A0001F910F91FF90EF900895F62E0B8D10E099
:1010B0000F5F1F4F0F731127E02E8C8D8E110BC009
:1010C0000FB607FCFACFE889F989808185FFF5CF53
:1010D000CE01A2DFF2CFEB8DEC0FFD2FF11DE35A15
:1010E000FF4FF0829FB7F8940B8FEA89FB898081CC
:1010F0008062D0CF682F87E59DE0B0CFCF93DF939C
:10110000EC01888D8823B1F0AA89BB89E889F98927
:101110008C9185FD03C0808186FD0CC00FB607FC55
:10112000F7CF8C9185FFF2CF808185FFEDCFCE0187
:1011300073DFEACFDF91CF91089580E090E0892BB3
:1011400021F061DF81110E94000080E090E0892B96
:1011500049F080E090E0892B29F00E940000811185
:101160000E94000080E090E0892B49F080E090E050
:10117000892B29F00E94000081110E94000080E06C
:1011800090E0892B49F080E090E0892B29F00E94C3
:10119000000081110C94000008958150823108F004
:1011A0005AC0E82FF0E08827E752F74F8F4F0C9492
:1011B000E061F908FD08EB08F108F5082B090009C2
:1011C00006090A091009140918091E0922092B0920
:1011D00026092C093009809180008F778093800048
:1011E0000895809180008F7DF9CF80918000877F66
:1011F000F5CF84B58F7784BD089584B58F7DFBCFFF
:101200008091B0008F778093B00008958091B000F6
:101210008F7DF9CF809190008F7780939000089513
:10122000809190008F7DF9CF80919000877FF5CFDE
:101230008091A0008F778093A00008958091A000F6
:101240008F7DF9CF8091A000877FF5CF809120011D
:101250008F77809320010895809120018F7DF9CFB1
:1012600080912001877FF5CFCF93DF93282F30E047
:10127000F901E35BFD4F8491F901E355FD4FD491F2
:10128000F901ED50FD4FC491CC2399F0811185DF18
:10129000EC2FF0E0EE0FFF1FED5CFD4FA591B49138
:1012A000EC91ED2381E090E009F480E0DF91CF91B3
:1012B000089580E090E0FACF1F93CF93DF93282F1B
:1012C00030E0F901E35BFD4F8491F901E355FD4FF7
:1012D000D491F901ED50FD4FC491CC23A1F0162F0C
:1012E00081115BDFEC2FF0E0EE0FFF1FE75EFD4F9B
:1012F000A591B4918FB7F894EC91111108C0D095D5
:10130000DE23DC938FBFDF91CF911F910895DE2BF9
:10131000F8CFCF93DF9390E0FC01E355FD4F24918C
:101320008D509D4FFC0184918823C9F090E0880F77
:10133000991FFC01ED56FD4FA591B491FC01E75EAC
:10134000FD4FC591D49161110DC09FB7F8948C9158
:10135000209582238C938881282328839FBFDF9147
:10136000CF910895623051F49FB7F8943C91822F49
:10137000809583238C93E8812E2BEFCF8FB7F89441
:10138000EC912E2B2C938FBFEACFCF938CB58C6032
:101390008CBD8CB58F7D8CBD8CB58C7F8CBD8DB597
:1013A0008E7F8DBDCFB7F8948091560D811123C0EB
:1013B000E8E2F3E08491E2EEF2E09491E82FF0E0CD
:1013C000EE0FFF1FED56FD4FA591B491EC91E9236F
:1013D00019F461E085E370DF61E085E39ADF8CB5A5
:1013E00080618CBD8CB580648CBD61E084E391DF4D
:1013F00061E083E38EDF8091560D8F5F8093560D01
:10140000CFBFCF9108953FB7F8948091C4089091D1
:10141000C508A091C608B091C70826B5A89B05C00D
:101420002F3F19F00196A11DB11D3FBFBA2FA92F63
:10143000982F8827BC01CD01620F711D811D911D60
:1014400042E0660F771F881F991F4A95D1F70895CC
:101450008F929F92AF92BF92CF92DF92EF92FF92C4
:101460006B017C01D0DF4B015C01C114D104E104AC
:10147000F104B1F0C8DF681979098A099B09683E4F
:1014800073408105910588F321E0C21AD108E10873
:10149000F10888EE880E83E0981EA11CB11CE5CFF0
:1014A000FF90EF90DF90CF90BF90AF909F908F9084
:1014B00008952FB7F8946091C0087091C108809189
:1014C000C2089091C3082FBF0895CF92DF92EF9288
:1014D000FF92CF93DF93EC01603282E07807CCF586
:1014E000653B710514F064EB70E0898128E830E019
:1014F000281B310987FD3395220F331F220F331F1D
:101500006901330FEE08FF088A8128E532E0281BC5
:10151000310987FD3395220F331F220F331F032E0E
:10152000000C440B550B2C193D094E095F09DB01DA
:1015300077FF02C0B0E0A0E00E94756024EB30E0CD
:1015400040E050E00E944F60C20ED31EE41EF51E24
:10155000B601E881E03370F5298188E890E0821BCC
:10156000910927FD9395880F991F880F991F681778
:1015700079077CF02A8188E592E0821B910927FD9A
:101580009395880F991F880F991F681779070CF496
:10159000CB010297880F991F4FB7F8942E2F30E098
:1015A000F901EE0FFF1FE20FF31FEC50F24F928391
:1015B00081834FBFDF91CF91FF90EF90DF90CF906D
:1015C00008951F93CF93DF93EC01162F888180330A
:1015D00008F04DC061E0812F9CDE8881282F30E02B
:1015E000F901EE0FFF1FE20FF31FEC50F24F1F73D4
:1015F0006081607C612B608319821A822CE0622FEB
:101600000E94C161829FB001112430E020E0AB0153
:10161000420F531FFA01EE0FFF1FE40FF51FEC50AE
:10162000F24F908196FD16C02F5F3F4F2C30310551
:1016300071F7813009F51092800082E0809381007B
:101640001092850010928400B19A80916F008260A0
:1016500080936F00E8818E2F90E0FC01EE0FFF1F5A
:10166000E80FF91FEC50F24F8081806480838881FD
:10167000DF91CF911F910895823061F41092900014
:1016800080939100109295001092940088BB8093F3
:101690007100E0CF833069F41092A00082E0809363
:1016A000A1001092A5001092A40089BB8093720043
:1016B000D1CF8111CFCF1092200182E08093210100
:1016C00010922501109224018ABB80937300C2CF2F
:1016D000AF92BF92CF92DF92EF92FF920F931F9340
:1016E000CF93DF936B017A01EC01C554D74F28816A
:1016F0003CE0389F8001399F100D1124A090840E8A
:10170000B12C27FF1FC0FB011182108288818F5FDF
:10171000888388819801280F311D87FD3A95F6014D
:101720002A153B051CF488818C30BCF180819181A5
:10173000049680349C4908F471C0F601808191813F
:1017400004966EC088819801280F311D87FD3A9557
:101750002A153B05DCF68881A801480F511D87FD3D
:101760005A95FA01EE0FFF1FE40FF51FEC50F24FF0
:10177000808186FFCBCF8881F801E80FF11D87FDBE
:10178000FA95CF01EE0FFF1FE80FF91FEC50F24F53
:10179000808160E08F7390DDB9CF80819181288155
:1017A000A801420F511D27FD5A959A01FA01EE0F2B
:1017B000FF1FE20FF31FEC50F24F21813281820FA5
:1017C000931FF7019183808388819801280F311D31
:1017D00087FD3A95F901EE0FFF1FE20FF31FEC5062
:1017E000F24F808186FF21C08881080F111D87FD7F
:1017F0001A95F801EE0FFF1FE00FF11FEC50F24FAA
:10180000808161E08F73DF91CF911F910F91FF90E5
:10181000EF90DF90CF90BF90AF904ECD80E49CE9E9
:10182000F701918380838FEF8883DF91CF911F91A0
:101830000F91FF90EF90DF90CF90BF90AF90089501
:101840008EBD00000DB407FEFDCF8EB50895DF926A
:10185000EF92FF920F931F93CF93DF93EC01D62E5D
:10186000122F032FF42EE52E60E0888525DD8D2DC7
:101870008068E6DF89878E2DE3DF8F2DE1DF802F03
:10188000DFDF812FDDDF61E0888516DD8985DF916F
:10189000CF911F910F91FF90EF90DF900895FF92ED
:1018A0000F931F93CF93DF93EC01F62E8A016DDD2A
:1018B00060E0888501DD8F2DC3DF898780E0C0DF90
:1018C00080E0BEDF80E0BCDF80E0BADF61E08885D9
:1018D000F3DC60E08885F0DC8F2DB2DF898780E063
:1018E000AFDF90E0B0E0A0E0BA2FA92F982F8827B3
:1018F000F80180839183A283B38380E0A1DFF801A4
:101900004081518162817381482B762F652F542F3E
:101910004427408351836283738380E091DFF80121
:101920004081518162817381482B762F652F542F1E
:101930004427408351836283738380E081DFF80111
:101940004081518162817381482B4083518362833E
:10195000738361E08885B0DC8985DF91CF911F9129
:101960000F91FF9008952F923F924F925F927F9236
:101970008F929F92AF92BF92CF92DF92EF92FF929F
:101980000F931F93CF93DF9300D01F92CDB7DEB795
:101990006C01762E49015A0117012801AE014F5FF3
:1019A0005F4F7DDF89819A81AB81BC818826992632
:1019B000AA26BB26A50194012E21332140235521BF
:1019C000282739274A275B27672DC60140DFF60104
:1019D00081850F900F900F900F90DF91CF911F9105
:1019E0000F91FF90EF90DF90CF90BF90AF909F90BE
:1019F0008F907F905F904F903F902F900895CF935E
:101A0000DF93EC0161E0888584DC61E0888554DC4B
:101A1000BCDC60E0888550DC80E012DF898780E0F4
:101A20000FDF80E00DDF80E00BDF80E009DF61E0A9
:101A30008885DF91CF9140CC8F929F92AF92BF92D9
:101A4000CF92DF92EF92FF920F931F93CF93DF938A
:101A5000EC018B015A016901D2DF85E090E0A0E042
:101A6000B0E008301105C1F1B4F487E090E0A0E0E7
:101A7000B0E00230110581F186E090E0A0E0B0E036
:101A80000430110549F101301105A1F488E090E01E
:101A9000A0E0B0E021C083E090E0A0E0B0E0003240
:101AA0001105D1F05CF484E090E0A0E0B0E00031FA
:101AB000110591F080E090E0DC010EC082E090E042
:101AC000A0E0B0E00034110539F081E090E0A0E042
:101AD000B0E00038110571F7582F4427332722272B
:101AE000E12CF12C00E01FE06CE6CE013CDFB501FB
:101AF00090E080E00E94215F25ED34E045E352E470
:101B00000E94825F20E030E04AE754E40E941161C5
:101B100028EB3EE145E05EE30E94825F4B015C0101
:101B200026E636E646EA5EE30E94116120E030E0F8
:101B300040E85FE30E94AC600E947E61603180F407
:101B40002CEE31E548E35EE3C501B4010E9411616A
:101B500020E030E040E85FE30E94AC600E947E61DC
:101B6000862F8F71262F30E050E040E0542F432F16
:101B7000322F222722273F7144275527282B60E147
:101B8000CE0165DE0D2C000CEE08FF08A601332700
:101B90002227E12CF12C01E010E06CE6CE01E3DE1F
:101BA000E12CF12C8701E39421E030E040E050E0AB
:101BB00060E0CE01D8DE1FE0E12EF12C00E010E065
:101BC00023E030E040E050E06CE6CE01CCDEE12CDA
:101BD00010E8F12E01E010E020E030E840E050E0B5
:101BE0006CE6CE01C0DEE12CF12C8701F39420E0FD
:101BF00031E040E050E060E0CE01B5DEE12C14E0E1
:101C0000F12E00E010E020E034E040E050E060E041
:101C1000CE01A9DE2FEF3FEF4FE050E064E1CE01AF
:101C200016DE2FEF3FEF4FE050E065E1CE010FDE13
:101C30001FE0E12EF12C00E010E025E030E040E074
:101C400050E06CE6CE018FDEE12CF12C8701F3949D
:101C500020E03FE040E050E06CE6CE0184DE64E648
:101C600070E080E090E0DF91CF911F910F91FF90A5
:101C7000EF90DF90CF90BF90AF909F908F90E8CB88
:101C80000F931F93CF93DF938B01EA01AB01415078
:101C900051094433510508F0E9C02230310508F0FC
:101CA000E5C048E3429FF001439FF00D1124E80F87
:101CB000F91FE60FF71F81E080836C2F232B09F4B7
:101CC000D2C061E0802F25DB209749F460E0802FAF
:101CD000F3DACE01DF91CF911F910F910895CF3F9D
:101CE000D10511F461E0BFC0F801E35BFD4FE49161
:101CF000E150E23108F0B2C0F0E08827ED57F14F33
:101D00008F4F0C94E061950E9C0EA10EAB0EB50E9C
:101D10002E0FBF0EC70ECF0ED90EE30EED0EFC0E2A
:101D2000060F2E0F100F1A0F240F84B5806884BD84
:101D3000C7BDD0E0C0E0CDCF84B5806284BDC8BD52
:101D4000F8CF80918000806880938000D0938900D4
:101D5000C0938800EECF80918000806280938000E5
:101D6000D0938B00C0938A00E4CF8091800088607C
:101D700080938000D0938D00C0938C00DACF809147
:101D8000B00080688093B000C093B300D2CF809140
:101D9000B00080628093B000C093B400CACF80913D
:101DA0009000806880939000D0939900C093980031
:101DB000C0CF80919000806280939000D0939B0070
:101DC000C0939A00B6CF8091900088608093900075
:101DD000D0939D00C0939C00ACCF8091A000806800
:101DE0008093A0008091A0008F7B8093A000D0936F
:101DF000A900C093A8009DCF8091A000806280932D
:101E0000A000D093AB00C093AA0093CF8091A00014
:101E100088608093A000D093AD00C093AC0089CFC0
:101E200080912001806880932001D0932901C09384
:101E300028017FCF80912001806280932001D09380
:101E40002B01C0932A0175CF809120018860809377
:101E50002001D0932D01C0932C016BCF60E0C038DE
:101E6000D1050CF03FCF802F27DA63CFC1E0D0E05F
:101E700030CFCF93DF93D0E0C0E0CE010E940307C4
:101E8000882319F0CE010E94D1012196C13ED105CF
:101E9000A1F7DF91CF9108954F925F926F927F9259
:101EA0008F929F92AF92BF92CF92DF92EF92FF926A
:101EB000CF93DF93EC016C897D898E899F89888817
:101EC0009988AA88BB88CE8CDF8C0D2C000CEE087C
:101ED000FF08603127E272078105910529F0161687
:101EE000170618061906ACF0A7019601C501B40142
:101EF0000E94B261DF91CF91FF90EF90DF90CF9081
:101F0000BF90AF909F908F907F906F905F904F9019
:101F100008950E94235F20E030E44CE156E40E94E3
:101F200011612B013C01488E598E6A8E7B8EC50152
:101F3000B4010E94235FA30192010E94825F4B01C2
:101F40005C01C701B6010E94235F9B01AC01C50182
:101F5000B4010E94825F0E947961CCCFFC011182A2
:101F600010821382128215821482178216821086C2
:101F70001186128613861486158616861786108A91
:101F8000118A128A138A108E118E128E138E158E5C
:101F9000148E178E168E10A211A212A213A214A2D2
:101FA00015A216A217A210A611A612A613A614A671
:101FB00015A681E090E097A786A780E197E2A0E0D0
:101FC000B0E0848B958BA68BB78B08952F923F92B0
:101FD0004F925F926F927F928F929F92AF92BF9239
:101FE000CF92DF92EF92FF920F931F93CF93DF93E5
:101FF00000D000D0CDB7DEB79E838D831B015A0180
:102000004901DC015596CD90DD90ED90FC905897FC
:10201000D701C60188279927AA27B17089839A8397
:10202000AB83BC83ED81FE81E958FF4F4080518036
:1020300062807380C301B20124E630E040E050E0EA
:102040000E947B60672B682B692BA1F5AD81BE8157
:102050001C968D919C911D971F969C938E931E9715
:102060001A968D919C911B971D969C938E931C970D
:1020700018968D919C9119971B969C938E931A9705
:1020800016968D919C91179719969C938E931897FD
:10209000F50160817181828193810E947961AD81B6
:1020A000BE8117967C936E931697F501108211826C
:1020B0001282138289819A81AB81BC81892B8A2B00
:1020C0008B2B59F4F7FC09C0CC24DD24EE249EE7C9
:1020D000F922CD28CE28CF28F1F0C301B2010E9409
:1020E000215FD8012D913D914D915C910E94AA6193
:1020F00087FD11C020E030E040E85FE3F50160813A
:102100007181828193810E94AD60D5016D937D9331
:102110008D939C931397ED81FE81EE5AFF4FFA83C6
:10212000E98380819181A281B381F40180839183CD
:10213000A283B383E981FA8180819181A281B381F5
:10214000F101808B918BA28BB38B26960FB6F894FE
:10215000DEBF0FBECDBFDF91CF911F910F91FF90DA
:10216000EF90DF90CF90BF90AF909F908F907F9037
:102170006F905F904F903F902F900895889A0895A8
:10218000889808958E9A08958E980895EBE0F1E06E
:102190008081886080830895EBE0F1E08081877F13
:1021A00080830895149A08951498089560E0FC01BE
:1021B000878D82C860E0FC01818D7EC861E0FC01F2
:1021C000878D7AC861E0FC01818D76C8CF93DF935B
:1021D000EC01FC01EB57FF4F1082379781E08083C1
:1021E00060E0898D69D88BA19CA1892B29F060E0E2
:1021F0008F8DDF91CF9160C8DF91CF910895CF93FC
:10220000DF93EC018FA130D82AA52817190621F4F5
:102210008BA5DF91CF91089580E0FBCFCF93DF9323
:10222000EC018DA121D82AA52817190621F48BA528
:10223000DF91CF91089580E0FBCFCF93DF93EC0146
:102240008B8DFE01EF5BFF4F908161E0911101C02A
:1022500060E032D889A1FE01EE5BFF4F90819923A7
:1022600031F0CD5BDF4F988161E0911101C060E0FA
:10227000DF91CF9121C8CF93DF93EC018B8DFE01CD
:10228000EF5BFF4F908160E0911101C061E014D8D5
:1022900089A1FE01EE5BFF4F9081992331F0CD5B68
:1022A000DF4F988160E0911101C061E0DF91CF9133
:1022B00003C8CF93DF93EC0161E08D8D0E945C0930
:1022C000FE01EE5BFF4F8081882321F061E08BA14E
:1022D0000E945C09CD57DF4F1882DF91CF9108959E
:1022E000CF93DF93EC01FC01E45AFC4F1082EE58CF
:1022F000F1098081811103C0CE014096DADFFE0131
:10230000E153FD4F8081811104C0CE018A559F4F5A
:10231000D0DFFE01E053FD4F8081811104C0CE016A
:10232000845C9E4FC6DF64E670E080E090E0DF9161
:10233000CF918EC8CF93DF93EC0160E08D8D0E942A
:102340005C09FE01EE5BFF4F8081882321F060E095
:102350008BA10E945C09CD57DF4F81E08883DF911C
:10236000CF9108958F929F92AF92BF92CF92DF92BA
:10237000EF92FF920F931F93CF93FC01E25BFF4F0D
:102380004083518362837383349640835183628395
:10239000738334960083118322833383DC01A65A2E
:1023A000BF4FEC925297CC91CC2351F018974C919F
:1023B000411152C037FF56C010821182128213821F
:1023C000DC01A75BBF4F4D915D916D917C9113979F
:1023D000141615061606170634F514963C91332389
:1023E00011F1C080D180E280F38046015701F7FEF1
:1023F00007C08824992454018C189D08AE08BF0892
:10240000481559056A057B0574F4F7FE07C07095F9
:102410006095509541955F4F6F4F7F4F408351833B
:1024200062837383C32FFC01E959FF4F108211822D
:102430001282138285589F4F31E0FC0130838C2F2C
:10244000CF911F910F91FF90EF90DF90CF90BF90B1
:10245000AF909F908F9008951016110612061306E4
:102460000CF4AACFC0E0ACCF0F931F93CF93DF93B0
:10247000EC01062F89A581110DC0CE01CFDE182FEA
:10248000CE01BDDE0111182F812FDF91CF911F9159
:102490000F910895CE01B3DE182FCE01BFDEF2CF2B
:1024A000CF93DF93EC01FC01E958FF4F80819181CC
:1024B000A281B3810196A11DB11D80839183A28366
:1024C000B3833E9681E08083AE014E5A5F4FFA019E
:1024D00080819181A281B3819E0124583F4FF901EF
:1024E0002081222309F440C00196A11DB11DFA01EB
:1024F00080839183A283B383FE01E857FF4F20813D
:102500003181C901959587958C0F9D1F3297019058
:10251000F081E02D20FF08C0DC012D913C91E20FFD
:10252000F31F0190F081E02D19958BA19CA1892BBF
:10253000F9F0FE01E457FF4F20813181C9019595E3
:1025400087958C0F9D1FC657DF4FE881F98120FFCB
:1025500008C0DC012D913C91E20FF31F0190F08146
:10256000E02DDF91CF9119940197A109B109BFCF57
:10257000DF91CF9108958F929F92AF92BF92CF92A9
:10258000DF92EF92FF920F931F93CF93DF93EC01B3
:10259000FC01E959FF4F60817181828193810E9422
:1025A000215F6B017C01FE01EC5BFF4F608171815B
:1025B000828193810E94235F9B01AC0160E074E201
:1025C00084E799E40E9411614B015C01FE01ED5822
:1025D000FF4F60817181828193810E94215F9B0105
:1025E000AC01C501B4010E9411614B015C018E0177
:1025F00005591F4F20E030E040E05FE30E94825F1A
:10260000A70196010E94AD600E947E61F80160837F
:10261000718382839383C159DF4FA5019401C70160
:10262000B6010E94AD600E947E61688379838A83CF
:102630009B83DF91CF911F910F91FF90EF90DF90DF
:10264000CF90BF90AF909F908F9008950F931F935E
:10265000CF93DF93FC01EB57FF4F20812223B9F08A
:102660007E9700811181228133813896408151818A
:1026700062817381041715072607370710F1EC01F3
:10268000A5DDCE01DF91CF911F910F9174CFFC0199
:10269000E558FF4F20812223A1F07497008111811A
:1026A0002281338134964081518162817381041784
:1026B00015072607370728F0DF91CF911F910F915B
:1026C000EFCEDF91CF911F910F910895FC01E55856
:1026D000FF4F2081222361F0749780819181A28134
:1026E000B3810196A11DB11D80839183A283B38321
:1026F00008950F931F93FC01E65AFF4F208121118B
:1027000012C0389700811181228133813496408133
:1027100051816281738104171507260737074CF42E
:102720001F910F91A8CDFC01E05CFF4F208121118A
:10273000F7CF1F910F9181CDCF92DF92EF92FF9251
:102740000F931F93CF93DF93EC017B016A01890103
:102750009A01AB01B801888199816ED98C81883545
:1027600071F49601A701B8018A819B81DF91CF9115
:102770001F910F91FF90EF90DF90CF905DC9DF9197
:10278000CF911F910F91FF90EF90DF90CF90089520
:10279000CF93DF93EC018C818835A9F583E593E134
:1027A0009983888383E893E19B838A8382EE90E117
:1027B000FE01EA57FF4F9183808332961182108287
:1027C0008EED90E132969183808332961182108251
:1027D0008AED90E132969183808332961182108245
:1027E00086ED90E132969183808332961182108239
:1027F0008881998104D98C81883589F48A819B816B
:10280000DF91CF91FCC8893529F483E693E1998360
:102810008883CCCF8A3551F683E793E1F8CFDF91F7
:10282000CF910895CF93DF93FC01DC0116968AE0E7
:10283000ED0119928A95E9F781E0808B818B138AEB
:10284000128A148A158A168A178A108E8CE291E0F1
:10285000A0E0B0E084A795A7A6A7B7A742E350E001
:1028600060E070E040AB51AB62AB73AB44AB55ABD7
:1028700066AB77AB80AF91AFA2AFB3AF88E790E024
:10288000A0E0B0E084AF95AFA6AFB7AFDF01A05C2A
:10289000BF4F1C9211961C9211961C9211961C927D
:1028A000119644E650E060E070E04D935D936D93C7
:1028B0007C93139714961C9211961D921D921D9253
:1028C0001C92139714961C9211961D921D921D92A4
:1028D0001C92139714961D921D921D921C92139791
:1028E00014961D921D921D921C92139714961C9281
:1028F00011961D921D921D921C92139714961D9273
:102900001D921D921C92139714961D921D921D925A
:102910001C92139714961D921D921D921C92139750
:1029200014961D921D921D921C92139714961D923F
:102930001D921D921C92139714961D921D921D922A
:102940001C92139714961D921D921D921C92139720
:1029500014961C9211961C9211961C9211961C9220
:1029600011961C9211961C9211961C9211961C9213
:1029700011961C9211961C9211961C92128E118E19
:10298000148E138E168E158E10A2178E12A211A2FF
:1029900014A213A216A215A210A617A2119682EED7
:1029A00090E111969C938E93129611961C921E9212
:1029B00012968EED90E111969C938E93129611963D
:1029C0001C921E9212968AED90E111969C938E9322
:1029D000129611961C921E92129686ED90E18D939E
:1029E0009C93EC56FF4F11821082DF91CF91089596
:1029F00008958FEF9FEF089508950895089508951D
:102A000008950895089508950895089508950895DE
:102A100008950895089508950895089508950895CE
:102A200008958091B9089091BA08892B41F481E00A
:102A300090E00E94A4599093BA088093B9088091BD
:102A4000B9089091BA0808950F931F93CF93DF931D
:102A50008B01E7DFF801C2A1D3A1868D978D853068
:102A6000910529F14CF40497B1F090E080E0DF91FA
:102A7000CF911F910F9108958630910511F10B9719
:102A8000A1F76BE070E08EE89EE00E94E10ABE01D3
:102A90008EE89EE009C064E070E085E89EE00E9458
:102AA000E10ABE0185E89EE00E94650ADECF65E08E
:102AB00070E088E89EE00E94E10ABE0188E89EE09E
:102AC000F3CF66E070E08BE89EE00E94E10ABE0171
:102AD0008BE89EE0E9CF8091B5089091B608892BEC
:102AE00091F480E790E00E94A459FC0131969C018A
:102AF0002B5C3F4F119217AAE217F307D9F7909377
:102B0000B6088093B5088091B5089091B6080895ED
:102B10004F925F926F927F92AF92BF92CF92DF926D
:102B2000EF92FF920F931F93CF93DF93EB01D3DFCD
:102B30008C01CAA8DBA84EA45FA468A879A8AEA09F
:102B4000BFA0EE8CFF8C4AA15BA19601B70198D87B
:102B5000C301B2010E94280A9601A501B701C8016C
:102B60008FD890E080E0DF91CF911F910F91FF907F
:102B7000EF90DF90CF90BF90AF907F906F905F907D
:102B80004F900895CF93DF93EB01A5DF6AA98E8D57
:102B90000E94890990E080E0DF91CF910895CF9362
:102BA000DF93EB0198DF2AA93BA94AA15BA16E8DB7
:102BB0007F8D66D890E080E0DF91CF91089580917D
:102BC000AE089091AF08892BE1F585E390E00E9473
:102BD000A459FC0181E090E0A0E0B0E08083918303
:102BE000A283B38384839583A683B78380879187E9
:102BF000A287B3871586148616861786108A118ACF
:102C0000128A138A148A158A168A178A108E118ED0
:102C1000138E128E12A213A214A215A217A216A22C
:102C200010A611A612A613A614A615A616A617A6D8
:102C300010AA11AA12AA13AA14AAF093AF08E0933B
:102C4000AE088091AE089091AF080895CF93DF93BE
:102C5000B6DFEC0185E40E94340921E0892B09F4F8
:102C600020E02C8FACDFEC0184E40E94340921E0E9
:102C7000892B09F420E02D8FA2DFEC0183E40E9470
:102C8000340921E0892B09F420E02E8F98DFEC0134
:102C900082E40E94340921E0892B09F420E02F8F7F
:102CA0008EDFEC0181E40E94340921E0892B09F4D4
:102CB00020E028A384DFEC0180E40E94340921E0B5
:102CC000892B09F420E029A3DF91CF91089577DFC4
:102CD000BDCF75DFFC0114AA90E080E00895FC01EF
:102CE00001900020E9F73197AF01481B590BBC0157
:102CF00087E59DE00C9499078F929F92AF92BF92C7
:102D00000F931F93CF93DF93CDB7DEB7A1970FB685
:102D1000F894DEBF0FBECDBF19A2423008F44AE0DE
:102D20008E010F5D1F4F842E912CB12CA12CA5017B
:102D300094010E947B60E62FB901CA01EA30ECF4ED
:102D4000E05DD801EE938D01232B242B252B79F701
:102D500090E080E0109711F0CD01C1DFA1960FB691
:102D6000F894DEBF0FBECDBFDF91CF911F910F91C1
:102D7000BF90AF909F908F900895E95CE2CFCF9283
:102D8000DF92EF92FF92CF93DF9397FF18C06B0112
:102D90007C018DE20E947A08EC0166277727CB013F
:102DA0006C197D098E099F094AE0A6DF8C0F9D1FD3
:102DB000DF91CF91FF90EF90DF90CF9008954AE0A0
:102DC000DF91CF91FF90EF90DF90CF9095CFBC0136
:102DD000990F880B990BD3CF82CF882319F08AE003
:102DE00098E0FACF83E098E0FCCF2F923F924F9289
:102DF0005F926F927F928F929F92AF92BF92CF928B
:102E0000DF92EF92FF920F931F93CF93DF93CDB793
:102E1000DEB762970FB6F894DEBF0FBECDBF1C01C0
:102E20008C010E5A1F4F1E870D87D8014D915D9161
:102E30006D917C917C01B6E5EB0EF11CF701808170
:102E40009181A281B3816101FAE5CF0ED11CF60117
:102E50002081065D1F4F5801B3964F012223B9F11F
:102E60009101205C3F4FF9012081F801208321E08E
:102E7000F4012083411551056105710559F4F101F3
:102E800000A911A922A933A9ED58FF4F008311838E
:102E9000228333838101025B1F4FF8014080518000
:102EA00062807380910125583F4F59014816590699
:102EB0006A067B06B4F5481759076A077B07DCF1F9
:102EC000D6018C91811137C0D5011C923AC121E005
:102ED000481759076A077B070CF020E0F5012083AB
:102EE0002A013B0177FF07C0442455243201441ACC
:102EF000550A660A770A8C019D01B7FF07C00027B3
:102F000011279801081B190B2A0B3B0BBB24B39408
:102F100040165106620673060CF4B12CF401B0821F
:102F2000A9CF84159505A605B70554F6841795070E
:102F3000A607B7072CF6F5018081882329F2D60170
:102F40008C9181110DC0F60180818111BDCFD4011A
:102F50006C9181E06827C10187DA8111B5CF05C086
:102F600060E0C10181DA8111EECFD101D8962D91B7
:102F70003D914D915C91DB9729833A834B835C8330
:102F80009C962D913D914D915C919F972D833E8311
:102F90004F835887D0962D913D914D915C91D39759
:102FA00029873A874B875C87F70180819181A281CD
:102FB000B381ED85FE85C080D180E280F380F80189
:102FC0004081518162817381F101E158FF4F10828C
:102FD000319610823101F1E86F0E711CF3011082FD
:102FE00091012E573F4FF9011082329610824C0109
:102FF0005D01841A950AA60AB70AB7FE08C0B09404
:10300000A09490948094811C911CA11CB11C481721
:1030100059076A077B072CF0C81AD90AEA0AFB0A83
:1030200004C0C41AD50AE60AF70AD501C401B59549
:10303000A795979587958D879E87AF87B88B8101D8
:103040000C571F4F8C149D04AE04BF0408F09EC0A3
:10305000D101D4960D90BC91A02DBA8BA98B81E0A3
:10306000F9018083D8018C93F1018489882309F4C4
:103070005CC00E94590AD10152960D911C91012EFB
:10308000000C220B330B601B710B820B930B693E00
:1030900073408105910508F448C00E94590AF10166
:1030A000738B628B86E993E097DE8AE993E094DE86
:1030B00060E070E0CB0163DE80EA93E08DDEC70163
:1030C000B6015DDE86EA93E087DEC501B40157DE16
:1030D0008CEA93E081DE4AE06D857E858F85988954
:1030E0000BDE83EB93E078DE69817A818B819C81B2
:1030F00046DE89EB93E070DE69857A858B859C8559
:103100003EDE8FEB93E068DE6D817E818F81988556
:1031100036DE85EC93E060DE82EA96E05DDE89894A
:103120009A8955DE8EE798E057DEF101ED58FF4FA2
:1031300009891A89C801B0E0A0E080839183A28345
:10314000B38360E0C10190D9882339F0F101EE5AD0
:10315000FF4F108211821282138262960FB6F8948A
:10316000DEBF0FBECDBFDF91CF911F910F91FF90BA
:10317000EF90DF90CF90BF90AF909F908F907F9017
:103180006F905F904F903F902F9008952D853E85D2
:103190004F8558892C153D054E055F0508F450C034
:1031A00089819A81AB81BC818C159D05AE05BF05D7
:1031B00044F4AD81BE811196BA8BA98B81E0F301F5
:1031C00050CFC701B6010E94235F2B013C016981EA
:1031D0007A818B819C810E94235F9B01AC01C3019A
:1031E000B2010E9411612B013C016D817E818F81B2
:1031F000988529853A854B855C85621B730B840B0A
:10320000950B0E94235F9B01AC01C301B2010E9498
:10321000825F2B013C0169857A858B859C850E94A4
:10322000235F9B01AC01C301B2010E94AD600E940B
:1032300079617A8B698B81E0F101E158FF4F11CF01
:10324000D501C40129813A814B815C81821B930B9A
:10325000A40BB50BC816D906EA06FB065CF44D8133
:103260005E814E5F5F4F5A8B498B81E0F101EF57D2
:10327000FF4FF7CEC501B4016C197D098E099F0976
:103280000E94235F2B013C0169817A818B819C81A3
:103290000E94235F9B01AC01C301B2010E94116136
:1032A0002B013C016D817E818F81988529853A852E
:1032B0004B855C85621B730B840B950B0E94235F0F
:1032C0009B01AC01C301B2010E94825F2B013C0152
:1032D00069857A858B859C850E94235F9B01AC0163
:1032E000C301B2010E94AD600E9479617A8B698B43
:1032F00081E0F101E058FF4FB4CECF93DF93EC01B2
:103300008BEC93E069DD6AA17BA18CA19DA137DDE7
:103310008EE798E0DF91CF915FCD0F931F93CF930E
:10332000DF938C01EB0188E793E056DD82EA96E0BB
:1033300053DDF80184810E947A08CE0148DD3FDC2C
:10334000DF91CF911F910F91D8CFEF92FF920F9302
:103350001F93CF93DF93182F092F7B016115710500
:1033600069F50E94340931E020E0019709F030E06E
:10337000C32FD22F82E0E816F10408F045C08EEC8E
:1033800093E02ADD82EA96E027DD82ED93E024DDFA
:10339000812F902F1CDD82EA96E01EDD8DE296E003
:1033A0001BDDCE0114DD0BDCA8DF90E080E0DF91B7
:1033B000CF911F910F91FF90EF900895D0E0C0E062
:1033C00061307105B9F6812F163310F08AEC810F48
:1033D00020917B00982F9870277F922B90937B00F1
:1033E0008770806480937C0080917A0080648093F1
:1033F0007A0080917A0086FDFCCF80917800C091A0
:103400007900DC2FC82FB6CF81E090E0D0CF0F93AA
:103410001F93CF93DF93FC0120813181211531056A
:10342000C1F1EC01822F0E94340921E0892B09F4BB
:1034300020E02B876A85261701F11E821F821886DD
:1034400019860E811F81288539858A819B81AC81EF
:10345000BD81081719072A073B07DCF081E06827C0
:1034600088810E945C0937DB70E060E08881998187
:10347000DF91CF911F910F9168CF8E819F81A88599
:10348000B9850196A11DB11D8E839F83A887B98739
:10349000D8CFDF91CF911F910F910895CF93DF93F4
:1034A000EB0119DB6AA97BA98E8D9F8D4EDF90E021
:1034B00080E0DF91CF910895CF92DF92EF92FF925B
:1034C000CF93DF93EB01CB010E940307882351F1D7
:1034D000FE01EE0FFF1FEE0FFF1FEE52F64FC080F2
:1034E000D180E280F38084ED93E076DC82EA96E09E
:1034F00073DC82ED93E070DCCE0169DC82EA96E059
:103500006BDC8DE296E068DCC701B60138DC57DB86
:10351000F4DE90E080E0DF91CF91FF90EF90DF90BC
:10352000CF90089588ED93E057DCF3CF0F931F936E
:10353000CF93DF938C01D0E0C0E0CE010E9403075F
:10354000882319F0BE01C801B7DF2196C13ED1051D
:10355000A1F7DF91CF911F910F9108958AEF93E02A
:103560003BDC88E292E038DC88E092E035DC8FEFEB
:1035700093E032DC24DBC1DE90E080E00895CF935D
:10358000DF93EC0189E094E027DC8DE094E024DC1B
:103590008C8D23DC81E194E01FDC8D8D1EDC85E1C8
:1035A00094E01ADC8E8D19DC89E194E015DC8F8DB6
:1035B00014DC8DE194E010DC88A10FDC81E294E062
:1035C0000BDC89A10ADCCE01DF91CF9196CEF7DA30
:1035D000D6CF85E294E000DCF2DA38DBF0DACFDF38
:1035E0007ADA70E060E088E090E0AFDE74DA70E0F4
:1035F00060E089E090E0A9DE6EDA70E060E08AE0E9
:1036000090E0A3DE68DA70E060E08DE090E09DDE9F
:1036100090E080E008954F925F926F927F928F9238
:103620009F92AF92BF92CF92DF92EF92FF920F9351
:103630001F93CF936B017C01742EAC019B010E9400
:10364000AE61882391F08CE294E0CF911F910F91AD
:10365000FF90EF90DF90CF90BF90AF909F908F90B2
:103660007F906F905F904F903ACB46015701E8945E
:10367000B7F82FEF3FEF4FE75FE7C501B4010E94B6
:10368000AE6181110DC02FEF3FEF4FE75FE7C5013E
:10369000B4010E941D5F18161CF480E394E0D5CF9E
:1036A0002FEF3FEF4FE75FE4C701B6010E94AA6129
:1036B00018161CF484E394E0C8CF2FEF3FEF4FE7D8
:1036C0005FECC701B6010E941D5F87FDF3CF20E0CC
:1036D00030E0A901C701B6010E941D5F10E000E0C3
:1036E00087FF08C08DE20E947A088C01F7FAF094F7
:1036F000F7F8F094C0E060E070E080E09FE37C16B3
:1037000041F020E030E040E251E40E941161CF5FDF
:10371000F6CFA70196010E94AD602B013C010E94EB
:103720007E614B015C014AE0E7DA7C01E00EF11EAC
:10373000CC23A9F1C501B4010E94215F9B01AC011A
:10374000C301B2010E94AC604B015C018EE20E9499
:103750007A08E80EF91EC15010F120E030E040E296
:1037600051E4C501B4010E94825F2B013C010E941B
:103770007E614B01B12CA12C4AE0C501B401BCDA39
:10378000E80EF91EC501B4010E94215F9B01AC0146
:10379000C301B2010E94AC604B015C01DCCFC701E8
:1037A000CF911F910F91FF90EF90DF90CF90BF903E
:1037B000AF909F908F907F906F905F904F90089503
:1037C0008F929F92AF92BF92CF92DF92EF92FF9231
:1037D0000F931F93CF93DF93EC0184E392E0FCDA25
:1037E0008DE494E0F9DA6E018EE2C81A8EEFD80A01
:1037F000C6010E944C0F0E94235F4B015C01FE0139
:10380000E151FD4F60817181828193810E94235F2C
:103810009B01AC01C501B4010E94116142E0FBDED5
:103820008DE594E0D9DA7E01E2E0EE0EFE1EC701DE
:103830000E944C0F0E94235F4B015C01FE01ED5082
:10384000FD4F60817181828193810E94235F9B0182
:10385000AC01C501B4010E94116142E0DCDE8DE6DD
:1038600094E0BADA8E010E5C1D4FC8010E944C0F25
:103870000E94235F4B015C01C950DD4F6881798153
:103880008A819B810E94235F9B01AC01C501B40129
:103890000E94116142E0BFDE92D92FDD80E392E009
:1038A0009BDA8DE494E098DAF601A68DB78D208935
:1038B0003189428953890E94756061DA8DE594E00F
:1038C0008BDAF701A68DB78D20893189428953891A
:1038D0000E94756054DA8DE694E07EDAF801A68DD8
:1038E000B78D20893189428953890E94756047DAF2
:1038F00066D9DF91CF911F910F91FF90EF90DF90EC
:10390000CF90BF90AF909F908F90F7CCCF92DF92E7
:10391000EF92FF92CF93DF93EC0188819981AA8186
:10392000BB81181619061A061B0644F081E090E0C8
:10393000A0E0B0E088839983AA83BB838C819D81BA
:10394000AE81BF81181619061A061B0644F081E0E5
:1039500090E0A0E0B0E08C839D83AE83BF83888538
:103960009985AA85BB85181619061A061B0644F008
:1039700081E090E0A0E0B0E088879987AA87BB87C4
:1039800088E394E029DA8DE494E026DA6E857F8579
:10399000888999890E94235F6B017C016881798104
:1039A0008A819B810E94235F9B01AC01C701B60104
:1039B0000E94116142E02FDE8DE594E00DDA6A8904
:1039C0007B898C899D890E94235F6B017C016C81BE
:1039D0007D818E819F810E94235F9B01AC01C70185
:1039E000B6010E94116142E016DE8DE694E0F4D942
:1039F0006E897F89888D998D0E94235F6B017C0180
:103A0000688579858A859B850E94235F9B01AC012F
:103A1000C701B6010E94116142E0FDDDCE01DF91D8
:103A2000CF91FF90EF90DF90CF9067CCC8D86EDF3A
:103A300090E080E00895FC0180819181009711F071
:103A40000C94405A08950C94405A0C94405A0C948B
:103A5000405A0C94405A0C94405A0C94405A0C947E
:103A6000405A0C94405A0C94405A0C94405A0C946E
:103A7000405A0C94405A0C94405A0C94405A0C945E
:103A8000405A0C94405A0C94405A0C94405A0C944E
:103A9000405A0C94405A0C94405A0C94405A0C943E
:103AA000405ACF92DF92EF92FF920F931F93CF93E2
:103AB000DF938C016A017B01EC01CC0FDD1F642FC9
:103AC000CE010E9441609927F7FC9A958F2D7E2D9B
:103AD0006D2DCE0101960E9441600D5811090330F1
:103AE000110588F4B701992777FD9095892FCE01AC
:103AF00044960E9441606F2D772788279927CE0131
:103B000045960E94416090E080E0DF91CF911F9147
:103B10000F91FF90EF90DF90CF9008954F925F92BA
:103B20006F927F928F929F92AF92BF92CF92DF92CD
:103B3000EF92FF920F931F93CF93DF938C01EC01D1
:103B4000CC0FDD1FCE010E943960882E912CB12C44
:103B5000A12CCE0101960E943960C82ED12CF12CE7
:103B6000E12C0D5811090330110508F05AC0CE019F
:103B700044960E943960482E512C712C612CCE0144
:103B800045960E943960082F10E030E020E08FEF6A
:103B9000481651046104710429F50F3F11052105F0
:103BA000310501F58FEF88169104A104B104C9F520
:103BB0008FEFC816D104E104F10499F56FEF7FEFA0
:103BC000CB01DF91CF911F910F91FF90EF90DF908C
:103BD000CF90BF90AF909F908F907F906F905F90AD
:103BE0004F90089500381105210531053CF7FE2C52
:103BF000ED2CDC2CCC24C701B601680D791D8A1D83
:103C00009B1D320155244424640D751D861D971D8E
:103C1000302F222711270027600F711F821F931F4B
:103C2000D0CF00E010E09801412C512C320180E807
:103C3000C816D104E104F104D4F2C0CFEF92FF9290
:103C40000F931F93CF93DF938091B3089091B408A3
:103C5000892B51F586E090E00E94A4597C0190E008
:103C600080E05CDF1616170654F1C7010E94390F79
:103C7000D0E0C0E0CE010E940307882369F0FE0176
:103C8000EE0FFF1FEE0FFF1FEE52F64F40815181E6
:103C900062817381CE0105DF2196C639D10551F7C6
:103CA000F092B408E092B3088091B3089091B40800
:103CB000DF91CF911F910F91FF90EF90089583E0D6
:103CC00090E02CDF613071058105910531F502ED41
:103CD00019E0D0E0C0E0CE010E9403078823B1F0D4
:103CE000CE011CDFF80160837183828393836F3F71
:103CF0007F4F8F4F9F4F51F4CE010E94D101F801A9
:103D00004081518162817381CE01CBDE21960C5FAF
:103D10001F4FC13ED105F9F6C3CFC7010E94390F2D
:103D2000BFCFCF92DF92EF92FF920F931F93CF936B
:103D3000DF937C016B018A01E90180DFF601EE0F60
:103D4000FF1FEE0FFF1FEE52F64F80819181F701AA
:103D50009183808373DF000F111F000F111FF80183
:103D6000EE52F64F81E04081518162817381413092
:103D700051056105710509F080E0F70182875EDF7A
:103D8000CC0FDD1FCC0FDD1FCE52D64F888199811D
:103D9000AA81BB81F70182839383A483B5831682B2
:103DA000178210861186DF91CF911F910F91FF909E
:103DB000EF90DF90CF900895CF93DF93EC012AEC42
:103DC00030E04BEC50E069EC70E0ABDF2EEC30E023
:103DD0004FEC50E06DEC70E0CE010C96A2DF24EDCC
:103DE00030E045ED50E063ED70E0CE01489699DF9C
:103DF00028ED30E049ED50E067ED70E0CE018496AB
:103E000090DF2EED30E04FED50E06DED70E0CE0133
:103E1000C096DF91CF9185CFCF93DF938091B70884
:103E20009091B808892BA1F48CE390E00E94A459EA
:103E3000EC01198218821D861C86198E188E1DA20F
:103E40001CA219AA18AAB8DFD093B808C093B70863
:103E50008091B7089091B808DF91CF9108950F93A2
:103E60001F93CF93DF93EC01E9DEFE01EB5DFC4F86
:103E700080918E0B90918F0B91838083DFDEFE010A
:103E8000E95DFC4F8091920B9091930B918380831D
:103E9000D5DEFE01E75DFC4F8091960B9091970B6C
:103EA00091838083CBDE8E01055D1C4F6091B60B44
:103EB0007091B70B8091B80B9091B90B0E94235F62
:103EC000F8016083718382839383B8DE0C5F1F4F98
:103ED0006091BA0B7091BB0B8091BC0B9091BD0BA4
:103EE0000E94235FF8016083718382839383A6DE3F
:103EF0000C5F1F4F6091BE0B7091BF0B8091C00B88
:103F00009091C10B0E94235FF801608371838283CB
:103F1000938394DEFE01E65CFC4F8091760B9091DA
:103F2000770B918380838ADEFE01E45CFC4F8091F5
:103F30007A0B90917B0B9183808380DEFE01E25CA3
:103F4000FC4F80917E0B90917F0B9183808376DE76
:103F5000FE01E05CFC4F80919E0B90919F0BA09125
:103F6000A00BB091A10B80839183A283B38366DE03
:103F7000FE01EC5BFC4F8091A20B9091A30BA091F2
:103F8000A40BB091A50B80839183A283B38356DEEB
:103F9000FE01E85BFC4F8091A60B9091A70BA091CE
:103FA000A80BB091A90B80839183A283B38346DED3
:103FB000FE01E45BFC4F8091C60B9091C70B91838F
:103FC00080833CDEFE01E25BFC4F8091CA0B909146
:103FD000CB0B9183808332DEFE01E05BFC4F80914E
:103FE000CE0B9091CF0B9183808328DEFE01EE5A99
:103FF000FC4F8091DE0B9091DF0B918380831EDE5E
:10400000FE01EC5AFC4F8091E20B9091E30B9183FF
:10401000808314DEFE01EA5AFC4F8091E60B9091FA
:10402000E70B918380830ADE8091660B9091670B8A
:10403000A091680BB091690BFE01E95CFC4F019700
:10404000A105B10551F581E08083F8DD80916A0B0F
:1040500090916B0BA0916C0BB0916D0BFE01E85C25
:10406000FC4F0197A105B105D1F481E08083E6DD25
:1040700080916E0B90916F0BA091700BB091710BB2
:10408000C75CDC4F0197A105B10559F481E0888335
:10409000DF91CF911F910F9108951082D6CF10829A
:1040A000E6CF1882F5CF2F923F924F925F926F9298
:1040B0007F928F929F92AF92BF92CF92DF92EF92B8
:1040C000FF920F931F93CF93DF93CDB7DEB7659722
:1040D0000FB6F894DEBF0FBECDBF998B888BAEDDD7
:1040E000E889F989E358FD4F81E040919E0A50919B
:1040F0009F0A6091A00A7091A10A452B462B472B7D
:1041000009F480E080839ADDE889F989E258FD4F5F
:1041100081E04091A20A5091A30A6091A40A709193
:10412000A50A452B462B472B09F480E0808386DDCA
:10413000E889F989E158FD4F81E04091A60A509144
:10414000A70A6091A80A7091A90A452B462B472B14
:1041500009F480E0808372DD8091EE0A9091EF0A8D
:10416000A091F00AB091F10AE889F989E058FD4F71
:1041700080839183A283B38361DD8091F20A909161
:10418000F30AA091F40AB091F50AE889F989EC578D
:10419000FD4F80839183A283B38350DD8091F60A23
:1041A0009091F70AA091F80AB091F90AE889F98983
:1041B000E857FD4F80839183A283B3833FDD8091D5
:1041C000C60A9091C70AA091C80AB091C90AE889A5
:1041D000F989E856FD4F80839183A283B3832EDD56
:1041E0008091CA0A9091CB0AA091CC0AB091CD0AD5
:1041F000E889F989E456FD4F80839183A283B383D4
:104200001DDD8091CE0A9091CF0AA091D00AB09185
:10421000D10AE889F989E056FD4F80839183A28312
:10422000B3830CDD8091D60A9091D70AA091D80A69
:10423000B091D90AE889F989EC55FD4F80839183C3
:10424000A283B383FBDC8091DA0A9091DB0AA09110
:10425000DC0AB091DD0AE889F989E855FD4F8083D1
:104260009183A283B383EADC8091DE0A9091DF0A16
:10427000A091E00AB091E10AE889F989E455FD4F7F
:1042800080839183A283B383D9DC8091760A909155
:10429000770AA091780AB091790AE889F989E055FE
:1042A000FD4F80839183A283B383C8DC80917A0A17
:1042B00090917B0AA0917C0AB0917D0AE889F989E6
:1042C000EC54FD4F80839183A283B383B7DC80914C
:1042D0007E0A90917F0AA091800AB091810AE889B4
:1042E000F989E854FD4F80839183A283B383A6DCD0
:1042F000E889F989E454FD4F81E020914E0A30911C
:104300004F0A2130310509F080E0808397DCE8898D
:10431000F989E354FD4F81E02091520A3091530A0C
:104320002130310509F080E0808388DCE889F98953
:10433000E254FD4F81E02091560A3091570A213016
:10434000310509F080E0808379DCE889F989E6525B
:10435000FD4F81E04091260A5091270A6091280A7A
:104360007091290A452B462B472B09F480E0808366
:1043700065DCE889F989E552FD4F81E040912A0A20
:1043800050912B0A60912C0A70912D0A452B462BD7
:10439000472B09F480E0808351DCE889F989E452F5
:1043A000FD4F81E040912E0A50912F0A6091300A12
:1043B0007091310A452B462B472B09F480E080830E
:1043C0003DDCE889F989E352FD4F81E04091FE0A26
:1043D0005091FF0A6091000B7091010B452B462B09
:1043E000472B09F480E0808329DCE889F989E252CF
:1043F000FD4F81E04091020B5091030B6091040B43
:104400007091050B452B462B472B09F480E08083E8
:1044100015DCE889F989E152FD4F81E04091060BF6
:104420005091070B6091080B7091090B452B462B9F
:10443000472B09F480E0808301DCE889F989E052A8
:10444000FD4F81E02091360A3091370A2130310545
:1044500009F080E08083F2DBE889F989EF51FD4FB4
:1044600081E020913A0A30913B0A2130310509F070
:1044700080E08083E3DBE889F989EE51FD4F81E03C
:1044800020913E0A30913F0A2130310509F080E049
:104490008083D4DB8091FE099091FF09A091000AEE
:1044A000B091010AE889F989ED51FD4F808391832C
:1044B000A283B383C3DB8091020A9091030AA09187
:1044C000040AB091050AE889F989E951FD4F808312
:1044D0009183A283B383B2DB8091060A9091070A8D
:1044E000A091080AB091090AE889F989E551FD4FC0
:1044F00080839183A283B383A1DBE889F989E253A6
:10450000FD4F81E040910E0A50910F0A6091100A10
:104510007091110A452B462B472B09F480E08083CC
:104520008DDBE889F989E153FD4F81E04091120A62
:104530005091130A6091140A7091150A452B462B6D
:10454000472B09F480E0808379DBE889F989E0531F
:10455000FD4F81E04091160A5091170A6091180AA8
:104560007091190A452B462B472B09F480E0808374
:1045700065DB8091060C9091070CA091080CB0911E
:10458000090CE889F989E154FD4F80839183A28366
:10459000B38354DB80910A0C90910B0CA0910C0C0E
:1045A000B0910D0CE889F989ED53FD4F808391831B
:1045B000A283B38343DB80910E0C90910F0CA091EA
:1045C000100CB091110CE889F989E953FD4F8083F3
:1045D0009183A283B38332DBE889F989EF52FD4FDF
:1045E00081E02091660A3091670A2130310509F097
:1045F00080E08083E889F989EE52FD4F1082E889D6
:10460000F989ED52FD4F108219DBE889F989EC52E6
:10461000FD4F81E02091620A3091630A213031051B
:1046200009F080E08083E889F989EB52FD4F108220
:10463000E889F989EA52FD4F108200DBE889F9899F
:10464000E952FD4F81E02091860A3091870A21309E
:10465000310509F080E08083F1DAE889F989E852D0
:10466000FD4F81E020918A0A30918B0A213031057B
:1046700009F080E08083E2DAE889F989E752FD4FAA
:1046800081E020918E0A30918F0A2130310509F0A6
:1046900080E08083D3DAE889F989E553FD4F81E032
:1046A0002091160C3091170C2130310509F080E073
:1046B0008083C4DAE889F989E453FD4F81E02091D1
:1046C0001A0C30911B0C2130310509F080E08083F9
:1046D000B5DAE889F989E353FD4F81E020911E0C9A
:1046E00030911F0C2130310509F080E08083A6DA7B
:1046F0000889198901511D4F8091AE0A9091AF0A26
:10470000A091B00AB091B10AF80180839183A2838D
:10471000B38394DAE888F988FDE0EF1AFDEFFF0A29
:104720008091B20A9091B30AA091B40AB091B50AEF
:10473000F70180839183A283B38380DA8091B60AE4
:104740009091B70AA091B80AB091B90AC888D988DF
:10475000F9E0CF1AFDEFDF0AF60180839183A2838F
:10476000B383F8014081518162817381141615066B
:104770001606170644F041E050E060E070E0408328
:10478000518362837383F701408151816281738118
:10479000141615061606170644F041E050E060E0D6
:1047A00070E04083518362837383181619061A06DA
:1047B0001B064CF081E090E0A0E0B0E0F6018083C1
:1047C0009183A283B3830E94DF15FC01D6018D90F3
:1047D0009D90AD90BC90D7014D915D916D917C9174
:1047E000D8010D911D912D913C910083118322835D
:1047F0003383448355836683778380869186A2863C
:10480000B386E889F9897096FB83EA83E889F98998
:10481000E553FD4F20812983E889F989E154FD4F53
:1048200080819181A281B381E889F989E952FD4FA4
:1048300020812A87E889F989E052FD4F20812C8365
:10484000E889F989EF52FD4F20812D83E889F989A4
:10485000EC52FD4F20812E83E889F989E352FD4F08
:1048600020812E87E889F989E652FD4F20812F8724
:10487000E889F989E454FD4F2080E889F989E358F3
:10488000FD4F3080E889F989ED51FD4F408151811C
:1048900062817381E889F989E055FD4F00811181BA
:1048A00022813381E889F989EC55FD4FC080D180A0
:1048B000E280F380E889F989E856FD4F8080918095
:1048C000A280B380E889F989E058FD4F408051808B
:1048D00062807380E889F98944AE55AE66AE77AEE2
:1048E000E05CFF4F80829182A282B382E889F989DD
:1048F000EC5BFF4FC082D182E282F382E889F989C2
:10490000E85BFF4F0083118322833383E889F989B1
:10491000E45BFF4F4083518362837383E889F989A5
:10492000E05BFF4F3082E889F989EF5AFF4F208220
:104930002F85E889F98921AF2E8522AF2C8123AFFD
:1049400040E450E060E070E0EC5AFF4F4083518358
:1049500062837383E889F989EE5AFF4F2E812083A1
:10496000E889F989ED5AFF4F2D812083E889F9897B
:10497000E85AFF4F2A852083E889F989E75AFF4FD3
:1049800080839183A283B383E889F989E35AFF4F37
:1049900089818083A889B98999968D919C919A97EC
:1049A0008633910509F083C28EEB90E1FD01EA5652
:1049B000FF4F9183808332961182108280EC90E1C8
:1049C000369691838083329611821082E889F98924
:1049D00087A590A94A97D1F482ED90E1E656FF4F62
:1049E00091838083E889F989E456FF4F1182108210
:1049F00084ED90E1E889F989EE55FF4F918380833A
:104A0000E889F989EC55FF4F1182108208891989CC
:104A10000A551F4FE889F989E453FD4F2081298306
:104A2000E889F989ED53FD4F80819181A281B3819D
:104A30008A879B87AC87BD87E889F989E852FD4F53
:104A400090819C83E889F989EF51FD4FA081AD8366
:104A5000E889F989EE52FD4FB081BE83E889F98972
:104A6000EB52FD4F20812E87E889F989E252FD4FF4
:104A70002080E889F989E552FD4F3080E889F9897D
:104A8000E354FD4F3081E889F989E258FD4F2081D8
:104A9000E889F989E951FD4F80819181A281B38133
:104AA000E889F989EC54FD4F40815181628173811D
:104AB000E889F989E855FD4FC080D180E280F38014
:104AC000E889F989E456FD4F80809180A280B38007
:104AD000E889F989EC57FD4F4080518062807380EE
:104AE000F80144A655A666A677A680AA91AAA2AA0E
:104AF000B3AAC4AAD5AAE6AAF7AA40AF51AF62AF3B
:104B000073AF84AF95AFA6AFB7AFE889F989EA5123
:104B1000FF4F2083E889F989E951FF4F3083D8019D
:104B200099963C9299979A962C929A97ED819B969A
:104B3000EC9380E490E0A0E0B0E0E889F989E651E8
:104B4000FF4F80839183A283B383E889F989E85179
:104B5000FF4F2E852083E889F989E751FF4F8E8129
:104B60008083E889F989E251FF4F9C819083E8892D
:104B7000F989E151FF4F8A859B85AC85BD8580838E
:104B80009183A283B383E889F989ED50FF4F99811E
:104B90009083D80159968D919C918633910509F0A7
:104BA000B8C18EEB90E1E889F989E45DFE4F91830D
:104BB0008083E889F989E25DFE4F1182108280ECE2
:104BC00090E1E889F989EC5CFE4F91838083E88964
:104BD000F989EA5CFE4F11821082F801878D90A15D
:104BE0004A97E1F482ED90E1E889F989E05DFE4FB2
:104BF00091838083E889F989EE5CFE4F11821082EF
:104C000084ED90E1E889F989E85CFE4F9183808327
:104C1000E889F989E65CFE4F11821082E888F988FC
:104C2000F4ECEF1AFEEFFF0AE889F989E353FD4F30
:104C300020812983E889F989E953FD4F8081918199
:104C4000A281B3818A879B87AC87BD87E889F98970
:104C5000E752FD4F90819C83E889F989EE51FD4F21
:104C60003080E889F989ED52FD4FA081AD83E88954
:104C7000F989EA52FD4F2080E889F989E152FD4F18
:104C8000C080E889F989E452FD4FD080E889F9892C
:104C9000E254FD4F3081E889F989E158FD4F2081C8
:104CA000E889F989E551FD4F80819181A281B38125
:104CB0008A8B9B8BAC8BBD8BE889F989E854FD4FBF
:104CC0004081518162817381E889F989E455FD4F02
:104CD00080809180A280B380E889F989E056FD4FF9
:104CE0004080518062807380E889F989E857FD4FE0
:104CF00080819181A281B381F70184A795A7A6A79E
:104D0000B7A740AA51AA62AA73AA84AA95AAA6AA7A
:104D1000B7AA40AF51AF62AF73AF8A899B89AC89A4
:104D2000BD8984AF95AFA6AFB7AFE889F989E458DC
:104D3000FE4F2083E889F989E358FE4F3083D7017D
:104D40009996DC9299979A96CC929A979B963C92D8
:104D500080E490E0A0E0B0E0E889F989E058FE4FF7
:104D600080839183A283B383E889F989E258FE4F57
:104D70002082E889F989E158FE4FBD81B083E88936
:104D8000F989EC57FE4F2C812083E889F989EB578C
:104D9000FE4F8A859B85AC85BD8580839183A283E8
:104DA000B383E889F989E757FE4F99819083D7014A
:104DB00059968D919C918633910509F0D2C08EEB66
:104DC00090E1E889F989EE53FE4F91838083E88969
:104DD000F989EC53FE4F1182108280EC90E1E88952
:104DE000F989E653FE4F91838083E889F989E4537A
:104DF000FE4F11821082F701878D90A14A97E1F44E
:104E000082ED90E1E889F989EA53FE4F918380832E
:104E1000E889F989E853FE4F1182108284ED90E110
:104E2000E889F989E253FE4F91838083E889F98903
:104E3000E053FE4F11821082E889F989E253FD4F59
:104E40008081882309F4B5C08A819B810E949A11D0
:104E5000E889F989E153FD4F8081882309F4AEC0C8
:104E6000C8010E949A118889998980539D4FDC015D
:104E70008C91882309F4A6C0C70165960FB6F894F3
:104E8000DEBF0FBECDBFDF91CF911F910F91FF907D
:104E9000EF90DF90CF90BF90AF909F908F907F90DA
:104EA0006F905F904F903F902F900C949A118C339D
:104EB0009105D9F482EC90E1E889F989EA56FF4F2F
:104EC00091838083E889F989E856FF4F1182108227
:104ED00084EC90E1E889F989E256FF4F9183808361
:104EE000E889F989E056FF4F6FCD8E9709F06ECDB6
:104EF00086EC90E1E889F989EA56FF4F9183808337
:104F0000E889F989E856FF4F118210828CEC90E114
:104F1000E1CF8C33910589F482EC90E1E889F9893D
:104F2000E45DFE4F91838083E889F989E25DFE4F5D
:104F30001182108284EC90E144CE8E9709F04DCE20
:104F400086EC90E1E889F989E45DFE4F91838083E6
:104F5000E889F989E25DFE4F118210828CEC90E1C4
:104F600030CE8C33910589F482EC90E1E889F9899F
:104F7000EE53FE4F91838083E889F989EC53FE4F0D
:104F80001182108284EC90E12ACF8E9709F033CF02
:104F900086EC90E1E889F989EE53FE4F9183808396
:104FA000E889F989EC53FE4F118210828CEC90E174
:104FB00016CF8A819B810E9459114ACFC8010E9455
:104FC000591151CFC70165960FB6F894DEBF0FBED9
:104FD000CDBFDF91CF911F910F91FF90EF90DF90A8
:104FE000CF90BF90AF909F908F907F906F905F9089
:104FF0004F903F902F900C945911AF92BF92CF9247
:10500000DF92EF92FF920F931F93CF93DF93EC0108
:105010008AE190E09AA789A78BE190E09CA78BA7F3
:1050200089E190E09EA78DA78FE090E098AB8FA7D5
:105030008EE190E09AAB89AB8EE090E09CAB8BABBD
:1050400085E490E09EAB8DAB84E490E098AF8FABAD
:10505000FE01EA55FF4F80E290E0928F818F81E25E
:1050600090E0948F838F8FE190E0968F858F10A2D0
:10507000178E12A211A214A213A283E490E096A3A9
:1050800085A382E490E090A787A3EA56FF4F83E2CE
:1050900090E0928F818F84E290E0948F838F82E200
:1050A00090E0968F858F10A2178E12A211A214A2E3
:1050B00013A281E490E096A385A380E490E090A7FA
:1050C00087A3E55CFE4F1182108232961182108216
:1050D000329611821082CE010E945320CE010E948E
:1050E0002F1FCE018E529E4F41E050E0FC0157A78A
:1050F00046A7DE01AE5FBD4F24E030E09F963C93B3
:105100002E939E975E01FEECAF1AFDEFBF0A28E0DA
:1051100030E0F50137A726A720E130E0FC0131831C
:10512000208321E130E0358324832FEF3FEF338369
:10513000228337832683628560876385618767E181
:1051400070E011967C936E9368E170E015967C9305
:105150006E93149713963C932E93129717963C9345
:105160002E9316971A966C911A9718966C93189717
:105170001B966C911B9719966C9319976DE170E0D3
:10518000F501718360836CE170E075836483338320
:105190002283378326836285608763856187BE01AA
:1051A0006E5A7C4FFB01608171818E01005C1C4F47
:1051B000F801C080D180E280F38006501109F80127
:1051C00000811181FC01158F048FC48AD58AE68A7B
:1051D000F78A6130710509F04EC0378F268FCE01F6
:1051E0008C5A9C4FFC01808191819E012C5B3C4F2D
:1051F000F901408151816281738128503109F9019F
:10520000208131815D963C932E935C9754964D930B
:105210005D936D937C935797019781F58FEF9FEF87
:105220005F969C938E935E97DE01AA5ABC4F8D9138
:105230009C9111971E974D915D916D917C91C25CEF
:10524000DC4F28813981F501358F248F448B558BB4
:10525000668B778B0197A9F48FEF9FEF978F868FDF
:10526000DF91CF911F910F91FF90EF90DF90CF9042
:10527000BF90AF900895578F468FB1CF81E090E0F7
:10528000CFCF81E090E0EACFEF92FF920F931F9390
:10529000CF93DF93EC010E941E1E00911E0B109114
:1052A0001F0B0E941E1EE0902E0BF0902F0B0E94F1
:1052B0001E1E2091460B3091470B1216130614F058
:1052C00021E030E0A701B801CE01845C9E4FDF9160
:1052D000CF911F910F91FF90EF900C949C13EF9240
:1052E000FF920F931F93CF93DF93EC010E941E1E3A
:1052F00000911A0B10911B0B0E941E1EE0902A0BAE
:10530000F0902B0B0E941E1E2091420B3091430BFC
:105310001216130614F021E030E0A701B801CE0107
:105320008A559F4FDF91CF911F910F91FF90EF9082
:105330000C949C13EF92FF920F931F93CF93DF93E4
:10534000EC010E941E1E0091160B1091170B0E947B
:105350001E1EE090260BF090270B0E941E1E20912F
:105360003E0B30913F0B1216130614F021E030E093
:10537000A701B801CE014096DF91CF911F910F9107
:10538000FF90EF900C949C138F929F92AF92BF92DC
:10539000CF92DF92EF92FF92CF93DF937B010E9437
:1053A0001E1EEC01F70182A093A0A4A0B5A0C68C9C
:1053B000D78CE0A0F1A08A819B818F30F7E29F0714
:1053C0000CF043C001969B838A838C819D818F3032
:1053D00027E29207ECF596012B7F21553109233006
:1053E000310530F096012B5531092330310518F481
:1053F00001969D838C83C6010E940307882359F17F
:10540000F601EE0FFF1FEE0FFF1FEE52F64F8082E8
:105410009182A282B382B501A401C6010E94511DEE
:10542000B601CE010E945C1A0E940C1F0E94DC1E75
:1054300090E080E0DF91CF91FF90EF90DF90CF90F0
:10544000BF90AF909F908F9008951B821A82BDCF1E
:105450001D821C82D0CF88ED93E00E94EC16E4CF31
:10546000CF93DF93EB010E941E1E6E8D7F8D0E94F5
:105470005C1A90E080E0DF91CF9108950E941E1E9B
:105480000E94961A8CE394E00E94EC160E94DF15AD
:105490000E947D1990E080E008950F931F93CF93B1
:1054A000DF93EC0188819981009759F02A813B8133
:1054B0002617370730F081E0DF91CF911F910F91D0
:1054C00008958B016F5F7F4F0E94FC61009759F038
:1054D000998388831B830A832C813D81232B59F771
:1054E000FC011082E8CF80E0E7CF0F931F93CF93AA
:1054F000DF93EC018B01D1DF28813981811112C04A
:105500002115310519F0C9010E94405A19821882EB
:105510001D821C821B821A82CE01DF91CF911F91C6
:105520000F9108951D830C8360E878E0C9010E9403
:10553000EE62F2CF70E060E0D8CF2F923F924F92B0
:105540005F926F927F928F929F92AF92BF92CF9213
:10555000DF92EF92FF920F931F93CF93DF93CDB71C
:10556000DEB7C659D1090FB6F894DEBF0FBECDBF66
:105570008C01FC0110821182128213821482158226
:105580001682178210861186128613861486158657
:10559000168617864C01F0E18F0E911CC4010E9403
:1055A0001214580186EAA80EB11CC5010E941214FB
:1055B0006801E4ECCE1AEEEFDE0AC6010E94121476
:1055C0007801FEE2EF1AFEEFFF0AC7010E94AE0F5C
:1055D000380182E0680E781EC3010E94AE0F2801D8
:1055E000EEEC4E1AEDEF5E0AC2010E94AE0FF8011A
:1055F000EE59FD4F1182108213821282158214829D
:10560000CF0198DFF801E859FD4F118210823296E0
:10561000118210823296118210823296118210828B
:105620003296108211821282138234961082319641
:105630001082319610823196118210823296118238
:105640001082329611821082329610823196108228
:105650003196108231961082118212821382349612
:105660001082118212821382349610821182128269
:105670001382349610821182128213823496108221
:105680001182128213823496108211821282138246
:105690003496108211821282138234961082118203
:1056A00012821382349610821182128213823496EF
:1056B0001082118212821382349610821182128219
:1056C00013823496108211821282138234961082D1
:1056D00011821282138234961082118212821382F6
:1056E000349610821182128213823496108231967F
:1056F00010823196108231961082118212821382AA
:105700003496108211821282138234961082118292
:105710001282138234961082319610823196108252
:105720003196108231961082319610823196108215
:105730003196108231961082319610823196108205
:1057400031961082319610823196108231961082F5
:1057500031961082319610823196108231961082E5
:1057600031961082319610823196108231961082D5
:1057700031961082319610821182128213823496F1
:105780001082118212821382349610821182128248
:105790001382D801A151BD4F8CE0E7E1F2E0019006
:1057A0000D928A95E1F7F801E550FD4F10821182C4
:1057B00012821382349610821182128213823496DE
:1057C00010821182128213823496118210823296D4
:1057D00011821082329611821082329610821182CA
:1057E00012821382349610821182128213823496AE
:1057F00010821182128213823496108211821282D8
:10580000138234961082118212821382349610828F
:105810001182128213823496118210823296118282
:105820001082329611821082329610821182128278
:10583000138234961082118212821382349610825F
:105840001182128213823496108231961082319620
:105850001082319611821082329611821082329615
:105860001182108232961082118212821382349633
:105870001082118212821382349610821182128257
:1058800013823496118210823296118210823296DF
:105890001182108232961182108232961182108209
:1058A00032961182108232961182108232961182C3
:1058B00010821801F4EA2F1AFCEF3F0AF10110825E
:1058C000319611821082329611821082CE01019699
:1058D0000E94121486E9FE013196D40101900D92C6
:1058E0008A95E1F7CE0101960E94121486E9FE0125
:1058F0003196D50101900D928A95E1F7CE0101967E
:105900000E94121486E9FE013196D60101900D9293
:105910008A95E1F788E5F801848BE655FF4F89E524
:105920008083EA56FF4F8AE58083CE0101960E946C
:10593000AE0F80E3FE013196D70101900D928A955A
:10594000E1F7CE0101960E94AE0F80E3FE01319691
:10595000D30101900D928A95E1F7CE0101960E9444
:10596000AE0F80E3FE013196D20101900D928A952F
:10597000E1F7C80142DBF1011082CA56DF4F0FB6D2
:10598000F894DEBF0FBECDBFDF91CF911F910F9175
:10599000FF90EF90DF90CF90BF90AF909F908F904F
:1059A0007F906F905F904F903F902F900895CF938E
:1059B000DF938091B1089091B208892B51F481E670
:1059C00093E00E94A459EC01B8DDD093B208C093D3
:1059D000B1088091B1089091B208DF91CF910895FC
:1059E000CF93DF938091B008811121C081E0809333
:1059F000B008DDDFEC0140960E946613CE018A55A7
:105A00009F4F0E946613CE01845C9E4F0E946613D6
:105A1000C059DD4F88819981AA81BB810196A11D62
:105A2000B11D88839983AA83BB831092B008DF914C
:105A3000CF910895CF93DF93EB0120E030E040E871
:105A40005FE36A817B818C819D810E941D5F811152
:105A500013C080E494E00E94EC16A9DFFC01EE592B
:105A6000FF4F10821182128213828E529E4FFC01D0
:105A7000108A118A128A138A20E030E040E85FE33E
:105A80006E817F81888599850E941D5F811113C079
:105A900080E594E00E94EC168ADFFC01E850FF4F9D
:105AA00010821182128213828E5F9D4FFC01108A38
:105AB000118A128A138A20E030E040E85FE36A85A9
:105AC0007B858C859D850E941D5F811113C080E6BA
:105AD00094E00E94EC166BDFFC01E257FE4F10824F
:105AE0001182128213828E5C9D4FFC01108A118AF2
:105AF000128A138A0E94DF150E947D1990E080E0CF
:105B0000DF91CF910895CF93DF93FC01EA59FD4FC8
:105B1000408151814115510501F1EC01C659DD4F1C
:105B2000288139818E599D4F24173507E8F4FC01EF
:105B3000808191810097A1F0820F931FFC018081E9
:105B40008A3031F08D3069F48EE798E00E94EC16CF
:105B500088819981019699838883DF91CF910895F7
:105B600080E00E947A08F4CF70E060E0BEDC198229
:105B70001882F3CFEF92FF920F931F93CF93DF938F
:105B80006115710541F480E0DF91CF911F910F9174
:105B9000FF90EF90089541155105A9F07B01EC01AC
:105BA0000C811D81040F151FB80177DC882359F380
:105BB000288139818C819D81B701820F931F0E94BA
:105BC000EE621D830C8381E0DFCFEF92FF920F9393
:105BD0001F93CF93DF93CDB7DEB764970FB6F894DA
:105BE000DEBF0FBECDBF7C01CB01BA018E010F5FBE
:105BF0001F4F22E044E00E948759FC0101900020E1
:105C0000E9F73197AF01481B590BBC01C701B2DF5F
:105C100064960FB6F894DEBF0FBECDBFDF91CF9173
:105C20001F910F91FF90EF900895EF92FF920F93C5
:105C30001F93CF93DF93CDB7DEB72D970FB6F894B0
:105C4000DEBF0FBECDBF7C01CB01BA012AE08E01C1
:105C50000F5F1F4FA8010E940E5BF801019000200A
:105C6000E9F73197AF01401B510BB801C70182DF43
:105C70002D960FB6F894DEBF0FBECDBFDF91CF914A
:105C80001F910F91FF90EF900895EF92FF920F9365
:105C90001F93CF93DF9300D000D01F921F92CDB7F8
:105CA000DEB77C01CB014AE08E010F5F1F4FB801C8
:105CB0000E94F65AF80101900020E9F73197AF01F0
:105CC000401B510BB801C70155DF28960FB6F89459
:105CD000DEBF0FBECDBFDF91CF911F910F91FF901F
:105CE000EF900895FB0101900020E9F73197AF0193
:105CF000461B570B3FCFFB01448155816081718169
:105D000039CFEF92FF920F931F93CF93DF93CDB7CD
:105D1000DEB72E970FB6F894DEBF0FBECDBF8C0155
:105D20007B01FC011182108213821282158214827F
:105D300001DC6BEC73E0C801D5DFF70162A173A150
:105D400084A195A12AE0AE014F5F5F4F7A010E94C6
:105D5000005BF70101900020E9F73197AF014E1980
:105D60005F09B701C80106DF6EE778E0C801BADF56
:105D7000C8012E960FB6F894DEBF0FBECDBFDF91DF
:105D8000CF911F910F91FF90EF900895CF92DF92E6
:105D9000EF92FF920F931F93CF93DF9300D000D029
:105DA000CDB7DEB76B017A018C010E591D4F68E348
:105DB00072E0C80197DF62EA76E0C80193DFF6017E
:105DC000848189831A8241E050E0BE016F5F7F4F7A
:105DD000C801D0DEB701C80158DF0E94DF15BC0141
:105DE000CE0101968EDFBE016F5F7F4FC80183DF5A
:105DF000CE0101960E941B1D26960FB6F894DEBFB9
:105E00000FBECDBFDF91CF911F910F91FF90EF900B
:105E1000DF90CF9008952F923F924F925F926F92B2
:105E20007F928F929F92AF92BF92CF92DF92EF922A
:105E3000FF920F931F93CF93DF93CDB7DEB7AF974A
:105E40000FB6F894DEBF0FBECDBF1C013B010E9410
:105E50005320C1010E942F1F0E94590A6B017C012F
:105E60009301220F331F220F331F3A832983220D00
:105E7000331D3D8B2C8B2C553D4F3C832B83D901FF
:105E80006D917D918D919C910E94235F9B01AC014E
:105E900060E074E284E796E40E94116120E030E063
:105EA00040E05FE30E94825F0E947E61688B798B95
:105EB0008A8B9B8B86E993E00E94EC1682EA96E03F
:105EC0000E94EC1680E794E00E94EC1682EA96E0CD
:105ED0000E94EC164AE0688979898A899B890E9428
:105EE0007C1682EA96E00E94EC168BE794E00E9412
:105EF000EC1682EA96E00E94EC1680E490E00E94A4
:105F0000E71682EA96E00E94EC1684E994E00E948B
:105F1000EC1682EA96E00E94EC16EB81FC8160812F
:105F20007181828193810E94BF1682EA96E00E946D
:105F3000EC168EE798E00E94EC160E9467160E940D
:105F4000E71AF1E06F16710409F460C022E06216EE
:105F5000710409F485C0A101405F5F4F5FA74EA7A0
:105F600021015EE2451A5EEF550AF101E652FD4F4E
:105F700080818B87D101A550BD4FBE83AD83E55B8A
:105F8000FF4FFF8BEE8B9101295C3C4F39A328A377
:105F9000A10149585D4F5D874C878DE890E09F8F48
:105FA0008E8FA5E1B0E0BF87AE878EA59FA50E942A
:105FB0000E11882309F47EC084EA94E00E94EC1656
:105FC0000E94DF1524E030E0DC0197963C932E938D
:105FD000969794E0692E712CC301AF960FB6F89492
:105FE000DEBF0FBECDBFDF91CF911F910F91FF900C
:105FF000EF90DF90CF90BF90AF909F908F907F9069
:106000006F905F904F903F902F900895F101EA5567
:10601000FF4FFFA7EEA72101F2E04F0E5F1EF10137
:10602000E552FD4F20812B87A10141505D4F5E83DA
:106030004D83C101895D9C4F9F8B8E8BD101A85CE4
:10604000BC4FB9A3A8A3E256F109FD87EC872EE85F
:1060500030E03F8F2E8F46E150E05F874E87A5CF1F
:10606000C101845C9E4F9FA78EA721019EEC491A17
:106070009DEF590AF101E452FD4FA081AB87B7961D
:10608000FE83ED839101275D3C4F3F8B2E8BA10159
:10609000475C5C4F59A348A3C10185589D4F9D871C
:1060A0008C87AFE8B0E0BF8FAE8FE7E1F0E0FF870D
:1060B000EE877BCF8EA59FA50E94FF1081117CCF1C
:1060C00086E993E00E94EC168AED94E00E94EC16BB
:1060D000EEA5FFA584810E947A0881EE94E00E94DB
:1060E000EC168EE798E00E94EC1681E090E0AC851B
:1060F000BD858D939C9341E050E06EA57FA5C101C5
:1061000045DE8EA59FA50E949A11EEA5FFA5E05C35
:10611000FF4F80810EA51FA504581F4F882309F447
:10612000C1C08EA59FA50E941D11F8011082C20159
:106130000E944C0FEEA5FFA5EE5AFF4F60837183BE
:1061400082839383ED81FE811082118212821382F9
:10615000F101E550FD4F10821182128213823496B4
:10616000108211821282138234961082118212825E
:10617000138286E090E0AC85BD858D939C9346E0CC
:1061800050E06EA57FA5C10101DE61E070E08EA543
:106190009FA50E948D1989819A81855D9C4FF1018F
:1061A000E80FF91FFBA3EAA389819A81835F9C4FC3
:1061B0009101280F391F3DA32CA389819A81855015
:1061C0009D4FA101480F591F5FA34EA31F82188640
:1061D00019861A868EA59FA5459699A788A7C101FD
:1061E000860D971DDC01A95CBC4FBBA7AAA78981BE
:1061F0009A81820D931DFC01ED51FD4FF98FE88FBF
:10620000910120593D4F3D8F2C8F4C895D894C5514
:106210005D4F5DA74CA748A559A56FE6AEA5BFA5E4
:106220008D919C910E944F0CEAA5FBA5808188234B
:1062300059F00AA11BA12CA13DA14EA15FA1B20161
:106240008EA59FA50E94E60F0E94590A6C157D0538
:106250008E059F0578F50E94590A6C157D058E05FF
:106260009F0508F460C087E59DE00E94F7071816B7
:1062700019060CF498C010E01C821B828EA59FA505
:106280000E940E11882309F4AFC084E595E00E94B6
:10629000EC168EA59FA50E940E11811101C08B8561
:1062A0008B8757C28EA59FA50E943B1181E0D80124
:1062B0008C933DCF0E94590A4B015C018C189D08BC
:1062C000AE08BF08A88DB98D2D913D914D915C917F
:1062D000A8EEB3E00E946B60681579058A059B05FE
:1062E00008F0B9CF8EA59FA50E945911B1E06B1699
:1062F000710471F1E2E06E16710409F442C084E6A3
:1063000092E00E94EC160E94DF150E947D1980E049
:1063100095E00E94EC160E94DF1522E030E0FC01BF
:1063200037A326A32AC00E94590A4B015C01A88DFD
:10633000B98D2D913D914D915C91A8EEB3E00E94F5
:106340006B60681579058A059B0508F08CCFCACF6C
:1063500080E692E00E94EC160E94DF150E947D19F3
:1063600085E195E00E94EC160E94DF1522E030E006
:10637000DC0197963C932E93969782E0682E712CC1
:106380002BCE8CE592E00E94EC160E94DF150E9455
:106390007D198AE295E00E94EC160E94DF15FC014F
:1063A00077A266A219CE87E59DE00E94D5078F7D72
:1063B0008534910509F05FCF8FE395E00E94EC16DC
:1063C0000E94DF15E1E0DC01D496EC9388E592E0D1
:1063D0000E94EC160E94DF150E947D1921E030E03A
:1063E0003C832B8311E04ACF8EA59FA50E94FF100E
:1063F00081114BCF111149CFAE89BF896D917C912D
:10640000072E000C880B990B0E94235F9B01AC01A7
:10641000ED81FE8160817181828193810E941D5F87
:1064200087FF33CF8EA59FA50E945012AC8DBD8DE6
:106430004D915D916D917C91088919892A893B89DB
:10644000040F151F261F371F4017510762077307D8
:1064500028F483EE93E00197F1F7F6CF2F8138858A
:1064600049855A852F5F3F4F4F4F5F4F2F833887A6
:1064700049875A87ACA5BDA52D913D914D915C9161
:10648000A3E0B0E00E946B609B01AC016F81788556
:1064900089859A850E944F60672B682B692B41F490
:1064A00084E592E00E94EC160E94DF150E947D199F
:1064B0008EA59FA50E94E610EC8DFD8D4081518137
:1064C00062817381088919892A893B89040F151F04
:1064D000261F371F401751076207730708F034C1A2
:1064E00083EE93E00197F1F7F5CF8EA59FA50E946B
:1064F0001D11F8011082A5C10E94590A9B01AC012F
:10650000281939094A095B092F83388749875A872F
:10651000A981BA812D913D914D915C91A8EEB3E096
:106520000E946B602F81388549855A8562177307F1
:106530008407950708F0F0C18EA59FA50E94591108
:1065400031E06316710451F142E06416710489F17F
:1065500084E692E00E94EC160E94DF150E947D19ED
:1065600080E095E0FFCE0E94590A6F837887898783
:106570009A87A981BA812D913D914D915C91A8EEA8
:10658000B3E00E946B602F81388549855A85621778
:1065900073078407950708F0C7C1CECF80E692E065
:1065A0000E94EC160E94DF150E947D1985E195E09E
:1065B000B0CE8CE592E00E94EC160E94DF150E949E
:1065C0007D198AE295E00E94EC160E94DF15DC013D
:1065D00097967C926E929697FFCC87E59DE00E94FD
:1065E000D5078F7D8534910509F0A6C18FE395E02D
:1065F0000E94EC160E94DF1521E0FC0124AB88E527
:1066000092E00E94EC160E94DF150E947D1941E085
:1066100050E05C834B8311E090C11111A5C1EE895C
:10662000FF8960817181072E000C880B990B0E94F5
:10663000235F9B01AC01AD81BE816D917D918D91F8
:106640009C910E941D5F87FF8FC18EA59FA50E9410
:106650005012BFEFCB1ADB0AEB0AFB0AEE85FF856F
:106660004081518162817381088919892A893B8916
:10667000040F151F261F371F4017510762077307A6
:1066800028F483EE93E00197F1F7F6CFAC89BD894A
:106690002D913D914D915C91A3E0B0E00E946B6023
:1066A0009B01AC01C701B6010E944F60672B682BAC
:1066B000692BC1F484E592E00E94EC160E94DF157C
:1066C0000E947D1986E993E00E94EC1683E995E02B
:1066D0000E94EC16C701B6010E94BF168EE798E033
:1066E0000E94EC168EA59FA50E94E610EE85FF8500
:1066F0004081518162817381088919892A893B8986
:10670000040F151F261F371F401751076207730715
:1067100008F0DCC083EE93E00197F1F7F5CF0E941B
:10672000DF15FC01C28AD38AE48AF58AA0C10E94DF
:10673000DF15DC015696CD92DD92ED92FC925997D1
:1067400096C10E94FF100DC12B813C81232B09F4BF
:1067500062CD62E070E08EA59FA50E948D1986E94A
:1067600093E00E94EC168AED94E00E94EC16AEA530
:10677000BFA514968C910E947A0888E695E00E9445
:10678000EC168EE798E00E94EC16EB81FC81EF2B73
:1067900009F58BE795E00E94EC1682EA96E00E94EC
:1067A000EC1682ED93E00E94EC168E859F850E9488
:1067B000E71682EA96E00E94EC168DE296E00E94CF
:1067C000EC16FB858F2F90E00E94E7160E94DF15E4
:1067D0000E947D190E9467160E94E71A86E993E0DD
:1067E0000E94EC168AED94E00E94EC16AEA5BFA5BF
:1067F00014968C910E947A088FE795E00E94EC161F
:106800008EE798E00E94EC160E94590A4B015C0149
:10681000ED81FE811082118212821382EEA5FFA506
:10682000E05CFF4F80810EA51FA504581F4F8823F1
:1068300009F45BCE8EA59FA50E943B1181E0D80193
:106840008C93C2010E944C0FEEA5FFA5EE5AFF4F9C
:106850006083718382839383F101E550FD4F108241
:106860001182128213823496108211821282138254
:1068700034961082118212821382C2010E944C0F40
:10688000688F798F8A8F9B8FC2010E944C0FC12C19
:10689000D12C7601C101860D971D9C01295C3C4FCE
:1068A0003D8F2C8F89819A81820D931DAC014D51B2
:1068B0005D4F5A834983C10180599D4F9F878E87C1
:1068C000AC89BD89AC55BD4FBD8BAC8BEB81FC81D8
:1068D000EF2B09F04DC048A559A56FE6AEA5BFA5A1
:1068E0008D919C910E944F0CEC8DFD8D80818823B1
:1068F00059F00AA11BA12CA13DA14EA15FA1B2019B
:106900008EA59FA50E94E60F0E94590A6815790579
:106910008A059B0508F0F0CD0E94590A6815790593
:106920008A059B0508F41FCE87E59DE00E94F707C6
:10693000181619060CF451CE10E05AE0C516D10411
:10694000E104F1043CF4AD81BE811D921D921D92C3
:106950001C921397BB858EA59FA5B111F2CE0E9404
:106960000E11882309F459CE84E595E00E94EC16B7
:1069700086E993E00E94EC168AED94E00E94EC1602
:10698000AEA5BFA514968C910E947A0881EA95E085
:106990000E94EC168EE798E00E94EC16C2010E945D
:1069A0004C0FE8A1F9A1EF2BA1F06B017C01288D20
:1069B000398D4A8D5B8DC21AD30AE40AF50AF7FEB7
:1069C00008C0F094E094D094C094C11CD11CE11C88
:1069D000F11C4B815C81452B19F58BE795E00E94FA
:1069E000EC1682EA96E00E94EC1682ED93E00E949B
:1069F000EC168E8D9F8D0E94E71682EA96E00E942B
:106A0000EC168DE296E00E94EC16C701B6010E94DA
:106A1000235F42E00E940B1B0E94DF150E947D193C
:106A200085E090E0AC85BD858D939C9345E050E07A
:106A30006EA57FA5C101AAD98EA59FA50E94591157
:106A40000E9467160E94E71AB1E06B16710409F400
:106A500066CEE2E06E16710409F469CE0E94DF157D
:106A6000DC011E96CD92DD92ED92FC9251970E9430
:106A7000DF150E94861CEC85FD851182108250E096
:106A800040E06EA57FA5C10181D970E060E08EA5D0
:106A90009FA50E948D190E94DF15EB81FC81DC010E
:106AA0009796FC93EE9396973F0196CAFA01DB0105
:106AB000A158BF4F2C91222331F122E030E0DB01BD
:106AC000AF57BF4F4C91442311F023E030E0DB017E
:106AD000A058BF4F4C91442311F024E030E0DB017B
:106AE000AE57BF4F4C91442311F026E030E0408177
:106AF00051814217530761F0121613063CF431839B
:106B00002083A90143C930E020E0D9CF118210824F
:106B100008952F923F924F925F926F927F928F9241
:106B20009F92AF92BF92CF92DF92EF92FF920F931C
:106B30001F93CF93DF93CDB7DEB7CC54D1090FB6F7
:106B4000F894DEBF0FBECDBF1C012A013B010F83AD
:106B5000188729873A87A4960EAD1FADA497FC012C
:106B6000E151FD4F60817181828193810E94235F99
:106B7000A30192010E94825F0E9479616D877E87E6
:106B80008F87988BF101ED50FD4F6081718182817B
:106B900093810E94235F2F81388549855A850E9401
:106BA000825F0E9479616B8B7C8B8D8B9E8BF10158
:106BB000E950FD4F60817181828193810E94235F42
:106BC000A70196010E94825F0E9479616FA378A756
:106BD00089A79AA70E94590A6F83788789879A871D
:106BE000F101E459FD4F1182108232961182108218
:106BF000D10157961C921E92569759961C921E923E
:106C000058975B961C921E925A975D961C921E9204
:106C10005C975F961C921E925E97E25CF140118237
:106C20001082329611821082329611821082329630
:106C300011821082329611821082E257FF4F118228
:106C40001082329611821082329611821082329610
:106C500011821082329611821082EA5CFE4FA114DA
:106C6000B10461F0C501B0E0A0E0408151816281D2
:106C7000738184179507A607B70714F0A080B18029
:106C8000F101EC57FD4F80819181A281B381811484
:106C9000910441F0A40170E060E0481759076A07C9
:106CA0007B070CF04C01F101E857FD4F8081918189
:106CB000A281B3810115110541F0A80170E060E0E7
:106CC000481759076A077B070CF08C012101B0E1D6
:106CD0004B0E511CC501B0E0A0E0F10184AF95AFAF
:106CE000A6AFB7AF3101F6EA6F0E711CB12CA12C23
:106CF000D3019C968D929D92AD92BC929F9751012B
:106D0000B4ECAB1ABEEFBB0A30E020E0F50104A7FB
:106D100015A726A737A70E94DF150E94DF150E943E
:106D2000DF150E94DF15DC011E962D913D914D91DE
:106D30005C9151972F8B388F498F5A8F0E94DF15A6
:106D4000DC0152962D913D914D915C9155972BA36D
:106D50003CA34DA35EA30E94DF15DC0156962D9146
:106D60003D914D915C9159972F8F38A349A35AA318
:106D7000F101E550FD4F1082118212821382349688
:106D80001082118212821382349610821182128232
:106D900013823496118210823296118210823296BA
:106DA0001182108232962F89388D498D5A8D208319
:106DB00031834283538334968BA19CA1ADA1BEA1A4
:106DC00080839183A283B38334962F8D38A149A108
:106DD0005AA12083318342835383A596EFACA597B4
:106DE0000D851E852F8538894F89588D698D7A8D3F
:106DF000C2010E94B2118823F9F080E592E00E945E
:106E0000EC168DE494E00E94EC16F101EA59FF4F74
:106E10006081718182819381E757FD4F20813181AB
:106E2000428153810E944F60CA01B9010E94BF167E
:106E30000E94DF150E947D19A696EFACA6970B89DC
:106E40001C892D893E894BA15CA16DA17EA1C30146
:106E50000E94B2118823F9F08CE492E00E94EC16B3
:106E60008DE594E00E94EC16F101E450FF4F608143
:106E7000718182819381E950FE4F2081318142816D
:106E800053810E944F60CA01B9010E94BF160E943F
:106E9000DF150E947D19A796EFACA7970FA118A543
:106EA00029A53AA54F8D58A169A17AA1C5010E94D3
:106EB000B2118823F9F088E492E00E94EC168DE686
:106EC00094E00E94EC16F101EE56FE4F6081718154
:106ED00082819381EB59FE4F208131814281538120
:106EE0000E944F60CA01B9010E94BF160E94DF15BF
:106EF0000E947D19D10155961C92F101E555FF4F75
:106F00001082EA56FF4F10820E9467160E94E71A0D
:106F1000C2010E947913C3010E947913C5010E9426
:106F2000791381E090E0F101E958FD4F918380836E
:106F30007101B7E8EB1ABDEFFB0AF701918380837B
:106F4000810105581D4FD8018D939C9341E050E07D
:106F5000B201C1010E94C62EF70140815181B301E7
:106F6000C1010E94C62ED8014D915C91B501C101AD
:106F70000E94C62E11E0F101E45AFC4F1083C201B9
:106F80000E949A11C3010E949A11C5010E949A1190
:106F900064E670E080E090E00E94280AD101AC58DD
:106FA000BD4F1C9391012B583D4FF9011083C10136
:106FB0008A589D4FFC011083A596FFADA597F1114E
:106FC0000FC0A6964FADA697411105C0A7965FAD1D
:106FD000A797552349F1C10185579F4FFC011082A6
:106FE000A696FFADA697F11105C0C1018F5D9E4F1A
:106FF000FC011082A796FFADA797F11105C0C10152
:1070000089549E4FFC011082A596FFADA597FC9375
:10701000A696EFADA697D901EC93F101EA58FD4F82
:10702000A7962FADA7972083F101E957FF4F108254
:10703000118212821382EA56FF4F1082118212824D
:107040001382EA56FF4F1082118212821382C2010C
:107050000E94F516C3010E94F516C5010E94F5169F
:10706000C2010E94BB12C3010E94BB12C5010E9453
:10707000BB120E94DF15DC01D4968C918D871DA672
:107080001EA61FA618AA19AA1AAA1BAA1CAA1DAADC
:107090001EAA1FAA18AE912C812CF101EC58FD4FAD
:1070A000FC8BEB8B91012B583D4F38A72FA3A101EF
:1070B0004A585D4F5CA74BA7C10189589D4F219647
:1070C0009FAF8EAF2197D101A758BD4F2396BFAF79
:1070D000AEAF239737962596FFAFEEAF2597275E85
:1070E00031403EAF2DAF4F535F4F27965FAF4EAF4E
:1070F0002797069629969FAF8EAF2997A35DB1403B
:10710000BAAFA9AF55962B96BFAFAEAF2B97EF5343
:10711000F140FCAFEBAF75962D96FFAFEEAF2D971C
:10712000AB89BC898C9181110AC0EFA1F8A580813F
:10713000811105C0ABA5BCA58C91882319F0BD8534
:10714000BB2369F081010A591D4FD8018D919C9193
:10715000892B09F479C6C1010E94832DF6CF2196AF
:107160004EAD5FAD2197B201C101A0DC23964EADBB
:107170005FAD2397B301C10199DC25964EAD5FAD9C
:107180002597B501C10192DCC2010E942613C301FB
:107190000E942613C5010E942613EDADFEAD80812D
:1071A000882309F44EC0C2010E94F516A1014B5D6F
:1071B0005F4F6FE6D10150968D919C910E944F0CCC
:1071C0002796EEADFFAD27978081882379F0810166
:1071D000055D1C4F9101235F3C4FA10145505D4F60
:1071E000B1016E527E4FC2010E94E60FADADBEAD41
:1071F0001C92A596BFADA597BB2319F12996EEADBC
:10720000FFAD29978081811116C02F89388D498D56
:107210005A8D12161306140615069CF02DA93EA9C8
:107220004FA958AD2F5F3F4F4F4F5F4F2DAB3EAB38
:107230004FAB58AF06C08F89988DA98DBA8DB7FF17
:10724000EDCFF101EC5DFE4F8081882309F44DC044
:10725000C3010E94F5162B964EAD5FAD2B976FE6DE
:10726000A9ADBAAD8D919C910E944F0CF101E85CE3
:10727000FC4F8081882379F08101015D1C4F9101D1
:107280002F5E3C4FA10141505D4FB1016E5F7D4FBC
:10729000C3010E94E60FF101EC5DFE4F1082A6963D
:1072A000BFADA697BB2309F1E65AFE4F808181113D
:1072B00016C02BA13CA14DA15EA112161306140607
:1072C00015069CF029A93AA94BA95CA92F5F3F4F4D
:1072D0004F4F5F4F29AB3AAB4BAB5CAB06C08BA1BA
:1072E0009CA1ADA1BEA1B7FFEDCFF101E654FE4FC9
:1072F0008081882309F44DC0C5010E94F5162D96A2
:107300004EAD5FAD2D976FE6ABADBCAD8D919C9151
:107310000E944F0CF101E75CFC4F8081882379F0DB
:1073200081010D5C1C4F91012B5E3C4FA1014D5F13
:107330005C4FB1016E5C7D4FC5010E94E60FF1010B
:10734000E654FE4F1082A796BFADA797BB2309F165
:10735000EB53FF4F8081811116C02F8D38A149A1B9
:107360005AA112161306140615069CF02DA53EA56B
:107370004FA558A92F5F3F4F4F4F5F4F2DA73EA7F7
:107380004FA758AB06C08F8D98A1A9A1BAA1B7FF8E
:10739000EDCFF101E557FF4F8081882309F466C0E6
:1073A000D101AB5DBC4F8D919C91D10156962D9131
:1073B0003C915797281739070CF458C058962D91CF
:1073C0003C915997281739070CF450C05A962D91C3
:1073D0003C915B97281739070CF448C05C962D91B7
:1073E0003C915D97281739070CF440C05E962D91AB
:1073F0003C9128173907D4F1108281010E591D4F95
:1074000066E973E0C8010E94722E6FEA75E0C80158
:107410000E94722EF10185A196A1A7A1B0A588278F
:107420009927AA27BE776BEC75E0892B8A2B8B2BCB
:1074300011F468ED75E0C8010E94722E6EE778E0E5
:10744000C8010E94722EA596FFADA597FF2309F4EF
:10745000B1C1F101EE52FE4F108A118A128A138ACD
:10746000E057F1401082118212821382F101EF5D28
:10747000FE4F8081882309F468C0D101A95DBC4F0B
:107480008D919C911197AB57B2402D913C911197E2
:10749000281739070CF459C012962D913C91119779
:1074A000281739070CF451C012962D913C91119771
:1074B000281739070CF449C012962D913C91119769
:1074C000281739070CF441C012962D913C912817CA
:1074D0003907DCF1108281010E591D4F66E973E016
:1074E000C8010E94722E65EE75E0C8010E94722EDE
:1074F000E9ADFAAD85899689A789B08D8827992746
:10750000AA27BE776BEC75E0892B8A2B8B2B11F4A5
:1075100068ED75E0C8010E94722E6EE778E0C80140
:107520000E94722EA696FFADA697FF2309F446C1CE
:10753000F101EE5FFD4F108A118A128A138AEA5018
:10754000F1401082118212821382F101E954FE4F40
:107550008081882309F468C0D101A75DBC4F8D915B
:107560009C911197A75EB1402D913C9111972817DE
:1075700039070CF459C012962D913C911197281798
:1075800039070CF451C012962D913C911197281790
:1075900039070CF449C012962D913C911197281788
:1075A00039070CF441C012962D913C9128173907E8
:1075B000DCF1108281010E591D4F66E973E0C801AC
:1075C0000E94722E61E076E0C8010E94722EEBAD3F
:1075D000FCAD85899689A789B08D88279927AA2728
:1075E000BE776BEC75E0892B8A2B8B2B11F468ED41
:1075F00075E0C8010E94722E6EE778E0C8010E9413
:10760000722EA796FFADA797FF2309F4DBC0F10107
:10761000EE5CFD4F108A118A128A138AE45AF1092E
:10762000108211821282138260E0C2010E94341221
:10763000882369F0F101EE59FF4F10821182128206
:107640001382E059FE4F108A118A128A138A60E071
:10765000C3010E943412882369F0F101E850FF4F02
:107660001082118212821382E65FFE4F108A118A05
:10767000128A138A60E0C5010E943412882369F0DF
:10768000F101E257FE4F1082118212821382EC55F3
:10769000FF4F108A118A128A138AF101E557FF4FB2
:1076A0008081AB89BC898C93EA56FF4F8081EFA122
:1076B000F8A58083F101E954FE4F8081ABA5BCA5FC
:1076C0008C93E555F14020813181428153812F8B8C
:1076D000388F498F5A8FEA56FF4F80819181A2815E
:1076E000B3818BA39CA3ADA3BEA3EA56FF4F208119
:1076F0003181428153812F8F38A349A35AA30E941D
:10770000DF152F89388D498D5A8DDC011E962D93FA
:107710003D934D935C9351970E94DF152BA13CA1A3
:107720004DA15EA1DC0152962D933D934D935C9348
:1077300055970E94DF152F8D38A149A15AA1DC0170
:1077400056962D933D934D935C9359970E946716DF
:10775000EB89FC898081882309F46AC00E94590A58
:107760002F81388549855A856217730784079507E5
:1077700068F50E94590A2F81388549855A85621714
:1077800073078407950708F053C00E94590A6B01DC
:107790007C01F101ED51FD4F208131814281538106
:1077A000A8EEB3E00E946B606C157D058E059F0509
:1077B00050F13EC07FE1872E912C58CE60E2862E9C
:1077C000912CC3CE51E2852E912C2ECF0E94590AC6
:1077D0006B017C012F81388549855A85C21AD30AED
:1077E000E40AF50AF101ED51FD4F2081318142811A
:1077F0005381A8EEB3E00E946B606C157D058E0589
:107800009F0508F0B6CF64E672E081010E591D4F66
:10781000C8010E94722E6EE778E0C8010E94722EA5
:1078200060E075E0C8010E94722E42E0842E912C27
:10783000AFA1B8A58C91882309F45DC00E94590AB4
:107840002F81388549855A85621773078407950704
:1078500008F50E94590A2F81388549855A85621793
:1078600073078407950708F046C00E94590A6B0108
:107870007C01F101E951FD4F208131814281538129
:10788000A8EEB3E00E946B606C157D058E059F0528
:10789000E8F031C00E94590A6B017C012F813885C4
:1078A00049855A85C21AD30AE40AF50AF101E95159
:1078B000FD4F2081318142815381A8EEB3E00E94C7
:1078C0006B606C157D058E059F0518F660E672E00D
:1078D00081010E591D4FC8010E94722E6EE778E09B
:1078E000C8010E94722E65E175E0C8010E94722EE7
:1078F00032E0832E912CABA5BCA58C91882309F492
:107900005DC00E94590A2F81388549855A856217C2
:1079100073078407950708F50E94590A2F81388557
:1079200049855A85621773078407950708F046C092
:107930000E94590A6B017C01F101E551FD4F208144
:10794000318142815381A8EEB3E00E946B606C15D7
:107950007D058E059F05E8F031C00E94590A6B0134
:107960007C012F81388549855A85C21AD30AE40AD9
:10797000F50AF101E551FD4F2081318142815381AA
:10798000A8EEB3E00E946B606C157D058E059F0527
:1079900018F66CE572E081010E591D4FC8010E9476
:1079A000722E6EE778E0C8010E94722E6AE275E0DE
:1079B000C8010E94722E22E0822E912C87E59DE064
:1079C0000E94F707181619060CF040C087E59DE0E5
:1079D0000E94D5078F7D85349105C1F56FE375E071
:1079E000C1018E599D4F0E94722E88E592E00E943F
:1079F000EC160E94DF150E947D19F101E557FF4F3B
:107A00001082EA56FF4F1082EA56FF4F1082AB8970
:107A1000BC891C92EFA1F8A51082ABA5BCA51C9255
:107A2000B1E0BD8788248394912C6DE176E0C1019B
:107A30008E599D4F0E94722EEB89FC891082AFA156
:107A4000B8A51C92EBA5FCA5108203C0811491047B
:107A500061F7C1010E94832DF101E259FD4F808140
:107A600091810196918380838D3291400CF458CBA3
:107A7000D101AA59BD4F8D919C911197892B09F085
:107A80004FCB14968D919C91892B09F049CB118293
:107A900010823297808191818130910589F1823005
:107AA000910509F4F0C0892BC9F464E572E0810105
:107AB0000E591D4FC8010E94722E0E94DF15BC0195
:107AC000CE0101960E94812EBE016F5F7F4FC801DB
:107AD0000E947B2ECE0101960E941B1DF101E459EC
:107AE000FD4F808191810196833091050CF0A9C1F1
:107AF00091838083F101E659FD4F1182108210CBF2
:107B00000E94DF158C01FC0180819181A281B381EB
:107B1000181619061A061B0644F081E090E0A0E052
:107B2000B0E080839183A283B383F801848195813F
:107B3000A681B781181619061A061B0644F081E0C3
:107B400090E0A0E0B0E084839583A683B783F8013A
:107B500080859185A285B385181619061A061B061D
:107B600044F081E090E0A0E0B0E080879187A287B8
:107B7000B3871A8219821C821B821E821D82CE014B
:107B800001960E949A2A68E374E0CE0101960E9451
:107B9000722E6DE474E0CE0101960E94722ED8011F
:107BA0001E966D917D918D919C9151970E94235FBE
:107BB0006B017C01F80160817181828193810E9457
:107BC000235F9B01AC01C701B6010E941161AB01AB
:107BD000BC01CE0101960E94E52D6DE574E0CE0159
:107BE00001960E94722ED80152966D917D918D91D1
:107BF0009C9155970E94235F6B017C01F801648181
:107C00007581868197810E94235F9B01AC01C7012A
:107C1000B6010E941161AB01BC01CE0101960E9428
:107C2000E52D6DE674E0CE0101960E94722ED8011A
:107C300056966D917D918D919C9159970E94235FED
:107C40006B017C01F80160857185828593850E94B6
:107C5000235F9B01AC01C701B6010E941161AB011A
:107C6000BC01CE0101960E94E52DBE016F5F7F4FE2
:107C700081010E591D4FC8010E947B2ECE01019635
:107C80000E941B1D1ACFD10158962D913C915997F6
:107C900056968D919C91821793070CF4C90197FF1A
:107CA00002C090E080E0F101228D338D2817390762
:107CB0000CF49C01D1015C968D919C9182179307E5
:107CC0000CF4C901F101068CF78DE02DFC87EB87E0
:107CD000E817F90714F49C878B87F101E255FF4FF1
:107CE00020813181329780819181821793070CF432
:107CF000C90197FF02C090E080E0F101E055FF4F1D
:107D000020813181281739070CF49C01F101EE54D0
:107D1000FF4F80819181821793070CF4C901F10113
:107D2000EC54FF4FC080D180C816D9060CF46C010A
:107D3000F101EC5BFE4F208131813297808191818E
:107D4000821793070CF4C90197FF02C090E080E00E
:107D5000F101EA5BFE4F20813181281739070CF4CD
:107D60009C01F101E85BFE4F8081918182179307AE
:107D70000CF4C901F101E65BFE4FE080F180E816EA
:107D8000F9060CF47C0166E973E081010E591D4F80
:107D9000C8010E94722E69E276E0C8010E94722E2C
:107DA000F101E957FF4F4081518162817381C80120
:107DB0000E94152E6DE474E0C8010E94722E6B853E
:107DC0007C85C8010E94452E6CE276E0C8010E94C5
:107DD000722EF101E35EFE4F608171818281938199
:107DE00024E630E040E050E00E947B6084E6829F21
:107DF000B001839F700D1124C8010E94452E6DE5CE
:107E000074E0C8010E94722EB601C8010E94452E7E
:107E10006FE276E0C8010E94722EF101ED54FE4F30
:107E20004081518162817381C8010E94152E6DE6E7
:107E300074E0C8010E94722EB701C8010E94452E4D
:107E40003CCE1182108256CE82E396E00E94EC1660
:107E5000A596BFADA597BB2379F181149104B9F51F
:107E6000ED85E11134C084E492E00E94EC160E949A
:107E7000DF150E947D19A696FFADA697FF2341F05E
:107E800080E492E00E94EC160E94DF150E947D19AA
:107E9000A7964FADA7974423D1F081149104B9F46C
:107EA0005D85511114C08CE392E00E94EC160E9493
:107EB000DF150E947D190BC0A6963FADA697332310
:107EC00039F38114910419F42D852223C9F285E038
:107ED00090E0D101A958BD4FB887AF838D939C9393
:107EE000810107581D4FF801918380839101255826
:107EF0003D4F3A8B298BD9018D939C9345E050E0FF
:107F0000B201C1010E94C62EF80140815181B30126
:107F1000C1010E94C62EA989BA894D915C91B50113
:107F2000C1010E94C62EC1010E947011F101EE59DB
:107F3000FF4F20813181428153812F8F38A349A384
:107F40005AA3EA56FF4F80819181A281B3818B8F22
:107F50009C8FAD8FBE8FEA56FF4FC080D180E280EC
:107F6000F3800E94DF152F8D38A149A15AA1DC01B1
:107F70001E962D933D934D935C9351970E94DF1570
:107F80002B8D3C8D4D8D5E8DDC0152962D933D9356
:107F90004D935C9355970E94DF15FC01C68AD78AE2
:107FA000E08EF18E0E94DF152DA93EA94FA958AD94
:107FB000DC0198962D933D934D935C939B970E9483
:107FC000DF1529A93AA94BA95CA9DC019C962D9340
:107FD0003D934D935C939F970E94DF152DA53EA581
:107FE0004FA558A9DC01D0962D933D934D935C93FA
:107FF000D3970E9467160E94E71A0E94DF150E941D
:10800000861CC1010E94E01BEF81F885118210825D
:10801000D8011D921C92E989FA891182108250E0E0
:1080200040E0B201C1010E94C62ED8014D915C9181
:10803000B301C1010E94C62EE989FA8940815181AC
:10804000B501C1010E94C62EC1010E947011F1014B
:1080500085A196A1A7A1B0A588279927AA27BE77B1
:10806000892B8A2B8B2BB1F080E496E00E94EC16D2
:1080700064E670E080E090E00E94280AC2010E945D
:10808000C813C1010E949A2964E670E080E090E084
:108090000E94280AF101EA55FF4F85899689A78930
:1080A000B08D88279927AA27BE77892B8A2B8B2BFF
:1080B000B1F084E596E00E94EC1664E670E080E0A2
:1080C00090E00E94280AC3010E94C813C1010E94C7
:1080D0006F2964E670E080E090E00E94280AF101D8
:1080E000E45CFE4F85899689A789B08D88279927FA
:1080F000AA27BE77892B8A2B8B2BB1F088E696E0D6
:108100000E94EC1664E670E080E090E00E94280A8D
:10811000C5010E94C813C1010E94442964E670E0B1
:1081200080E090E00E94280AD10158962D913C9160
:10813000599756968D919C91821793070CF4C9011B
:1081400097FF02C090E080E0F101228D338D281767
:1081500039070CF49C01D1015C968D919C9182179A
:1081600093070CF4C901F101C68CD78CC816D90647
:108170000CF46C01F101E255FF4F208131813297FF
:1081800080819181821793070CF4C90197FF02C087
:1081900090E080E0F101E055FF4F20813181281708
:1081A00039070CF49C01F101EE54FF4F808191815D
:1081B000821793070CF4C901F101EC54FF4FE080E2
:1081C000F180E816F9060CF47C01F101EC5BFE4F3E
:1081D00020813181329780819181821793070CF43D
:1081E000C90197FF02C090E080E0F101EA5BFE4F19
:1081F00020813181281739070CF49C01F101E85BDB
:10820000FE4F80819181821793070CF4C901F1011F
:10821000E65BFE4F00811181081719070CF48C01F1
:1082200086E993E00E94EC1689E296E00E94EC1643
:10823000F101E957FF4F60817181828193814AE0AA
:108240000E947C168DE494E00E94EC16C6010E9408
:10825000E7168CE296E00E94EC16F101E35EFE4F19
:10826000608171818281938124E630E040E050E0BA
:108270000E947B6064E6629FC001639F900D1124A1
:108280000E94E7168DE594E00E94EC16C7010E945B
:10829000E7168FE296E00E94EC16F101ED54FE4FD6
:1082A00060817181828193814AE00E947C168DE613
:1082B00094E00E94EC16C8010E94E7160E94DF15A8
:1082C000BC01CE0101960E94812E4D815E816981A3
:1082D0007A8187E59DE00E949907CE0101960E9470
:1082E0001B1DFD85FF2349F00E94DF1521E0DC0105
:1082F000D4962C9388248394912C8CE796E00E944A
:10830000EC16C4010E94E7168EE798E00E94EC1676
:108310000E94DF15FC0197A286A2C401C45BDF4F57
:108320000FB6F894DEBF0FBECDBFDF91CF911F9186
:108330000F91FF90EF90DF90CF90BF90AF909F9004
:108340008F907F906F905F904F903F902F90089507
:108350004F925F926F927F928F929F92AF92BF9255
:10836000CF92DF92EF92FF920F931F93CF93DF9301
:1083700000D01F92CDB7DEB70E941E1EC090AE0A7D
:10838000D090AF0AE090B00AF090B10A0E941E1E91
:108390008090B20A9090B30AA090B40AB090B50A47
:1083A0000E94DF15FC0146845784608871880E9412
:1083B000DF159A838983C301B2010E94235F2B01D9
:1083C0003C01C701B6010E94235F9B01AC01C301C0
:1083D000B2010E9411612B013C01E981FA8162899D
:1083E0007389848995890E94235F6B017C01C50193
:1083F000B4010E94235F9B01AC01C701B6010E943A
:10840000116169837A838B839C830E94D72C1F928E
:108410001F921F921F921F92912C812CB12CA12C84
:10842000C12CD12C760109811A812B813C81B301A9
:10843000A2010E9489350E94D72C1F921F921F9281
:108440001F921F9297018601B301A2010E948935F4
:108450000E94D72C1F921F921F921F921F9297016A
:10846000B701A6010E9489350FB6F894DEBF0FBE92
:10847000CDBF90E080E00F900F900F900F90DF91B4
:10848000CF911F910F91FF90EF90DF90CF90BF9011
:10849000AF909F908F907F906F905F904F900895D6
:1084A0008F929F92AF92BF92CF92DF92EF92FF9204
:1084B0000F931F93CF93DF93EB010E94D72C8A88F1
:1084C0009B88AE84BF84CA84DB84EC84FD840E81E7
:1084D0001F81288539854A815B816C817D811F924E
:1084E0001F921F92EF89EF93EE89EF930E948935D7
:1084F0000F900F900F900F900F9090E080E0DF9121
:10850000CF911F910F91FF90EF90DF90CF90BF9090
:10851000AF909F908F9008958F929F92AF92BF924D
:10852000CF92DF92EF92FF920F931F930E94D72C6E
:1085300062E070E00E940B2F892BD1F40E94D72CAF
:1085400021E02F931F921F921F921F92912C812C3A
:10855000B12CA12CC12CD12C760197018601B70139
:10856000A6010E9489350F900F900F900F900F90E9
:1085700090E080E01F910F91FF90EF90DF90CF90FF
:10858000BF90AF909F908F9008958F929F92AF92DF
:10859000BF92CF92DF92EF92FF920F931F930E94B0
:1085A000D72C61E070E00E940B2F892BD1F40E9440
:1085B000D72C1F9221E02F931F921F921F92912C74
:1085C000812CB12CA12CC12CD12C760197018601D4
:1085D000B701A6010E9489350F900F900F900F9060
:1085E0000F9090E080E01F910F91FF90EF90DF904F
:1085F000CF90BF90AF909F908F9008958F929F9251
:10860000AF92BF92CF92DF92EF92FF920F931F93A0
:108610000E94D72C70E060E00E940B2F892BD1F4D0
:108620000E94D72C1F921F9221E02F931F921F921E
:10863000912C812CB12CA12CC12CD12C760197012D
:108640008601B701A6010E9489350F900F900F9007
:108650000F900F9090E080E01F910F91FF90EF90AE
:10866000DF90CF90BF90AF909F908F9008952F9202
:108670003F924F925F926F927F928F929F92AF92B2
:10868000BF92CF92DF92EF92FF920F931F93CF93FF
:10869000DF93CDB7DEB72F970FB6F894DEBF0FBECE
:1086A000CDBF0E94D72C21E02F931F921F921F92C3
:1086B0001F92912C812CB12CA12CC12CD12C760194
:1086C00097018601B701A6010E9489350E941E1EEE
:1086D000E090A60AF090A70A0E941E1E2091B60AFA
:1086E0003091B70A3A8329830E941E1E4090960B50
:1086F0005090970B6090980B7090990B0E941E1EE3
:108700008091BE0B9091BF0BA091C00BB091C10B9B
:108710000F900F900F900F900F90E981FA811E1625
:108720001F060CF073C19C01240D351D38872F8363
:1087300046EF642E77247A94EA94EF2819F03AE011
:10874000632E712C0E94DF15DC011E966D917D91C8
:108750008D919C9151970E94235F6B017C010E9437
:108760001E1E6091AE0A7091AF0A8091B00A90917E
:10877000B10A0E94235F9B01AC01C701B6010E94B0
:1087800011616B837C838D839E830E94DF15FC01C6
:1087900062897389848995890E94235F6B017C01BA
:1087A0000E941E1E6091B20A7091B30A8091B40AB1
:1087B0009091B50A0E94235F9B01AC01C701B601ED
:1087C0000E9411611B012C010E94DF150E941E1ED8
:1087D0000E94D72C1F921F921F921F921F92912CC2
:1087E000812CB12CA12CC12CD12C760192018101BC
:1087F0004B815C816D817E810E9489350E94DF15ED
:10880000DC01D4968C9189878F819885880F991F78
:10881000EF81F885E80FF91FF887EF830F900F902D
:108820000F900F900F901F861E86C301770CAA0B26
:10883000BB0B8A879B87AC87BD870E94D72C3C01E6
:108840006A857B858C859D850E94235F6B017C01F9
:108850001F921F921F921F921F92912C812CB12C5C
:10886000A12C920181014B815C816D817E81C301CC
:108870000E9489350E94DF150F900F900F900F9086
:108880000F90DC01D4968C918111D3C00E94D72C1B
:10889000B1E0BF931F921F921F921F92C12CD12C47
:1088A000760192014B815C816D817E810E948935C8
:1088B0000E94DF150F900F900F900F900F90FC010A
:1088C00084A98111B6C087E896E00E94EC168CE975
:1088D00096E00E94EC160E94DF15DC0198966D91DF
:1088E0007D918D919C919B970E94BF1680EA96E0A6
:1088F0000E94EC160E94DF15FC0160A571A582A5FF
:1089000093A520813181428153810E944F60CA0129
:10891000B9010E94BF1684EA96E00E94EC160E94FC
:10892000DF15FC0164A575A586A597A50E94BF1655
:1089300080EA96E00E94EC160E94DF15FC0164A517
:1089400075A586A597A524813581468157810E940A
:108950004F60CA01B9010E94BF1688EA96E00E94E2
:10896000EC160E94DF15DC01D0966D917D918D9102
:108970009C91D3970E94BF1680EA96E00E94EC1665
:108980000E94DF15FC0160A971A982A993A9208525
:108990003185428553850E944F60CA01B9010E940A
:1089A000BF168EE798E00E94EC160E94DF15FC01CE
:1089B0008F81988569817A810E94CD616B01B4E1D4
:1089C000CB0ED11C0D2C000CEE08FF0860A971A97C
:1089D00082A993A920853185428553850E944F60E5
:1089E0002C153D054E055F05C4F4EE85FF853196D7
:1089F000FF87EE873397CCF00E94DF15DC01569697
:108A00001D921D921D921C92599713C018861F82A9
:108A100081E090E09A8389838BCE64EF71E080E0FF
:108A200090E00E94280A1F861E869985992309F4E2
:108A300004CF90E080E02F960FB6F894DEBF0FBE13
:108A4000CDBFDF91CF911F910F91FF90EF90DF90FD
:108A5000CF90BF90AF909F908F907F906F905F90DE
:108A60004F903F902F9008952F923F924F925F9298
:108A70006F927F928F929F92AF92BF92CF92DF922E
:108A8000EF92FF920F931F93CF93DF93CDB7DEB793
:108A900061970FB6F894DEBF0FBECDBF0E941E1EB9
:108AA0002091A20A3091A30A3E832D830E941E1EAC
:108AB0008091B20A9091B30A9A8389830E941E1E04
:108AC000C090920BD090930BE090940BF090950B8C
:108AD0000E941E1E8091BA0B9091BB0BA091BC0B03
:108AE000B091BD0BE981FA811E161F060CF05AC128
:108AF0009C012C0D3D1D3C832B83AD81BE811197C4
:108B000009F057C1E6EFFFEFFD87EC870E94DF1504
:108B1000DC011E966D917D918D919C9151970E94E3
:108B2000235F6B017C010E941E1E6091AE0A709152
:108B3000AF0A8091B00A9091B10A0E94235F9B0115
:108B4000AC01C701B6010E9411616D837E838F83E2
:108B500098870E94DF150E941E1E0E94DF15FC01EF
:108B600066897789808D918D0E94235F6B017C01DE
:108B70000E941E1E6091B60A7091B70A8091B80AD1
:108B80009091B90A0E94235F9B01AC01C701B60115
:108B90000E9411612B013C010E94D72C1F921F9251
:108BA0001F921F921F92912C812CB12CA12C73012A
:108BB000620100E010E098014D815E816F8178854F
:108BC0000E9489350E94DF15DC01D4968C918B8739
:108BD0008B819C81880F991FEB81FC81E80FF91F25
:108BE000FA87E9870F900F900F900F900F90312C1C
:108BF000212C8C859D85092E000CAA0BBB0B8C8724
:108C00009D87AE87BF870E94D72C998B888B6C85F8
:108C10007D858E859F850E94235F8B019C011F921D
:108C20001F921F921F921F92912C812CB12CA12C6C
:108C3000730162014D815E816F8178858889998990
:108C40000E9489350E94DF150F900F900F900F90B2
:108C50000F90DC01D4968C918111BCC00E94D72C5E
:108C60001F92B1E0BF931F921F921F9200E010E08D
:108C700098014D815E816F8178850E9489350E94BF
:108C8000DF150F900F900F900F900F90FC0184A9AB
:108C90008111A0C087E896E00E94EC168CE996E06E
:108CA0000E94EC160E94DF15FC0160A571A582A54B
:108CB00093A520813181428153810E944F60CA0176
:108CC000B9010E94BF1684EA96E00E94EC160E9449
:108CD000DF15FC0164A575A586A597A524813581BE
:108CE000468157810E944F60CA01B9010E94BF1698
:108CF00088EA96E00E94EC160E94DF15FC0160A94C
:108D000071A982A993A920853185428553850E9446
:108D10004F60CA01B9010E94BF168CEA96E00E941A
:108D2000EC168B819C810E94E7168CEA96E00E94EB
:108D3000EC1689819A810E94E7168EE798E00E94DE
:108D4000EC160E94DF15FC0189859A8569817A817C
:108D50000E94CD616B0124E1C20ED11C0D2C000CD0
:108D6000EE08FF0864A575A586A597A52481358121
:108D7000468157810E944F60C216D306E406F5066D
:108D8000ECF03FEF231A330A83E028163104F4F0A5
:108D90000E94DF15DC0152961D921D921D921C92BD
:108DA000559718C01C821B8281E090E09A838983CA
:108DB000A4CE2AE030E03D872C87A8CE64EF71E096
:108DC00080E090E00E94280A312C212C9B85992379
:108DD00009F419CF90E080E061960FB6F894DEBFF9
:108DE0000FBECDBFDF91CF911F910F91FF90EF90FC
:108DF000DF90CF90BF90AF909F908F907F906F90BB
:108E00005F904F903F902F9008952F923F924F92F6
:108E10005F926F927F928F929F92AF92BF92CF920A
:108E2000DF92EF92FF920F931F93CF93DF93CDB713
:108E3000DEB72F970FB6F894DEBF0FBECDBF0E94EE
:108E40001E1EE0909E0AF0909F0A0E941E1E209116
:108E5000AE0A3091AF0A3A8329830E941E1E4090C9
:108E60008E0B50908F0B6090900B7090910B0E9426
:108E70001E1E8091B60B9091B70BA091B80BB091CC
:108E8000B90BE981FA811E161F060CF072C19C0114
:108E9000240D351D38872F8346EF642E77247A946E
:108EA000EA94EF2819F03AE0632E712C0E94DF1546
:108EB0000E941E1E0E94DF15DC0152966D917D916D
:108EC0008D919C9155970E94235F6B017C010E94BC
:108ED0001E1E6091B20A7091B30A8091B40A9091FB
:108EE000B50A0E94235F9B01AC01C701B6010E9435
:108EF00011616B837C838D839E830E94DF15FC014F
:108F000066897789808D918D0E94235F6B017C013A
:108F10000E941E1E6091B60A7091B70A8091B80A2D
:108F20009091B90A0E94235F9B01AC01C701B60171
:108F30000E9411611B012C010E94D72C1F921F92CD
:108F40001F921F921F92912C812CB12CA12C720187
:108F500061010B811C812D813E8140E050E0BA010E
:108F60000E9489350E94DF15DC01D4968C91898797
:108F70008F819885880F991FEF81F885E80FF91F79
:108F8000F887EF830F900F900F900F900F901F8630
:108F90001E86C301770CAA0BBB0B8A879B87AC8705
:108FA000BD870E94D72C3C016A857B858C859D8579
:108FB0000E94235FAB01BC011F921F921F921F9260
:108FC0001F92912C812CB12CA12C720161010B817B
:108FD0001C812D813E81C3010E9489350E94DF15CD
:108FE0000F900F900F900F900F90DC01D4968C9102
:108FF0008111D2C00E94D72C1F921F92B1E0BF9363
:109000001F921F920B811C812D813E8140E050E018
:10901000BA010E9489350E94DF150F900F900F90C2
:109020000F900F90FC0184A98111B6C087E896E0EB
:109030000E94EC168CE996E00E94EC160E94DF1567
:10904000DC0198966D917D918D919C919B970E94EA
:10905000BF1680EA96E00E94EC160E94DF15FC0124
:1090600060A571A582A593A520813181428153819C
:109070000E944F60CA01B9010E94BF1684EA96E0BF
:109080000E94EC160E94DF15FC0164A575A586A55B
:1090900097A50E94BF1680EA96E00E94EC160E94F7
:1090A000DF15FC0164A575A586A597A524813581EA
:1090B000468157810E944F60CA01B9010E94BF16C4
:1090C00088EA96E00E94EC160E94DF15DC01D0963B
:1090D0006D917D918D919C91D3970E94BF1680EAEE
:1090E00096E00E94EC160E94DF15FC0160A971A9B0
:1090F00082A993A920853185428553850E944F60BE
:10910000CA01B9010E94BF168EE798E00E94EC16D2
:109110000E94DF15FC018F81988569817A810E9408
:10912000CD616B01B4E1CB0ED11C0D2C000CEE080F
:10913000FF0860A571A582A593A520813181428198
:1091400053810E944F602C153D054E055F05C4F408
:10915000EE85FF853196FF87EE873397CCF00E942E
:10916000DF15DC011E961D921D921D921C925197D7
:1091700013C018861F8281E090E09A8389838CCE89
:1091800064EF71E080E090E00E94280A1F861E864E
:109190009985992309F405CF90E080E02F960FB6CA
:1091A000F894DEBF0FBECDBFDF91CF911F910F911D
:1091B000FF90EF90DF90CF90BF90AF909F908F90F7
:1091C0007F906F905F904F903F902F9008951F92E7
:1091D0000F920FB60F9211240BB60F922F933F935D
:1091E0004F935F936F937F938F939F93AF93BF93AF
:1091F000EF93FF9387E59DE00E940C08FF91EF91AC
:10920000BF91AF919F918F917F916F915F914F919E
:109210003F912F910F900BBE0F900FBE0F901F909C
:1092200018951F920F920FB60F9211240BB60F9242
:109230002F938F939F93EF93FF93E091670DF0919E
:10924000680D8081E0916D0DF0916E0D82FD1DC065
:1092500090818091700D8F5F8F732091710D8217B7
:1092600041F0E091700DF0E0E95AF24F958F809354
:10927000700DFF91EF919F918F912F910F900BBEE9
:109280000F900FBE0F901F9018958081F2CF1F9204
:109290000F920FB60F9211242F933F938F939F93AA
:1092A000AF93BF938091C0089091C108A091C2086C
:1092B000B091C3083091BF0823E0230F2D3758F534
:1092C0000196A11DB11D2093BF088093C008909303
:1092D000C108A093C208B093C3088091C4089091BC
:1092E000C508A091C608B091C7080196A11DB11D7F
:1092F0008093C4089093C508A093C608B093C7088C
:10930000BF91AF919F918F913F912F910F900FBE81
:109310000F901F90189526E8230F0296A11DB11DEE
:10932000D2CF1F920F920FB60F9211240BB60F924D
:109330002F933F934F935F936F937F938F939F935D
:10934000AF93BF93EF93FF9348E251E064E271E083
:1093500090E080E00E94680BFF91EF91BF91AF9188
:109360009F918F917F916F915F914F913F912F913D
:109370000F900BBE0F900FBE0F901F9018951F926D
:109380000F920FB60F9211240BB60F922F933F93AB
:109390004F935F936F937F938F939F93AF93BF93FD
:1093A000EF93FF9348EA50E064EA70E083E090E0D6
:1093B0000E94680BFF91EF91BF91AF919F918F91A8
:1093C0007F916F915F914F913F912F910F900BBEC5
:1093D0000F900FBE0F901F9018951F920F920FB60F
:1093E0000F9211240BB60F922F933F934F935F93DD
:1093F0006F937F938F939F93AF93BF93EF93FF935D
:1094000048E950E064E970E082E090E00E94680B77
:10941000FF91EF91BF91AF919F918F917F916F914C
:109420005F914F913F912F910F900BBE0F900FBE08
:109430000F901F9018951F920F920FB60F92112444
:109440000BB60F922F933F934F935F936F937F933E
:109450008F939F93AF93BF93EF93FF9348E850E0B0
:1094600064E870E081E090E00E94680BFF91EF916A
:10947000BF91AF919F918F917F916F915F914F912C
:109480003F912F910F900BBE0F900FBE0F901F902A
:1094900018951F920F920FB60F9211240BB60F92D0
:1094A0002F933F934F935F936F937F938F939F93EC
:1094B000AF93BF93EF93FF93E091C908F091CA086F
:1094C0001995FF91EF91BF91AF919F918F917F91EE
:1094D0006F915F914F913F912F910F900BBE0F9025
:1094E0000FBE0F901F901895FF920F931F93CF936D
:1094F000DF93EC01F62E8C01065F1F4F1B861A8648
:109500001D861C861F861E86C8010E949A2AF88620
:10951000198670E060E0C801DF91CF911F910F9133
:10952000FF900C94752A10925A0D1092590D88EEE6
:1095300093E0A0E0B0E080935B0D90935C0DA0936E
:109540005D0DB0935E0D80E893E09093580D80938D
:10955000570D85EC90E09093640D8093630D84EC3F
:1095600090E09093660D8093650D80EC90E0909371
:10957000680D8093670D81EC90E090936A0D809365
:10958000690D82EC90E090936C0D80936B0D86ECEE
:1095900090E090936E0D80936D0D1092700D10926F
:1095A000710D1092720D1092730D68E183E594E1D4
:1095B0009BDF6CE183E694E197DF67E183E794E169
:1095C00093DF6DE183E894E18FDF68E183E194E16B
:1095D0008BDF6CE183E294E187DF67E183E394E171
:1095E00083DF6DE183E494E17FDFE5E8FEE02FEFC8
:1095F00048EB5BE08091840E803308F083C191E0FA
:10960000980F9093840E808390E0DC01AA0FBB1F1B
:10961000A80FB91FAC50B24F12965C934E9311979E
:1096200033968EE0E139F80729F768E183ED93E19D
:109630005BDF6CE183EE93E157DF67E183EF93E15A
:1096400053DF6DE183E094E14FDF68E183E993E16B
:109650004BDF6CE183EA93E147DF67E183EB93E162
:1096600043DF6DE183EC93E13FDF68E183E593E164
:109670003BDF6CE183E693E137DF67E183E793E16A
:1096800033DF6DE183E893E12FDF68E183E193E16C
:109690002BDF6CE183E293E127DF67E183E393E172
:1096A00023DF6DE183E493E11FDF68E183ED92E165
:1096B0001BDF6CE183EE92E117DF67E183EF92E15C
:1096C00013DF6DE183E093E10FDF68E183E992E16D
:1096D0000BDF6CE183EA92E107DF67E183EB92E164
:1096E00003DF6DE183EC92E1FFDE68E183E592E167
:1096F000FBDE6CE183E692E1F7DE67E183E792E16E
:10970000F3DE6DE183E892E1EFDE82E090E00E941B
:10971000A45922E933E0FC01318320839093920E17
:109720008093910E68E183E192E1DEDE6CE183E2F9
:1097300092E1DADE67E183E392E1D6DE6DE183E474
:1097400092E1D2DE68E183ED91E1CEDE6CE183EE61
:1097500091E1CADE67E183EF91E1C6DE6DE183E06E
:1097600092E1C2DE68E183E991E1BEDE6CE183EA69
:1097700091E1BADE67E183EB91E1B6DE6DE183EC66
:1097800091E1B2DE68E183E591E1AEDE6CE183E672
:1097900091E1AADE67E183E791E1A6DE6DE183E86E
:1097A00091E1A2DE68E183E191E19EDE6CE183E27A
:1097B00091E19ADE67E183E391E196DE6DE183E476
:1097C00091E192DE68E183ED90E18EDE6CE183EE63
:1097D00090E18ADE67E183EF90E186DE6DE183E070
:1097E00091E182DE68E183E990E17EDE6CE183EA6B
:1097F00090E17ADE67E183EB90E176DE6DE183EC68
:1098000090E172DE68E183E590E16EDE6CE183E673
:1098100090E16ADE67E183E790E166DE6DE183E86F
:1098200090E162DE68E183E190E15EDE6CE183E27B
:1098300090E15ADE67E183E390E156DE6DE183E477
:1098400090E152DE68E183ED9FE04EDE6CE183EE55
:109850009FE04ADE67E183EF9FE046DE6DE183E053
:1098600090E142DE68E183E99FE03EDE6CE183EA5D
:109870009FE03ADE67E183EB9FE036DE6DE183EC4B
:109880009FE032DE68E183E59FE02EDE6CE183E657
:109890009FE02ADE67E183E79FE026DE6DE183E853
:1098A0009FE022DE68E183E19FE01EDE6CE183E25F
:1098B0009FE01ADE67E183E39FE016DE6DE183E45B
:1098C0009FE012DE68E183ED9EE00EDE6CE183EE48
:1098D0009EE00ADE67E183EF9EE006DE6DE183E055
:1098E0009FE002DE68E183E99EE0FEDD6CE183EA51
:1098F0009EE0FADD67E183EB9EE0F6DD6DE183EC4F
:109900009EE0F2CD20838CCE789484B5826084BDB5
:1099100084B5816084BD85B5826085BD85B5816073
:1099200085BD80916E00816080936E0010928100F1
:1099300080918100826080938100809181008160AC
:10994000809381008091800081608093800080916D
:10995000B10084608093B1008091B00081608093F9
:10996000B00080919100826080939100809191007D
:10997000816080939100809190008160809390003D
:109980008091A10082608093A1008091A1008160FC
:109990008093A1008091A00081608093A0008091BD
:1099A0002101826080932101809121018160809357
:1099B00021018091200181608093200180917A00B3
:1099C000846080937A0080917A00826080937A002C
:1099D00080917A00816080937A0080917A0080681B
:1099E00080937A001092C100E091670DF091680DAC
:1099F00082E08083E091630DF091640D1082E0912C
:109A0000650DF091660D10E1108310926F0DE091DD
:109A10006B0DF0916C0D86E08083E091690DF09103
:109A20006A0D808180618083E091690DF0916A0DFB
:109A3000808188608083E091690DF0916A0D80815A
:109A400080688083E091690DF0916A0D80818F7D3F
:109A5000808364E670E080E090E00E94280A8DE652
:109A600092E00E94EC168BE692E00E94EC1680EBEE
:109A700096E00E94EC1688E692E00E94EC168DE6D5
:109A800092E00E94EC168BE692E00E94EC168AECC3
:109A900096E00E94EC1688E692E00E94EC1661E0E7
:109AA00089E10E94890961E08BE10E94890961E0F6
:109AB0008AE10E94890962E085E40E94890962E0E6
:109AC00084E40E94890961E089E10E945C0960E008
:109AD0008BE10E945C0960E08AE10E945C0961E020
:109AE0008FE10E94890961E081E20E94890961E0B9
:109AF00080E20E94890962E083E40E94890962E0B1
:109B000082E40E94890961E08FE10E945C0960E0C3
:109B100081E20E945C0960E080E20E945C0961E0F1
:109B200082E20E94890961E084E20E94890961E081
:109B300083E20E94890962E081E40E94890962E06F
:109B400080E40E94890961E082E20E945C0960E091
:109B500084E20E945C0960E083E20E945C0961E0AB
:109B60008EE00E94890961E08EE10E94890961E02E
:109B70008FE00E94890961E08EE00E945C0960E04C
:109B80008EE10E945C0960E08FE00E945C0961E068
:109B900088E20E94890961E089E20E94890961E006
:109BA00085E20E94890960E088E20E945C0960E029
:109BB00089E20E945C0960E085E20E945C0961E044
:109BC0008DE00E94890961E089E00E94890961E0D5
:109BD00088E00E94890961E087E00E94890961E0CC
:109BE0008AE00E94890961E08CE00E94890960E0B6
:109BF0008DE00E945C0960E089E00E945C0960E001
:109C000088E00E945C0960E087E00E945C0960E0F7
:109C10008AE00E945C0960E08CE00E945C0962E0DE
:109C20008FE30E94890962E08BE30E94890961E069
:109C300084E00E94890961E085E00E94890961E071
:109C400086E00E94890961E08BE00E94890960E05A
:109C500084E00E945C0960E085E00E945C0960E0AD
:109C600086E00E945C0960E08BE00E945C098DE662
:109C700092E00E94EC168BE692E00E94EC168BEECE
:109C800096E00E94EC1688E692E00E94EC160E9494
:109C90001E1E0E94961A8DE692E00E94EC168BE63C
:109CA00092E00E94EC168BEF96E00E94EC1688E69C
:109CB00092E00E94EC168DE692E00E94EC168BE694
:109CC00092E00E94EC168CE097E00E94EC1688E689
:109CD00092E00E94EC160E94D72CEC0140960E9464
:109CE000C813CE018A559F4F0E94C813CE01845CD1
:109CF0009E4F0E94C8138DE692E00E94EC168BE600
:109D000092E00E94EC1681E297E00E94EC1688E651
:109D100092E00E94EC160E94D72CEC010E949A2936
:109D2000CE010E946F29CE010E9444298DE692E067
:109D30000E94EC168BE692E00E94EC1689E397E015
:109D40000E94EC1688E692E00E94EC160E94D72C46
:109D50000E94FD278DE692E00E94EC168BE692E0D1
:109D60000E94EC1680E597E00E94EC1688E692E0EF
:109D70000E94EC1661E089E10E945C0961E08EE0DE
:109D80000E945C0961E08FE10E945C0961E082E26F
:109D90000E945C098DE692E00E94EC168BE692E050
:109DA0000E94EC1686E697E00E94EC1688E692E0A8
:109DB0000E94EC160E940C1F0E94DC1E0E94590A91
:109DC0000E94590A6093CB087093CC088093CD0809
:109DD0009093CE088DE692E00E94EC168BE692E01E
:109DE0000E94EC1686E797E00E94EC1688E692E067
:109DF0000E94EC1680EF9CE29093CA088093C908F9
:109E0000C1E0C0936F001093810010928000C09356
:109E1000C80880E092E0909387008093860081E1FB
:109E2000809381001092810010928500109284002E
:109E30008091C8088061809381000E94590A6093D4
:109E4000CE097093CF098093D0099093D1098DE604
:109E500092E00E94EC168BE692E00E94EC1686E8F7
:109E600097E00E94EC1688E692E00E94EC160E94B1
:109E70001E1E8091DA099091DB09A091DC09B09156
:109E8000DD090197A105B10559F50E941E1E8091BB
:109E9000220A9091230AA091240AB091250A0197E1
:109EA000A105B105E9F48BE997E00E94EC160E9448
:109EB000D72CCF931F921F921F921F92912C812C0F
:109EC000B12CA12CC12CD12C760197018601B701B0
:109ED000A6010E9489350F900F900F900F900F9060
:109EE0000E941E1E8091DA099091DB09A091DC0985
:109EF000B091DD090197A105B10561F50E941E1E13
:109F000080911E0A90911F0AA091200AB091210A07
:109F10000197A105B105F1F483EB97E00E94EC16DF
:109F20000E94D72C1F9221E02F931F921F921F9205
:109F3000912C812CB12CA12CC12CD12C7601970114
:109F40008601B701A6010E9489350F900F900F90EE
:109F50000F900F900E941E1E8091DA099091DB09EC
:109F6000A091DC09B091DD090197A105B10561F56A
:109F70000E941E1E80911A0A90911B0AA0911C0A31
:109F8000B0911D0A0197A105B105F1F48BEC97E0A2
:109F90000E94EC160E94D72C1F921F9221E02F9353
:109FA0001F921F92912C812CB12CA12CC12CD12C51
:109FB000760197018601B701A6010E9489350F90AD
:109FC0000F900F900F900F9086E792E00E94EC1692
:109FD00084E792E00E94EC1683EE97E00E94EC1674
:109FE00081E792E00E94EC16EEE0CE2ED12CFCEE42
:109FF0002F2EF2E03F2E0E94590AAB01BC01809146
:10A00000CB089091CC08A091CD08B091CE0848170C
:10A0100059076A077B0708F060C04093CB0850934C
:10A02000CC086093CD087093CE0887E59DE00E9430
:10A03000F707892B09F433C30E94590A6093CE09AC
:10A040007093CF098093D0099093D10987E59DE063
:10A050000E94D5078093C409982F9F7D953409F4F9
:10A0600068C02091C2093091C309F901E25AF64F44
:10A0700080832F5F3F4F3093C3092093C2098091A3
:10A08000C2099091C3098336910564F02AE02093B8
:10A09000C409FC01E25AF64F208301969093C3094C
:10A0A0008093C2092091C2093091C3098091C409EB
:10A0B0008A3021F0243631050CF4F1C2C901019730
:10A0C000A9EFB8E0EEE5F9E0AF014E555940481769
:10A0D0005907B4F541914D93F7CF481B590B6A0BC3
:10A0E0007B0B483E53406105710508F49ECF8851B3
:10A0F0009C4FAF4FBF4F8093CB089093CC08A09359
:10A10000CD08B093CE080E940C1FEC010E94071AE4
:10A11000CE010C960E94071ACE0148960E94071A9B
:10A12000CE0184960E94071ACE01C0960E94071A9B
:10A130007CCF0E94DF1521E0DC01D4962C939FCFC9
:10A140008750974FFC011082223031050CF4A3C2D6
:10A1500088E693E00E94EC1682EA96E00E94EC16F4
:10A160008CEF97E00E94EC1689EF98E00E94EC16C5
:10A170008CEF97E00E94EC168EE798E00E94EC16B8
:10A180008AE390E00E94A459EC011A821B821C828F
:10A190001D821E821F82188619861A861B861C86BF
:10A1A0001D861E861F86188A198A1A8A1B8A1C8A8F
:10A1B0001D8A1E8A1F8A188E198E1A8E1B8E1C8E5F
:10A1C0001D8E1E8E1F8E18A219A21AA21BA21CA2DF
:10A1D0001DA21EA21FA218A619A61AA61BA61CA67F
:10A1E0001DA61EA61FA618AA19AA1AAA1BAA1CAA4F
:10A1F0001DAA1EAA1FAA18AE19AE63E272E089EF6B
:10A2000098E00E94CC5A8C01DC018C9186548230FB
:10A2100008F0EEC16EEF77E0C8010E94E562892B7D
:10A2200009F49EC161E078E0C8010E94E562892BD3
:10A2300009F496C165E078E0C8010E94E562892BC7
:10A2400009F491C168E078E0C8010E94E562892BB9
:10A2500009F489C16CE078E0C8010E94E562892BAD
:10A2600009F484C160E178E0C8010E94E562892BAD
:10A2700009F47FC164E178E0C8010E94E562892B9E
:10A2800009F477C167E178E0C8010E94E562892B93
:10A2900009F472C16BE178E0C8010E94E562892B84
:10A2A00009F46DC16FE178E0C8010E94E562892B75
:10A2B00009F468C163E278E0C8010E94E562892B75
:10A2C00009F463C167E278E0C8010E94E562892B66
:10A2D00009F45EC16BE278E0C8010E94E562892B57
:10A2E00009F459C16FE278E0C8010E94E562892B48
:10A2F00009F454C163E378E0C8010E94E562892B48
:10A3000009F44FC167E378E0C8010E94E562892B38
:10A3100009F44AC16BE378E0C8010E94E562892B29
:10A3200009F445C16FE378E0C8010E94E562892B1A
:10A3300009F440C163E478E0C8010E94E562892B1A
:10A3400009F43BC167E478E0C8010E94E562892B0B
:10A3500009F436C16BE478E0C8010E94E562892BFC
:10A3600009F431C16FE478E0C8010E94E562892BED
:10A3700009F42CC163E578E0C8010E94E562892BED
:10A3800009F427C167E578E0C8010E94E562892BDE
:10A3900009F422C16BE578E0C8010E94E562892BCF
:10A3A00009F41DC16FE578E0C8010E94E562892BC0
:10A3B00009F418C163E678E0C8010E94E562892BC0
:10A3C00009F013C188EB90E09093010280930002A2
:10A3D0000115110509F412C1F8018081883541F495
:10A3E000C80101960E94C95A6A837B838C839D832E
:10A3F000D8018C91893541F4C80101960E94C95A4F
:10A400006E837F8388879987F80180818A3541F43C
:10A41000C80101960E94C95A6A877B878C879D87ED
:10A42000D8018C91813451F4C80101960E94C95A17
:10A430000E9479616E877F87888B998BF801808174
:10A44000823451F4C80101960E94C95A0E94796170
:10A450006A8B7B8B8C8B9D8BD8018C91833451F4D0
:10A46000C80101960E94C95A0E9479616E8B7F8B48
:10A47000888F998FF8018081833541F4C801019656
:10A480000E94C95A6A8F7B8F8C8F9D8FD8018C91C7
:10A49000803551F4C80101960E94C95A0E94796121
:10A4A0006E8F7F8F88A399A3F8018081863551F440
:10A4B000C80101960E94C95A0E9479616AA37BA3D0
:10A4C0008CA39DA3D8018C91873551F4C8010196C6
:10A4D0000E94C95A0E9479616EA37FA388A799A799
:10A4E000F8018081853451F4C80101960E94C95A4F
:10A4F0000E9479616AA77BA78CA79DA7D8018C9140
:10A50000843551F4C80101960E94C95A0E947961AC
:10A510006EA77FA788AB99ABF80180818D3451F489
:10A52000C80101960E94C95A0E9479616AAB7BAB4F
:10A530008CAB9DABD8018C91813551F4C80101964B
:10A540000E94C95A0E9479616EAB7FAB88AF99AF08
:10A5500067E678E090E080E00E94CC5A8C0138CF2A
:10A5600090E080E031CF81E090E02ECF8CE190E070
:10A570002BCF8DE690E028CF8FE690E025CF80E7C7
:10A5800090E022CF81E790E01FCF82E790E01CCFE0
:10A5900083E790E019CF84E790E016CF88E790E05A
:10A5A00013CF89E790E010CF8AE790E00DCF83E8E2
:10A5B00090E00ACF84E890E007CF8DE890E004CFE8
:10A5C0008EE890E001CF8FE890E0FECE80E990E049
:10A5D000FBCE81EA90E0F8CE85EB90E0F5CE86EBFD
:10A5E00090E0F2CE87EB90E0EFCE8FEF9FEFECCED6
:10A5F0008FEF9FEF90930102809300020E94DF157E
:10A60000FC0114A90E941E1E4090E6095090E70923
:10A610006090E8097090E9098EA89FA8A8ACB9AC31
:10A620000E94DF15DC0192968D929D92AD92BC92B4
:10A63000959780910002909101028230910508F473
:10A64000C0C49C012F5631092530310508F4B9C426
:10A65000992493948437910509F0912C112309F4DE
:10A66000B4C48D36910509F4B0C49C012857310952
:10A670002330310508F4A9C4855B9109039708F4D8
:10A68000A4C484E693E00E94EC160E94DF150E94A9
:10A690007D19CE01F5D61092C3091092C20980919E
:10A6A000C5098111A4C00E94DF15FC0184A988237B
:10A6B00009F49DC00E94D72CEC01FC01E45AFC4F28
:10A6C000108240960E945911CE018A559F4F0E94D8
:10A6D0005911CE01845C9E4F0E9459110E946B1546
:10A6E0008C010F5F1F4FC1E0D0E0D8018D918D012B
:10A6F0008823D9F086E993E00E94EC1681E898E07F
:10A700000E94EC16CE010E94E7168EE798E00E94A8
:10A71000EC1660E08C2F0E945C0970E060E0CE01D6
:10A720000E94A519F80131971082F80187A98823A2
:10A73000F9F086E993E00E94EC1688E998E00E941F
:10A74000EC16CE010E94E7168EE798E00E94EC1608
:10A7500061E08C2F0E94890960E08C2F0E945C09C7
:10A7600061E070E0CE010E94A519D801D7961C9235
:10A770002196C533D10509F0B8CF0E94111520915B
:10A78000850E30E0C901880F991F820F931FFC01CD
:10A79000EC50F24F80818F7B80832091880E30E0D7
:10A7A000C901880F991F820F931FFC01EC50F24FD3
:10A7B00080818F7B808320918B0E30E0C901880FD0
:10A7C000991F820F931FFC01EC50F24F80818F7B09
:10A7D000808320918E0E30E0C901880F991F820F6F
:10A7E000931FFC01EC50F24F80818F7B80830E948D
:10A7F000DF15FC0184A98093C5090E941E1E2091CB
:10A80000C8093091C909DC0112968D919C912817D5
:10A81000390791F10E941E1EFC0182819381909361
:10A82000C9098093C8090E941E1E2091C609309153
:10A83000C709DC0114968D919C9128173907A1F066
:10A840000E941E1EFC01848195819093C70980930C
:10A85000C6090E94D72CEC010E949A29CE010E94C1
:10A860006F29CE010E9444290E94D72C0E94FD2707
:10A870000E940C1F0E94DC1E0E94590A0091CE0902
:10A880001091CF092091D0093091D109601771073B
:10A890008207930708F0FEC20E94590A6093CE090E
:10A8A0007093CF098093D0099093D1090E949D089D
:10A8B000A2CB209781F48CE593E00E94EC160E94D5
:10A8C000DF150E947D190E94DF15DC019796DC924E
:10A8D000CE929697DECEE0900002F0900102BFEF9C
:10A8E000EB16FB0671F48CE593E00E94EC160E94D7
:10A8F000DF150E947D190E94DF15FC01D7A2C6A2B8
:10A90000C8CEE114F10409F083C08091F70890915A
:10A91000F808892B61F482E090E016D526E433E054
:10A92000DC012D933C939093F8088093F7080091F5
:10A93000F7081091F808B1E7EB16F10409F09EC092
:10A940008091ED089091EE08892B61F482E090E00F
:10A95000FBD424E133E0FC01318320839093EE08A3
:10A960008093ED080091ED081091EE08F9E7EF16DD
:10A97000F10409F09EC08091E3089091E408892BCE
:10A9800061F482E090E0E0D4E2EEF2E0DC01ED93ED
:10A99000FC939093E4088093E3080091E3081091FE
:10A9A000E408F0E9EF16F10409F09EC08091D9089F
:10A9B0009091DA08892B61F482E090E0C5D4E0EB55
:10A9C000F2E0DC01ED93FC939093DA088093D908D0
:10A9D0000091D9081091DA08F8EBEF16F10409F0AC
:10A9E0009EC08091CF089091D008892B61F482E0BD
:10A9F00090E0AAD4EEE7F2E0DC01ED93FC939093B3
:10AA0000D0088093CF080091CF081091D00887C05C
:10AA1000BCE1EB16F104B9F48091F5089091F608C9
:10AA2000892B61F482E090E08FD42CE333E0FC01C9
:10AA3000318320839093F6088093F5080091F50800
:10AA40001091F60878CFFDE6EF16F10409F083C007
:10AA50008091F3089091F408892B61F482E090E0F2
:10AA600073D422E333E0DC012D933C939093F408FC
:10AA70008093F3080091F3081091F408F2E7EF16C1
:10AA8000F10409F083C08091EB089091EC08892BC8
:10AA900061F482E090E058D42AE033E0DC012D93A9
:10AAA0003C939093EC088093EB080091EB08109195
:10AAB000EC08FAE7EF16F10409F083C08091E10891
:10AAC0009091E208892B61F482E090E03DD4E8EDBA
:10AAD000F2E0DC01ED93FC939093E2088093E108AF
:10AAE0000091E1081091E208F1EAEF16F10409F093
:10AAF00083C08091D7089091D808892B61F482E0B7
:10AB000090E022D4E6EAF2E0DC01ED93FC9390932E
:10AB1000D8088093D7080091D7081091D80801155C
:10AB2000110509F045C18CE593E00E94EC160E94E6
:10AB3000DF150E947D190E94DF15DC019796DC92DB
:10AB4000CE9296978BE698E00E946F168EE798E07B
:10AB50000E946F169ECDBFE6EB16F10409F068C0A7
:10AB60008091F1089091F208892B61F482E090E0E5
:10AB7000EBD328E233E0FC01318320839093F20889
:10AB80008093F1080091F1081091F208B3E7EB16F9
:10AB9000F10409F0BBC08091E9089091EA08892B83
:10ABA00061F482E090E0D0D320E033E0FC01318317
:10ABB00020839093EA088093E9080091E9081091B6
:10ABC000EA08FDE8EF16F10409F0BBC08091DF0848
:10ABD0009091E008892B61F482E090E0B5D3EEEC2F
:10ABE000F2E0DC01ED93FC939093E0088093DF08A2
:10ABF0000091DF081091E008F5EBEF16F10409F081
:10AC0000BBC08091D5089091D608892B61F482E071
:10AC100090E09AD3ECE9F2E0DC01ED93FC939093A1
:10AC2000D6088093D5080091D5081091D60877CF23
:10AC3000F0E7EF16F10409F066C08091EF089091FB
:10AC4000F008892B61F482E090E07ED32EE133E0BE
:10AC5000DC012D933C939093F0088093EF080091D2
:10AC6000EF081091F008B8E7EB16F10409F07ECE7A
:10AC70008091E5089091E608892B51F482E090E0FC
:10AC800063D3FC01318220829093E6088093E5082B
:10AC90000091E5081091E608FFE8EF16F10409F0CD
:10ACA00080CE8091DB089091DC08892B61F482E0F2
:10ACB00090E04AD3EAEBF2E0DC01ED93FC93909351
:10ACC000DC088093DB080091DB081091DC08F7EBCF
:10ACD000EF16F10409F080CE8091D1089091D2084E
:10ACE000892B61F482E090E02FD3E8E8F2E0DC0108
:10ACF000ED93FC939093D2088093D1080091D108F2
:10AD00001091D2080CCF10E000E015CEF4E7EF165A
:10AD1000F10409F0A8CF8091E7089091E808892B09
:10AD200061F482E090E010D326EF32E0DC012D9355
:10AD30003C939093E8088093E7080091E70810910E
:10AD4000E808FEE8EF16F10409F0A6CF8091DD08CF
:10AD50009091DE08892B61F482E090E0F5D2E4EC7A
:10AD6000F2E0DC01ED93FC939093DE088093DD0824
:10AD70000091DD081091DE08F6EBEF16F10409F002
:10AD8000A6CF8091D3089091D408892B61F482E0FA
:10AD900090E0DAD2E2E9F2E0DC01ED93FC939093EB
:10ADA000D4088093D3080091D3081091D408B7CE6B
:10ADB00088E593E00E94EC160E94DF150E947D1941
:10ADC0000E94DF15FC0117A216A2F12CE12C2FEF37
:10ADD000E21AF20A31E0E316F10441F084E593E06F
:10ADE0000E94EC160E94DF150E947D19D801ED919A
:10ADF000FC910480F581E02DBE01C80119950E94E7
:10AE0000DF15FC01A6A0B7A00E94DF15DC01D496D7
:10AE10008C9181110AC0E414F5043CF4A114B1042E
:10AE200021F0F2E0AF16B10491F687E59DE00E94B3
:10AE3000F707181619062CF487E59DE00E94D50740
:10AE4000F4CFAB2809F4ABC0992099F00E941E1EE4
:10AE50008091E2099091E309A091E409B091E5099C
:10AE60000197A105B10529F40E94DF1521E0FC013D
:10AE700024AB8CE493E00E94EC168CE296E00E94F6
:10AE8000EC160E94DF15DC0196968D919C910E9434
:10AE9000E71689C0601B710B820B930B69387341F5
:10AEA0008105910508F402CD0E94DF15DC01D496DE
:10AEB0008C91882309F470C084E793E00E94EC161B
:10AEC0000E94DF150E947D190E94D72CEC010E9480
:10AED000DF15FE01EE59FF4F408151816281738180
:10AEE000FC0146875787608B718B0E94DF15FE013E
:10AEF000E850FF4F4081518162817381DC0152969D
:10AF00004D935D936D937C9355970E94DF15C257C7
:10AF1000DE4F488159816A817B81FC01468B578BCA
:10AF2000608F718F0E94DF150E94861C0E94D72CB3
:10AF30000E94E01B0E94DF150E9426160E94DF156A
:10AF40000E94BF1A0E941E1E8091DA099091DB09AF
:10AF5000A091DC09B091DD090197A105B10541F08F
:10AF60008CE693E00E94EC160E94DF150E947D198A
:10AF70008091CA099091CB09A091CC09B091CD09DB
:10AF80000196A11DB11D8093CA099093CB09A0938E
:10AF9000CC09B093CD0980CC80E793E08FCF80E5DA
:10AFA00093E00E94EC160E94DF150E947D190E941A
:10AFB000DF15DC0192961D921D921D921C929597B1
:10AFC00068CB9924939411115CCB0E941E1E809132
:10AFD000DA099091DB09A091DC09B091DD090197B4
:10AFE000A105B10509F465CC992009F462CC80E68D
:10AFF00093E00E94EC160E94DF150E947D190E94CA
:10B00000DF152FE030E0FC0137A326A342CB8DEC07
:10B010009EE00E941B1D8DEB9EE00E941B1D8DEA91
:10B020009EE00E941B1D8DE99EE00E941B1D8DE08D
:10B030009FE00E941B1D8DEF9EE00E941B1D8DEE68
:10B040009EE00E941B1D8DED9EE00E941B1D8DE465
:10B050009FE00E941B1D8DE39FE00E941B1D8DE25F
:10B060009FE00E941B1D8DE19FE00E941B1D8DE84B
:10B070009FE00E941B1D8DE79FE00E941B1D8DE637
:10B080009FE00E941B1D8DE59FE00E941B1D8DEC23
:10B090009FE00E941B1D8DEB9FE00E941B1D8DEA0F
:10B0A0009FE00E941B1D8DE99FE00E941B1D8DE00B
:10B0B00090E10E941B1D8DEF9FE00E941B1D8DEEF5
:10B0C0009FE00E941B1D8DED9FE00E941B1D8DE4E3
:10B0D00090E10E941B1D8DE390E10E941B1D8DE2FB
:10B0E00090E10E941B1D8DE190E10E941B1D8DE8E7
:10B0F00090E10E941B1D8DE790E10E941B1D8DE6D3
:10B1000090E10E941B1D8DE590E10E941B1D8DECBE
:10B1100090E10E941B1D8DEB90E10E941B1D8DEAAA
:10B1200090E10E941B1D8DE990E10E941B1D8DE0A6
:10B1300091E10E941B1D8DEF90E10E941B1D8DEE81
:10B1400090E10E941B1D8DED90E10E941B1D8DE47E
:10B1500091E10E941B1D8DE391E10E941B1D8DE278
:10B1600091E10E941B1D8DE191E10E941B1D8DE864
:10B1700091E10E941B1D8DE791E10E941B1D8DE650
:10B1800091E10E941B1D8DE591E10E941B1D8DEC3C
:10B1900091E10E941B1D8DEB91E10E941B1D8DEA28
:10B1A00091E10E941B1D8DE991E10E941B1D8DE024
:10B1B00092E10E941B1D8DEF91E10E941B1D8DEEFF
:10B1C00091E10E941B1D8DED91E10E941B1D8DE4FC
:10B1D00092E10E941B1D8DE392E10E941B1D8DE2F6
:10B1E00092E10E941B1D8DE192E10E941B1D8DE8E2
:10B1F00092E10E941B1D8DE792E10E941B1D8DE6CE
:10B2000092E10E941B1D8DE592E10E941B1D8DECB9
:10B2100092E10E941B1D8DEB92E10E941B1D8DEAA5
:10B2200092E10E941B1D8DE992E10E941B1D8DE0A1
:10B2300093E10E941B1D8DEF92E10E941B1D8DEE7C
:10B2400092E10E941B1D8DED92E10E941B1D8DE479
:10B2500093E10E941B1D8DE393E10E941B1D8DE273
:10B2600093E10E941B1D8DE193E10E941B1D8DE85F
:10B2700093E10E941B1D8DE793E10E941B1D8DE64B
:10B2800093E10E941B1D8DE593E10E941B1D8DEC37
:10B2900093E10E941B1D8DEB93E10E941B1D8DEA23
:10B2A00093E10E941B1D8DE993E10E941B1D8DE01F
:10B2B00094E10E941B1D8DEF93E10E941B1D8DEEFA
:10B2C00093E10E941B1D8DED93E10E941B1D8DE4F7
:10B2D00094E10E941B1D8DE394E10E941B1D8DE2F1
:10B2E00094E10E941B1D8DE194E10E941B1D8DE8DD
:10B2F00094E10E941B1D8DE794E10E941B1D8DE6C9
:10B3000094E10E941B1D8DE594E10C941B1DEF92AE
:10B310000F931F93CF93DF93E80134E047FD34E1AF
:10B32000042E000C550B57FF03C051954195510950
:10B33000E32E022F242FAE01ABD1CE01DF91CF91AE
:10B340001F910F91EF9008950F931F93CF93DF9369
:10B350008230910510F482E090E0E0919714F09132
:10B36000981430E020E0B0E0A0E0309799F4211587
:10B37000310509F44AC0281B390B24303105D8F5B2
:10B380008A819B816115710589F1FB019383828319
:10B39000FE0111C040815181028113814817590774
:10B3A000E0F04817590799F4109761F012960C9342
:10B3B000129713961C933296CF01DF91CF911F9174
:10B3C0000F9108950093971410939814F4CF2115BA
:10B3D000310551F04217530738F0A901DB019A01FA
:10B3E000BD01DF01F801C1CFEF01F9CF90939814AF
:10B3F00080939714CDCFFE01E20FF31F81939193B9
:10B400002250310939832883D7CF20919514309168
:10B410009614232B41F420910402309105023093BD
:10B420009614209395142091020230910302211565
:10B43000310541F42DB73EB7409106025091070205
:10B44000241B350BE0919514F0919614E217F30745
:10B45000A0F42E1B3F0B2817390778F0AC014E5F84
:10B460005F4F2417350748F04E0F5F1F5093961417
:10B4700040939514819391939FCFF0E0E0E09CCFAF
:10B48000CF93DF930097E9F0FC0132971382128289
:10B49000A0919714B0919814ED0130E020E010973E
:10B4A000A1F420813181820F931F20919514309156
:10B4B00096142817390709F061C0F0939614E093A9
:10B4C0009514DF91CF910895EA01CE17DF07E8F5D3
:10B4D0004A815B819E0141155105B1F7E901FB836A
:10B4E000EA8349915991C40FD51FEC17FD0761F408
:10B4F000808191810296840F951FE9019983888349
:10B50000828193819B838A83F0E0E0E012968D91A3
:10B510009C9113970097B9F52D913C911197CD010E
:10B520000296820F931F209195143091961428173C
:10B53000390739F6309751F51092981410929714F4
:10B54000B0939614A0939514BCCFD383C28340814B
:10B550005181840F951FC817D90761F44E5F5F4F63
:10B5600088819981480F591F518340838A819B812B
:10B57000938382832115310509F0B0CFF09398149D
:10B58000E09397149ECFFD01DC01C0CF138212829D
:10B59000D7CF66277727F4C143E954E100C0FA0109
:10B5A000A191B081009719F41097E1F0CD01DC0171
:10B5B000CD010D90002011F4C00113C0FB012191B9
:10B5C000222319F02015D9F7F3CFFB012191201583
:10B5D00019F41E92119606C02223C1F70D90002087
:10B5E000A1F7D001FA01A193B0830895BB274A3097
:10B5F00031F4992322F4BDE2909581959F4F30C09C
:10B60000BB272A3051F4992342F4BDE290958095EE
:10B61000709561957F4F8F4F9F4F01C0BB27FA01F7
:10B62000A62F6217710581059105330B30FB66F07B
:10B63000AA27660F771F881F991FAA1FA21710F04D
:10B64000A21B63953850A9F7A05DAA3308F0A95D45
:10B65000A19336F7B111B1931082CA01DEC3BB27A3
:10B66000FB015527AA27880F991FAA1FA41710F0BE
:10B67000A41B83955051B9F7A05DAA3308F0A95DCA
:10B68000A193009779F7B111B1931192CB01C5C382
:10B690008F929F92AF92BF92CF92DF92EF92FF92E2
:10B6A0000F931F93CF93DF9300D000D000D0CDB77E
:10B6B000DEB76A01F22EB02E102FFBE3AF2EA016DC
:10B6C00008F41BE31F5F012F27E0AE014F5F5F4FC0
:10B6D000ACD2BC018981982F9970913009F44EC089
:10B6E0009BE2E1FC04C09E2D9170E0FC49C05E2D00
:10B6F0005071E82FE87083FF55C084E0911101C0BC
:10B7000083E0EF2DE81B8F1508F0E0E0D6018E2FC7
:10B7100020E25523C9F1992329F0D6019C93C60153
:10B7200001966C0196012D5F3F4FE2FE33C08EE41F
:10B73000D6018C9391E411969C93119712968C9359
:10B74000D9018E2F90E281112AC0E20FF32FF11D53
:10B7500010828EEF9FEF29960FB6F894DEBF0FBED2
:10B76000CDBFDF91CF911F910F91FF90EF90DF90B0
:10B77000CF90BF90AF909F908F9008959DE2B7CFEC
:10B7800090E2B5CF2D9381508111FCCFCE0ED11C0C
:10B79000E0E0C1CF8EE6D6018C9391E6CCCF9D93AD
:10B7A0008150D1CF482F447082FF3DC084E0911179
:10B7B00001C083E08F1510F4EF2DE81BD6018E2F0A
:10B7C00020E2552309F1992329F0D6019C93C60163
:10B7D00001966C0196012D5F3F4FE2FE1BC089E48C
:10B7E000D6018C938EE411968C93119786E4129671
:10B7F0008C93D9018E2F90E2882309F4A6CF9D93D4
:10B800008150FACF2D9381508111FCCFCE0ED11CE7
:10B81000E0E0D9CF89E6D6018C938EE611968C9321
:10B82000119786E6E4CF9B0177FF02C030E020E06D
:10B83000A1E0B0E0911102C0B0E0A0E0F9013196C2
:10B84000AE0FBF1F8B2C912CBB2009F461C054019B
:10B85000EFEFAE1ABE0AAA0DBB1DFA161B0619F0B1
:10B8600014F04F2D4A1B511188C0E3FC59C07601DA
:10B87000A42FB0E2A1114FC0C40ED11C992309F42A
:10B880005BC040E0D6011196F60190836D0155230F
:10B8900009F448C0012F060F9A81582F507184FF78
:10B8A00003C0913309F4015010160CF047C0093061
:10B8B00008F008E0EEE2FE2E5B01A01AB108850157
:10B8C0009194819491082F3F320729F4D601FC927C
:10B8D000F60131966F016217730794F1021713078F
:10B8E0007CF5DB01A21BB30BAA24A394B12CAC0EF4
:10B8F000BD1EAA0DBB1D11968C9121503109D60198
:10B90000119628153905F4F0F60180836D01DBCF1F
:10B91000B12CA12CA0CFF701B1937F01A150AACFE8
:10B920009111B0CFD601942F50E302C05D93915096
:10B930009111FCCFC40ED11C40E0ACCF01E0BACFD6
:10B9400080E3DBCF6217730731F4963388F49533C5
:10B9500011F4552369F0F6018083FD01842F90E2F4
:10B96000811108C0A40FB11D1C9290E080E0F3CEBD
:10B9700081E3F1CF91938150F3CF911183CF8ACF9F
:10B980008F929F92AF92BF92CF92DF92EF92FF92EF
:10B990000F931F93CF93DF935C017B0161157105BA
:10B9A00019F0DB018D939C9385010F5F1F4FF5010B
:10B9B000D0818D2F90E011D26C01892BA9F5DD3259
:10B9C000A9F50F5F1F4FD5011196DC91C1E0580119
:10B9D000F1E0AF1AB10843E050E06CEE70E0C50151
:10B9E00004D2892B61F5680182E0C80ED11C45E0C4
:10B9F00050E067EE70E0C601F8D1892B21F46801B0
:10BA000097E0C90ED11CE114F10419F0D701CD92D1
:10BA1000DC9260E070E080E89FEFC111F9C060E067
:10BA200070E080E89FE7F4C05801BECFDB3229F414
:10BA300085010E5F1F4FF501D181C0E0C8CF43E003
:10BA400050E064EE70E0C501D0D1892BE9F0F80137
:10BA500010E000E020E030E0A9015F01B0ED8B2EA6
:10BA60008D0E89E08815C0F19C2E689491F88C2F7A
:10BA70008870C2FF16C0811102C00F5F1F4F319640
:10BA8000D501DC91C92DE9CFE114F10429F00E5F55
:10BA90001F4FF7011183008360E070E080EC9FE7A7
:10BAA000B7C0882311F001501109A5E0B0E013D30D
:10BAB0009B01AC01220F331F441F551F280D311D60
:10BAC000411D511D283999E93907490799E159075D
:10BAD000B0F2C6609C2ED3CFAEEF8A1206C0C3FD73
:10BAE0003CC09C2E689493F8CACFDF7DD534A9F56D
:10BAF00080818D3239F4C061DF011296818162E06C
:10BB000070E006C0DF018B32C1F3119661E070E096
:10BB100080535D01A61AB70A8A30F8F4E0E8CE1621
:10BB2000ECE0DE065CF4B601660F771F660F771F48
:10BB3000C60ED71ECC0CDD1CC80ED11C5D01FFEF5C
:10BB4000AF1ABF0A8C9180538A3098F1C4FF03C0AA
:10BB5000D194C194D1080C0D1D1DC1FF09C0E11481
:10BB6000F10431F081E0A81AB108D701AD92BC927E
:10BB7000CA01B90166D1C370C33009F490584B01B2
:10BB80005C0120E030E0A90158D1882309F43EC0CF
:10BB9000CBE1D1E017FF05C0119501951109C3E074
:10BBA000D1E06E01B8E1CB1AD10880E2E82EF12C89
:10BBB0000EC0D501B3CFFE01259135914591549129
:10BBC0000E191F09C501B4019DD14B015C01D501BE
:10BBD000C4010E151F057CF72497F594E794CC1645
:10BBE000DD06A9F78A2F880F8B2F881F8F3F41F022
:10BBF00020E030E0A901C501B4011FD1811106C0C8
:10BC000082E290E090939A1480939914C501B40154
:10BC1000DF91CF911F910F91FF90EF90DF90CF9028
:10BC2000BF90AF909F908F900895283008F027E044
:10BC30003327DA01990F311D87FD91600096610568
:10BC4000710539F432602E5F3D9330E32A95E1F7B8
:10BC500008959F3F30F080387105610509F03C5F21
:10BC60003C5F3D93913008F08068911DDF93CF9346
:10BC70001F930F93FF92EF92192F987F9695E92FBC
:10BC800096959695E90FFF27E758FE4F992733279A
:10BC9000EE24FF24A701E70105900894079428F4F7
:10BCA000360FE71EF81E491F511D660F771F881FAC
:10BCB000991F0694A1F70590079428F4E70EF81E43
:10BCC000491F561FC11D770F881F991F661F0694B5
:10BCD000A1F70590079428F4F80E491F561FC71FB7
:10BCE000D11D880F991F661F771F0694A1F7059035
:10BCF000079420F4490F561FC71FD81F990F661FBE
:10BD0000771F881F0694A9F784911095177041F04A
:10BD1000D695C79557954795F794E7941A95C1F727
:10BD2000EFE1F1E068941590159135916591959149
:10BD300005907FE27395E118F10A430B560BC90B8E
:10BD4000D009C0F7E10CF11E431F561FC91FD01DBB
:10BD50007EF4703311F48A95E6CFE894015030F008
:10BD6000080F0AF40027021708F4202F2395022F4A
:10BD70007A3328F079E37D932A95E9F710C07D9313
:10BD80002A9589F606949795679537951795179490
:10BD9000E118F10A430B560BC90BD00998F0239513
:10BDA0007E9173957A3308F070E37C932013B8F793
:10BDB0007E9170617D9330F0839571E37D9370E3A4
:10BDC0002A95E1F71124EF90FF900F911F91CF91E9
:10BDD000DF91992787FD909508959111F6C08032E3
:10BDE00019F089508550D0F70895FB01DC014150CE
:10BDF000504088F08D9181341CF08B350CF4805EBE
:10BE0000659161341CF06B350CF4605E861B61112A
:10BE100071F3990B0895881BFCCFDC01FC01672F9F
:10BE200071917723E1F7329704C07C916D93708311
:10BE30006291AE17BF07C8F3089540D008F481E0BF
:10BE40000895E89409C097FB3EF49095809570950D
:10BE500061957F4F8F4F9F4F9923A9F0F92F96E956
:10BE6000BB279395F695879577956795B795F111CB
:10BE7000F8CFFAF4BB0F11F460FF1BC06F5F7F4F68
:10BE80008F4F9F4F16C0882311F096E911C077237A
:10BE900021F09EE8872F762F05C0662371F096E883
:10BEA000862F70E060E02AF09A95660F771F881F52
:10BEB000DAF7880F9695879597F90895990F0008F6
:10BEC000550FAA0BE0E8FEEF16161706E807F9076C
:10BED000C0F012161306E407F50798F0621B730B07
:10BEE000840B950B39F40A2661F0232B242B252B88
:10BEF00021F408950A2609F4A140A6958FEF811D2B
:10BF0000811D08950BD07BC06CD028F071D018F043
:10BF1000952309F05DC062C01124A5C081D0A0F3B3
:10BF2000959FD1F3950F50E0551F629FF001729FCE
:10BF3000BB27F00DB11D639FAA27F00DB11DAA1FED
:10BF4000649F6627B00DA11D661F829F2227B00D3A
:10BF5000A11D621F739FB00DA11D621F839FA00DC5
:10BF6000611D221F749F3327A00D611D231F849F15
:10BF7000600D211D822F762F6A2F11249F5750406C
:10BF80008AF0E1F088234AF0EE0FFF1FBB1F661F07
:10BF9000771F881F91505040A9F79E3F510570F0C0
:10BFA00017C061C05F3FECF3983EDCF38695779550
:10BFB0006795B795F795E7959F5FC1F7FE2B880FBB
:10BFC000911D9695879597F9089599278827089543
:10BFD00097F99F6780E870E060E008959FEF80EC3C
:10BFE000089500240A9416161706180609060895DF
:10BFF00000240A9412161306140605060895092E45
:10C000000394000C11F4882352F0BB0F40F4BF2BB3
:10C0100011F460FF04C06F5F7F4F8F4F9F4F0895F3
:10C0200057FD9058440F551F59F05F3F71F04795E9
:10C03000880F97FB991F61F09F3F79F087950895CE
:10C04000121613061406551FF2CF4695F1DF08C0ED
:10C05000161617061806991FF1CF8695710561050A
:10C0600008940895E894BB2766277727CB0197F9B2
:10C070000895F999FECF92BD81BDF89A992780B5B0
:10C080000895262FF999FECF1FBA92BD81BD20BD1C
:10C090000FB6F894FA9AF99A0FBE01960895052EF4
:10C0A00097FB16F400940FD057FD05D024D007FC61
:10C0B00002D046F408C050954095309521953F4FE9
:10C0C0004F4F5F4F089590958095709561957F4F84
:10C0D0008F4F9F4F089531D0A59F900DB49F900D25
:10C0E000A49F800D911D11240895B7FFF4CFF3DFB5
:10C0F000821B930B0895A1E21A2EAA1BBB1BFD0104
:10C100000DC0AA1FBB1FEE1FFF1FA217B307E40736
:10C11000F50720F0A21BB30BE40BF50B661F771F8E
:10C12000881F991F1A9469F760957095809590956E
:10C130009B01AC01BD01CF010895A29FB001B39F47
:10C14000C001A39F700D811D1124911DB29F700D20
:10C15000811D1124911D08955058BB27AA270ED088
:10C160004ECF3FDF30F044DF20F031F49F3F11F439
:10C170001EF434CF0EF4E095E7FB2ACFE92F50DF11
:10C1800080F3BA17620773078407950718F071F4F4
:10C190009EF568CF0EF4E0950B2EBA2FA02D0B0163
:10C1A000B90190010C01CA01A0011124FF27591BFC
:10C1B00099F0593F50F4503E68F11A16F040A22F02
:10C1C000232F342F4427585FF3CF46953795279573
:10C1D000A795F0405395C9F77EF41F16BA0B620B72
:10C1E000730B840BBAF09150A1F0FF0FBB1F661FB9
:10C1F000771F881FC2F70EC0BA0F621F731F841FFC
:10C2000048F4879577956795B795F7959E3F08F021
:10C21000B3CF9395880F08F09927EE0F97958795E0
:10C2200008950CD0ECCEE4DE40F0DBDE30F021F4FB
:10C230005F3F19F0CDCE511116CFD0CEF1DE98F37D
:10C240009923C9F35523B1F3951B550BBB27AA2797
:10C2500062177307840738F09F5F5F4F220F331F09
:10C26000441FAA1FA9F333D00E2E3AF0E0E830D0D5
:10C2700091505040E695001CCAF729D0FE2F27D0D8
:10C28000660F771F881FBB1F261737074807AB07A6
:10C29000B0E809F0BB0B802DBF01FF2793585F4F1B
:10C2A0002AF09E3F510568F093CEDDCE5F3FECF360
:10C2B000983EDCF3869577956795B795F7959F5FE0
:10C2C000C9F7880F911D9695879597F90895E1E034
:10C2D000660F771F881FBB1F621773078407BA0793
:10C2E00020F0621B730B840BBA0BEE1F88F7E095EE
:10C2F000089504D06894B111B6CE089599DE88F0FF
:10C300009F5790F0B92F9927B751A0F0D1F0660F41
:10C31000771F881F991F1AF0BA95C9F712C0B1305C
:10C3200081F0A0DEB1E008959DCE672F782F882799
:10C33000B85F39F0B93FCCF3869577956795B3959B
:10C34000D9F73EF490958095709561957F4F8F4F0A
:10C350009F4F0895B3DD08F48FEF0895AFDD880B8C
:10C36000990B0895DB018F939F93B5DEBF91AF9139
:10C37000A29F800D911DA39F900DB29F900D11243F
:10C380000895991B79E004C0991F961708F0961B31
:10C39000881F7A95C9F78095089597FB072E16F4A4
:10C3A000009406D077FD08D013D007FC05D03EF4EA
:10C3B000909581959F4F0895709561957F4F089551
:10C3C000EE0FFF1F881F8BBF0790F691E02D199489
:10C3D000AA1BBB1B51E107C0AA1FBB1FA617B707AB
:10C3E00010F0A61BB70B881F991F5A95A9F78095C7
:10C3F0009095BC01CD0108954F925F926F927F920C
:10C400008F929F92AF92BF92CF92DF92EF92FF9264
:10C410000F931F93CF93DF938C01009799F4CB0177
:10C42000DF91CF911F910F91FF90EF90DF90CF9010
:10C43000BF90AF909F908F907F906F905F904F9044
:10C440000C94A459FC01E60FF71F9C0122503109FE
:10C45000E217F30708F4ADC0D901CD91DC91119733
:10C46000C617D70720F1C530D10578F0CE01049763
:10C470008617970750F0C61BD70B2297C193D1930D
:10C480006D937C93CF010E94405AC801DF91CF91F8
:10C490001F910F91FF90EF90DF90CF90BF90AF90E2
:10C4A0009F908F907F906F905F904F9008955B0169
:10C4B000AC1ABD0A4C018C0E9D1EA0919714B09130
:10C4C0009814512C412CF12CE12C109731F58091CE
:10C4D0009514909196148815990509F05CC046163C
:10C4E000570608F058C0809102029091030200970D
:10C4F00041F48DB79EB74091060250910702841B0C
:10C50000950BE817F90708F054C0F0939614E093E0
:10C510009514F90171836083B8CF8D919C91119727
:10C5200012966C90129713967C901397A815B905E4
:10C5300059F56C0142E0C40ED11CCA14DB0420F191
:10C54000AC014A195B09DA011296159780F06282F4
:10C55000738251834083D9016D937C93E114F1047C
:10C5600071F0D7011396FC93EE9312978ECF22961B
:10C570008C0F9D1FF90191838083F301EFCFF0931E
:10C580009814E093971481CF4816590608F42C01AB
:10C590007D01D3019ACFCB010E94A4597C01009761
:10C5A00041F0AE01B80108D0C8010E94405A87018D
:10C5B0006CCF10E000E069CFFB01DC0102C001900C
:10C5C0000D9241505040D8F70895FB01DC018D9148
:10C5D000019080190110D9F3990B0895FB01DC013A
:10C5E00001900D920020E1F7089511E0CEE9D1E02D
:10C5F00000E005C0802FFE01E3DE2196011DCF394A
:0CC60000D10780E00807B1F7F894FFCFE5
:10C60C00FFFF00009B1480002E452E65787072652C
:10C61C0073734B3130000001000000010000000179
:10C62C00000000200A0D0000362E352E323200009C
:10C63C005238350052383400523035005231330004
:10C64C005231320052313100523137005231360002
:10C65C0052313500523034005238370052373300E3
:10C66C0052373200523731000D0A0020005239394E
:10C67C00000D0A0020005239390000000000FE14A1
:10C68C002B1D1A2D00000000FF142D1DAE1A0000EA
:10C69C00000000152F1D161D000000000115311D96
:10C6AC00E91A000000000215331D241500000000DB
:10C6BC000315351D8815000000000415371DC21523
:10C6CC00000000000515391D4E1A0000000006156B
:10C6DC003B1DCF150000000007153D1DC4290000AF
:10C6EC00000008153F1D302A000000000915411DEF
:10C6FC003E2A000000000A15431D8C420000000079
:10C70C000B15451DC542000000000C15471DFE42CF
:10C71C00000000000D15491D3743000000000E15E8
:10C72C004B1D3445000000000F154D1D0547000042
:10C73C00000010154F1D691600000000FC14231D8D
:10C74C00A84100000000FD14291D50425230330056
:10C75C0052303200523037005230310052303900F2
:10C76C0052383800523837005230380052383800BE
:10C77C005230300052383700523036000000000082
:10C78C002E089907C6077E08F707D507E9070000AA
:10C79C000000F814251D52393900207374612000F3
:10C7AC0020637572200020656E6420002068616C27
:10C7BC00662000206C656E2000206D696E200020C4
:10C7CC006D61782000207370642000205100523479
:10C7DC003100500052323100523939204572726F9B
:10C7EC00723A20696E76616C696420706172616D59
:10C7FC00657465722069640D0A0052383320002D6F
:10C80C00383966626431373900523831002058416A
:10C81C0000205842002059410020594200205A4122
:10C82C0000205A4200686F6D650D0A006E616E0043
:10C83C00696E66006F7666005238320052323000F4
:10C84C005239392057696C6C207A65726F20580008
:10C85C005239392057696C6C207A65726F205900F7
:10C86C005239392057696C6C207A65726F205A00E6
:10C87C007469636B2064656C6179004D4F56454D4E
:10C88C00454E545F494E544552525550545F535087
:10C89C00454544007370656564486F6D655B6178F0
:10C8AC0069735D005239392043616C69627261743D
:10C8BC00696F6E206572726F723A20656E642073B8
:10C8CC00746F7020616374697665206265666F723F
:10C8DC00652073746172740D0A002061786973208D
:10C8EC0000206D6F766520746F20737461727420F4
:10C8FC00666F722063616C6962726174696F6E003D
:10C90C005239392074696D656F75742058206178BF
:10C91C0069730D0A005239392074696D656F75742D
:10C92C00205920617869730D0A00523939207469D5
:10C93C006D656F7574205A20617869730D0A005209
:10C94C00393920656D657267656E63792073746F14
:10C95C00700D0A00523939206D6F76656D656E74F5
:10C96C0020646F6E650D0A0020617420737461720F
:10C97C0074696E6720706F696E74005232330020D8
:10C98C0063616C6962726174696E67206C656E6755
:10C99C00746800207374657020636F756E743A2030
:10C9AC000020617420656E6420706F696E740020C5
:10C9BC0064656163746976617465206D6F746F7200
:10C9CC0020582064756520746F2000647269766548
:10C9DC0072206572726F72006D6973736564207377
:10C9EC007465707300206465616374697661746545
:10C9FC00206D6F746F7220592064756520746F20E0
:10CA0C00002064656163746976617465206D6F7470
:10CA1C006F72205A2064756520746F20005239396A
:10CA2C00206572726F720D0A00205500205600208E
:10CA3C0057005239392073746F707065640D0A0099
:10CA4C00523939207265736574206D6F746F722062
:10CA5C00580D0A00523939207265736574206D6F58
:10CA6C00746F7220590D0A00523939207265736542
:10CA7C0074206D6F746F72205A0D0A005239392070
:10CA8C006572726F72200052393920686F6D696E51
:10CA9C006720646973706C616365640020582000C2
:10CAAC00202F200020592000205A2000204D20004B
:10CABC0053657269616C20636F6E6E656374696F28
:10CACC006E20737461727465640053657420696EB2
:10CADC007075742F6F7574707574206661726D62E9
:10CAEC006F74206578707265737300526561642091
:10CAFC00706172616D6574657273004C6F61642056
:10CB0C00544D43206472697665727300496E697482
:10CB1C0020544D4332313330206472697665727320
:10CB2C00004C6F616420544D4332313330207061BE
:10CB3C0072616D6574657273004C6F6164206D6F0A
:10CB4C0076656D656E742073657474696E677300B9
:10CB5C00536574206D6F746F7220656E61626C65C5
:10CB6C0073206F66660053746172742070696E2056
:10CB7C00677561726400537461727420696E7465B8
:10CB8C00727275707400436865636B20686F6D69B1
:10CB9C006E67206F6E20626F6F74005239392048B7
:10CBAC004F4D45205A204F4E20535441525455500E
:10CBBC000D0A0052393920484F4D452059204F4E0F
:10CBCC0020535441525455500D0A005239392048C3
:10CBDC004F4D452058204F4E2053544152545550E0
:10CBEC000D0A0041524455494E4F20535441525462
:10CBFC00555020434F4D504C455445002A0047306A
:10CC0C0000473030004731004730310047323800A0
:10CC1C004630390046390046313100463132004643
:10CC2C00313300463134004631350046313600464A
:10CC3C003230004632310046323200463331004643
:10CC4C003332004634310046343200463433004629
:10CC5C00343400463631004638310046383200460E
:10CC6C0038330046383400200A0D00523939206818
:10CC7C00616E646C6572203D3D204E554C4C0D0A26
:10CC8C000020726573657474696E672064696769E6
:10CC9C0074616C2070696E002072657365747469C0
:0ECCAC006E6720616E616C6F672070696E00AC
:00000001FF
